:100000000C94E7140C9418150C9418150C941815EE
:100010000C9418150C9418150C9418150C941815AC
:100020000C9418150C9418150C9418150C9418159C
:100030000C9418150C94FB510C9418150C9418156D
:100040000C9418150C9473470C9418150C941815EF
:100050000C9418150C9418150C9479750C94B151D6
:100060000C9418150C9499C60C9418150C9418152A
:100070000C9418150C9418150C9418150C9418154C
:100080000C9418150C9418150C9418150C9418153C
:100090000C9418150C9418150C9418150C9418152C
:1000A0000C9418150C9418150C9418150C9418151C
:1000B0000C9418150C9418150C9418150C9418150C
:1000C0000C9418150C9418150C9418150C941815FC
:1000D0000C9418150C9418150C9400470C94C146F8
:1000E0000C941815F72B142C452C622C772CA02C73
:1000F0000D2D732D1C2E643272326B329232963279
:10010000B0320A37C532113338335F338833DD33C9
:10011000EE33FF331034213432340A3715360A37C0
:10012000203690369636B636F7A3FAA3E9A3EDA3A8
:10013000F3A331A4FEA302A408A40CA410A416A443
:100140001AA41EA431A424A428A42CA494A999A977
:100150009EA9A8A9B2A92BAABCA9C4A9CCA9D6A911
:10016000E0A9EAA9F9A903AA2BAA0DAA17AA21AA0C
:10017000084AD73B3BCE016E84BCBFFDC12F3D6C0E
:1001800074319ABD56833DDA3D00C77F11BED9E474
:10019000BB4C3E916BAAAABE000000803F05A84C54
:1001A000CDB2D44EB93836A9020C50B99186880820
:1001B0003CA6AAAA2ABE000000803F004E414E493C
:1001C0004E495459494E46CDCCCC3D0AD7233C1715
:1001D000B7D13877CC2B329595E6241FB14F0A0062
:1001E0000020410000C84200401C4620BCBE4CCA52
:1001F0001B0E5AAEC59D74434F4D4D554E4943415C
:1002000054494F4E0044525952554E004552524F98
:10021000525300494E464F004543484F0047322F46
:1002200047332062616420706172616D657465722C
:10023000730A00206F6620004D424C20473239205F
:10024000706F696E74200059206F7574206F66207E
:1002500072616E67652028312D35292E0A005820DD
:100260006F7574206F662072616E67652028312D6E
:1002700035292E0A004D6573682070726F62696EB1
:100280006720646F6E652E0A005374617274206D6E
:100290006573682070726F62696E67207769746831
:1002A0002022473239205331222066697273742E1E
:1002B0000A004732380A47323920533200537461FA
:1002C00074653A20004D65736820626564206C6532
:1002D00076656C696E6720686173206E6F2064615B
:1002E00074612E0A0053206F7574206F662072614E
:1002F0006E67652028302D35292E0A004D657368FC
:1003000020706F696E742063616E6E6F7420626519
:10031000207265736F6C7665640A00456E642066B2
:10032000696C65206C6973740A00426567696E20A8
:1003300066696C65206C6973740A00286E6F2066AC
:10034000696C6529005344207072696E74696E6728
:10035000206279746520004E6F74205344207072BF
:10036000696E74696E670A0043757272656E7420F7
:1003700066696C653A200046696C652064656C6549
:100380007465643A0044656C6574696F6E206661DB
:10039000696C65642C2046696C653A200025697398
:1003A0000025696D20256973002569682025696D20
:1003B0002025697300256964202569682025696DF9
:1003C00020256973002569792025696420256968DD
:1003D0002025696D20256973005072696E74207440
:1003E000696D653A20006F6E2E0A006F66662E0AF0
:1003F00000473236204465627567200018021302F8
:100400000C020502F7016F66660044454255473A03
:10041000004B494C4C45442E20004D313133205384
:10042000006F6B002C20002C2000544845524D4199
:100430004C5F50524F54454354494F4E0041555420
:100440004F5245504F52545F53445F53544154559B
:100450005300454D455247454E43595F5041525315
:10046000455200434153455F4C494748545F42520F
:10047000494748544E45535300544F47474C455FF6
:100480004C494748545300534F4654574152455FD7
:10049000504F574552004255494C445F50455243D6
:1004A000454E54004C4556454C494E475F444154D7
:1004B00041005A5F50524F4245004155544F4C4500
:1004C00056454C005052494E545F4A4F42005052DC
:1004D0004F4752455353004155544F5245504F5288
:1004E000545F54454D5000564F4C554D455452495C
:1004F0004300454550524F4D0053455249414C5FD2
:10050000584F4E5F584F4646004649524D5741524C
:10051000455F4E414D453A4D61726C696E20312EFA
:10052000312E3920284769746875622920534F5548
:100530005243455F434F44455F55524C3A6874748B
:1005400070733A2F2F6769746875622E636F6D2F11
:100550004D61726C696E4669726D776172652F4D7F
:1005600061726C696E2050524F544F434F4C5F562E
:10057000455253494F4E3A312E30204D4143484960
:100580004E455F545950453A3344205072696E7459
:1005900065722045585452554445525F434F554E5D
:1005A000543A3120555549443A63656465326132A5
:1005B000662D343161322D343734382D3962313281
:1005C0002D6335356336326633363766660A002F5B
:1005D0002F2000205400205200416363656C657237
:1005E0006174696F6E3A2050005741524E494E4730
:1005F00021204C6F77205A204A65726B206D6179FB
:10060000206C65616420746F20756E77616E74650F
:1006100064207061757365732E0A00546F6F2066D5
:1006200061722066726F6D207265666572656E63B9
:100630006520706F696E740A00205A0020590058B6
:100640000020204D61783A2000205A00205900589F
:100650000020204D696E3A20004F6E20004F6666E4
:1006600000536F667420656E6473746F70733A2004
:100670000020466C6F773A20000001363726032BA6
:10068000FFFFFF3C3D382AFFFFFFFF2E303E12FFE9
:10069000FFFFFFFFFFFF0809FF2C071A1C18FFFFD1
:1006A000FF08440A2C4324221E20643A0020693AA1
:1006B0000020703A00496E76616C69642065787438
:1006C00072756465720A0043290A0061626C656490
:1006D00020286D696E2074656D702000436F6C6416
:1006E00020657874727564657320617265200020DE
:1006F000643A0020693A0020703A004E6F2063612E
:100700007365206C696768740A00454550524F4D07
:10071000204F4B0A00205A004475616C20456E64DE
:1007200073746F702041646A7573746D656E7420A4
:10073000286D6D293A20003F4B2076616C7565204D
:100740006F7574206F662072616E67652028302D8A
:100750003130292E0A00416476616E6365204B3D7D
:1007600000416374697665204578747275646572BA
:100770003A2000496E76616C696420657874727500
:100780006465720A0043616E6E6F7420656E7465F5
:1007900072207375626469723A20004739310A47E2
:1007A00031205A2D302E30320A47393000537065CF
:1007B0006369616C204D656E753A205A20446F77ED
:1007C0006E20302E310A004739310A4731205A2D28
:1007D000302E30320A473930005370656369616CDE
:1007E000204D656E753A205A20446F776E20302E6A
:1007F00030320A004739310A4731205A2B302E3027
:10080000320A473930005370656369616C204D6569
:100810006E753A205A20557020302E30320A00472B
:1008200039310A4731205A2B302E310A47393000EE
:100830005370656369616C204D656E753A205A206E
:10084000557020302E310A00473239205332005380
:1008500070656369616C204D656E753A204E6578F0
:1008600074204D65736820506F696E740A004732BA
:1008700039205331005370656369616C204D656E9A
:10088000753A205374617274204D657368204C650D
:1008900076656C696E670A004D313430205336300E
:1008A000005370656369616C204D656E753A205028
:1008B000726568656174204265640A004D353031A7
:1008C000005370656369616C204D656E753A205206
:1008D00065616420454550524F4D0A004D3530301A
:1008E000005370656369616C204D656E753A2053E5
:1008F00061766520454550524F4D0A004D333033E7
:1009000020452D31205338302043382055310053B5
:1009100070656369616C204D656E753A2041757430
:100920006F2054756E6520486F746265642050694D
:10093000640A004D31303620533137380A4D333098
:100940003320453020533234302043382055310095
:100950005370656369616C204D656E753A20417511
:10096000746F2054756E6520486F74656E642050F6
:1009700049440A003C5370656369616C5F4D656E64
:10098000753E003C5370656369616C5F4D656E75C3
:100990003E002F002F002F002F2E2E0A002F2E2E6C
:1009A000002F2E2E003C5370656369616C5F4D65AE
:1009B0006E753E0A003C5370656369616C204D653D
:1009C0006E753E003C5370656369616C204D656EC9
:1009D000753E003C5265616420454550524F4D3E86
:1009E000003C5265616420454550524F4D3E003CED
:1009F0004175746F2054756E6520486F746265642C
:100A0000205049443E003C4175746F2054756E651A
:100A100020486F74626564205049443E003C417533
:100A2000746F2054756E6520486F74656E64205035
:100A300049443E003C4175746F2054756E652048F2
:100A40006F74656E64205049443E003C457869747B
:100A50003E003C457869743E003C53617665204514
:100A60004550524F4D3E003C536176652045455000
:100A7000524F4D3E003C4E657874204D65736820A2
:100A8000506F696E743E003C4E657874204D6573FE
:100A90006820506F696E743E003C5374617274201C
:100AA0004D657368204C6576656C696E673E003CE9
:100AB0005374617274204D657368204C6576656C63
:100AC000696E673E003C50726568656174206265BE
:100AD000643E003C50726568656174206265643EE6
:100AE000003C5A20446F776E20302E313E003C5A35
:100AF00020446F776E20302E313E003C5A20446FE8
:100B0000776E20302E30323E003C5A20446F776E94
:100B100020302E30323E003C5A20557020302E308E
:100B2000323E003C5A20557020302E30323E003C80
:100B30005A20557020302E313E003C5A20557020EE
:100B4000302E313E0056313136004A333320004DCD
:100B50003530300A4D3432302053310A4731205A73
:100B6000313020463234300A473120583020593055
:100B7000204636303030004A3232004A32320047A6
:100B800031205A3520463234300A47312058313925
:100B900030205932302046363030300A4731205A22
:100BA000302046323430004731205A352046323426
:100BB000300A4731205831393020593139302046F8
:100BC000363030300A4731205A3020463234300037
:100BD0004731205A3520463234300A4731205831C7
:100BE0003930205932302046363030300A473120F3
:100BF0005A302046323430004739310A4731205AC2
:100C0000313020463234300A4739300A4732380A08
:100C10004732390A47312058323020593230204685
:100C2000363030300A4731205A30204632343000D6
:100C30004A3032004A3132004731205A3130004FB9
:100C40004B004731205A31300047393000473120BE
:100C50004525694635303000473120452D302E314D
:100C60004625690047312045302E31462569004729
:100C700031205A2569462569004731205A2D302EEA
:100C800031462569004731205A302E31462569000A
:100C900047312059256946256900473120592D30B3
:100CA0002E314625690047312059302E31462569BD
:100CB0000047312058256946256900473120582DC5
:100CC000302E314625690047312058302E314625D7
:100CD00069004739310047323800473238205A001E
:100CE00047323820590047323820580041323056B8
:100CF00020004731205A3130004A3034004A323126
:100D0000004A3230004B494C4C45442E20004A30BA
:100D10003400454E4400464E20004A3032003939F6
:100D2000393A393939004D004800413756200041E1
:100D30003656202D2D2D004A3032004136562000E7
:100D40005A3A2000593A2000583A200041355600BE
:100D50004134562000413356200041325620004194
:100D60003156200041305620004D3834004A31368B
:100D7000004A3138004739310A4731205A31302092
:100D8000463234300A473930004A3134004A303074
:100D9000004A3031004A313000696E206D6F76654F
:100DA0005F746F282920666565645F76616C756580
:100DB00020666F722058593A002C2065793D002931
:100DC000202D3E202865783D002C2073793D0020A1
:100DD000436F6E6E656374696E672077697468200F
:100DE000766572746963616C206C696E6520287326
:100DF000783D002C2065793D0029202D3E20286576
:100E0000783D002C2073793D0020436F6E6E656342
:100E100074696E67207769746820686F72697A6F89
:100E20006E74616C206C696E65202873783D003F9C
:100E300053706563696669656420582C5920636F37
:100E40006F7264696E617465206F7574206F6620BF
:100E5000626F756E64732E0A003F285229657065B3
:100E600061742076616C7565206E6F7420706C61A2
:100E7000757369626C653B206D75737420626520C3
:100E80006174206C6561737420312E0A003F285212
:100E9000296570656174206D7573742062652073B7
:100EA0007065636966696564207768656E206E6F3A
:100EB00074207573696E6720616E204C43442E0A5E
:100EC000003F537065636966696564206E6F7A7A66
:100ED0006C652074656D7065726174757265206EE5
:100EE0006F7420706C61757369626C652E0A003FC7
:100EF0005370656369666965642066696C616D65D8
:100F00006E742073697A65206E6F7420706C6175E1
:100F10007369626C652E0A003F5370656369666988
:100F20006564207072696D65206C656E67746820F9
:100F30006E6F7420706C61757369626C652E0A0047
:100F40003F5072696D65206C656E677468206D75C1
:100F500073742062652073706563696669656420D7
:100F60007768656E206E6F74207573696E67206197
:100F70006E204C43442E0A003F53706563696669D6
:100F80006564206E6F7A7A6C652073697A65206E6D
:100F90006F7420706C61757369626C652E0A003F16
:100FA0005370656369666965642052657472616334
:100FB00074696F6E204D756C7469706C6965722010
:100FC0006E6F7420706C61757369626C652E0A00B7
:100FD0003F52657472616374696F6E204D756C74F5
:100FE00069706C696572206D757374206265207319
:100FF00070656369666965642E0A003F53706563B6
:101000006966696564206C617965722068656967E5
:101010006874206E6F7420706C61757369626C65A2
:101020002E0A003F537065636966696564206265D6
:10103000642074656D7065726174757265206E6F81
:101040007420706C61757369626C65202834302D72
:1010500031343043292E0A0047323620636F6D6DDC
:10106000616E6420737461727465642E20576169C7
:1010700074696E6720666F72206865617465722896
:1010800073292E0A0024F4D43050C38E20C2A2400B
:1010900017828B7011127A910D816CD90AA861E1C7
:1010A00008C7586607615143061E4B5D05C145A739
:1010B000041A411104093D9803713931034036DBAC
:1010C0000265339102D4305402802E1D02632CEE4F
:1010D00001752AC501B028A001102781018F256460
:1010E000012B244B01E0223401AC211F018D200D86
:1010F00001801FFC00841EED00971DDF00B81CD28C
:1011000000E61BC600201BBC00641AB200B219A87E
:10111000000A19A0006A189900D117910040178B96
:1011200000B516840031167E00B31579003A1573A8
:1011300000C7146F0058146A00EE1366008813632A
:101140000025135E00C7125B006C12570015125485
:1011500000C111510070114F0021114B00D61049F0
:10116000008D1047004610440002104200C00F409E
:1011700000800F3E00420F3C00060F3B00CB0E38B4
:1011800000930E37005C0E3500270E3400F30D324D
:1011900000C10D3100900D3000600D2E00320D2D7C
:1011A00000050D2C00D90C2B00AE0C2900850C2954
:1011B000005C0C2700350C27000E0C2600E80B24E1
:1011C00000C40B2400A00B23007D0B23005A0B212D
:1011D00000390B2100180B2000F80A1F00D90A1E45
:1011E00000BB0A1E009D0A1D00800A1D00630A1C28
:1011F00000470A1B002C0A1B00110A1A00F7091AE3
:1012000000DD091900C4091900AB0919009209177A
:10121000007B091800630917004C091600360916EF
:1012200000200916000A091500F5081500E0081449
:1012300000CC081400B8081400A408140090081387
:10124000007D0812006B08130058081200460812AF
:1012500000340811002308110012081100010811C0
:1012600000F0071000E0071000D0071000C00710C2
:1012700000B0070F00A107100091070E0083070FB1
:101280000074070F0065070E0057070E0049070E90
:10129000003B070D002E070E0020070D0013070D61
:1012A0000006070D00F9060C00ED060D00E0060C27
:1012B00000D4060C00C8060C00BC060C00B0060CDE
:1012C00000A4060B0099060C008D060B0082060B8D
:1012D0000077060B006C060B0061060A0057060B30
:1012E000004C060A0042060A0038060A002E060ACA
:1012F0000024060A001A060A001006090007060A5A
:1013000000FD050900F4050900EB050900E20509E7
:1013100000D9050900D0050900C7050900BE050967
:1013200000B5050800AD050800A50509009C0508E5
:1013300000940508008C050800840508007C050859
:1013400000740508006C050700650508005D0507C9
:1013500000560508004E0507004705070040050830
:101360000038050700310507002A05070023050797
:10137000001C050600160507000F050700080506F6
:101380000002050700FB040600F5040700EE040652
:1013900000E8040600E2040700DB040600D50406AA
:1013A00000CF040600C9040600C3040600BD0406FD
:1013B00000B7040600B1040500AC040600A604064C
:1013C00000A00405009B0406009504050090040697
:1013D000008A04050085040500800406007A0405DF
:1013E0000075040500700405006B04050066040523
:1013F00000610405005C0405005704050052040563
:10140000004D04050048040500430405003E0404A3
:10141000003A04050035040500300404002C0405DE
:101420000027040400230405001E0404001A040419
:101430000016040500110404000D0404000904054D
:10144000000404040000040400FC030400F8030486
:1014500000F4030400F0030400EC030400E80304B8
:1014600000E4030400E0030400DC030400D80304E8
:1014700000D4030400D0030400CC030400C8030319
:1014800000C503030024F404D9201BC40C5C0E988F
:1014900004C4095F0265077101F405F900FB04B398
:1014A0000048048700C10369005803550003034541
:1014B00000BE023A008402310053022A00290225AC
:1014C0000004022000E4011C00C8011900AF01174C
:1014D00000980114008401130071011000610110D3
:1014E0000051010E0043010D0036010B002B010BD2
:1014F0000020010B00150109000C0109000301087F
:1015000000FB000800F3000800EB000700E4000601
:1015100000DE000600D8000600D2000600CC000560
:1015200000C7000500C2000500BD000400B90004AA
:1015300000B5000400B1000400AD000400A90004DF
:1015400000A5000300A20003009F0004009B00030D
:101550000098000300950002009300030090000330
:10156000008D0002008B000300880002008600024C
:101570000084000300810002007F0002007D000261
:10158000007B000200790002007700010076000273
:10159000007400020072000100710002006F00027E
:1015A000006D0001006C0002006A00010069000289
:1015B0000067000100660001006500010064000290
:1015C000006200010061000100600001005F000294
:1015D000005D0001005C0001005B0001005A000199
:1015E0000059000100580001005700010056000199
:1015F0000055000100540001005300000053000199
:10160000005200010051000100500001004F000194
:10161000004E0000004E0001004D0001004C000192
:10162000004B0000004B0001004A0001004900018E
:10163000004800000048000100470001004600008B
:101640000046000100450000004500010044000183
:10165000004300000043000100420000004200017E
:10166000004100000041000100400001003F000077
:10167000003F0001003E0000003E0001003D000070
:10168000003D0001003C0000003C0000003C000167
:10169000003B0000003B0001003A0000003A00015E
:1016A0000039000000390001003800000038000057
:1016B000003800010037000000370001003600004C
:1016C0000036000000360001003500000035000043
:1016D0000035000100340000003400000034000137
:1016E000003300000033000000330001003200002E
:1016F0000032000000320001003100000031000023
:101700000031000100300000003000000030000116
:10171000002F0000002F0000002F0000002F00010C
:10172000002E0000002E0000002E0001002D000001
:10173000002D0000002D0000002D0001002C0000F5
:10174000002C0000002C0000002C0001002B0000E9
:10175000002B0000002B0000002B0001002A0000DD
:10176000002A0000002A0000002A000100290000D1
:1017700000290000002900000029000000290001C4
:1017800000280000002800000028000000280000B9
:1017900000280001002700000027000000270000AB
:1017A000002700000027000100260000002600009E
:1017B0000026000000260000002600010025000091
:1017C0000025000000250000002500000025000085
:1017D0000025000100240000002400000024000077
:1017E000002400000024000100230000002300006A
:1017F000002300000023000000230000002300005D
:10180000002300010022000000220000002200004E
:101810000022000000220000002200010021000040
:101820000021000000210000002100000021000034
:101830000021000000210001002000000020000025
:101840000020000000200000002000000020000018
:101850000020000000200001001F0000001F000009
:10186000001F0000001F0000001F0000001F0000FC
:10187000001F0001001E0000001E0000001E0000EE
:10188000001E000000C23100001C260000F41900F8
:1018900000D80F0000EB080000C004000075020033
:1018A0000040010000024A3135004A3132004A311D
:1018B00037002020506C616E6E65724275666665F9
:1018C0007242797465733A20002046726565204D36
:1018D000656D6F72793A2000436F6D70696C656455
:1018E0003A204E6F7620323420323031380A0020D0
:1018F0007C20417574686F723A202864617669644F
:1019000072616D69726F2C20666F7220416E79630F
:1019100075626963206933204D656761290A003269
:101920003031392D31312D313500204C6173742027
:10193000557064617465643A2000312E312E390A85
:10194000004D61726C696E0020536F66747761722E
:10195000652052657365740A00205761746368647A
:101960006F672052657365740A002042726F776E4C
:10197000206F75742052657365740A002045787471
:1019800065726E616C2052657365740A00506F77E2
:10199000657255700A0073746172740A004D3234B6
:1019A000004D3233202573006175746F25692E67F1
:1019B000006572726F722077726974696E67207445
:1019C0006F2066696C650A00205A3A0020593A0077
:1019D00020583A00656E6473746F70732068697480
:1019E0003A2000446F6E6520736176696E672066E9
:1019F000696C652E0A004D32390020746F6F206CBF
:101A00006F6E6720657874727573696F6E2070727F
:101A10006576656E7465640A0020636F6C6420658A
:101A20007874727573696F6E2070726576656E7406
:101A300065640A00454550524F4D206461746173DE
:101A4000697A65206572726F722E0A00290A002079
:101A500062797465733B206372632000536574740C
:101A6000696E67732053746F726564202800290AB9
:101A7000002062797465733B2063726320002073D9
:101A8000746F7265642073657474696E6773207215
:101A90006574726965766564202800202863616C2E
:101AA00063756C6174656429210A0020213D200062
:101AB000454550524F4D20435243206D69736D612F
:101AC000746368202D202873746F72656429200068
:101AD0002053697A653A2000496E6465783A20009F
:101AE000204D61726C696E3D563535290A002845D6
:101AF0004550524F4D3D00454550524F4D20766563
:101B00007273696F6E206D69736D61746368200014
:101B10006F70656E206661696C65642C2046696C27
:101B2000653A200043616E6E6F74206F70656E20A1
:101B300073756264697220004A3035004A3233009E
:101B40004739310A4731205A2D313020463234305E
:101B50000A4739300053442063617264206F6B0A76
:101B6000006F70656E526F6F74206661696C65649A
:101B70000A00766F6C756D652E696E6974206661FA
:101B8000696C65640A004572726F723A00534420B2
:101B9000696E6974206661696C0A006563686F3AF2
:101BA000001000C90210012C01400122017001182F
:101BB00001B0010E01F00104015002FA00B002F080
:101BC000003003E600D003DC009004D2007005C8AA
:101BD00000A006BE000008B400B009AA00D00BA007
:101BE00000600E960060118C0000158200201978AC
:101BF00000C01D6E00A0226400B0275A00902C5037
:101C00000000314600E0343C0010383200903A28A1
:101C100000603C1E00A03D1400803E0A00203F00F2
:101C2000002CFFFFFFFFFF0001010101016265645D
:101C30000A002C2073797374656D2073746F707053
:101C4000656421204865617465725F49443A2000EB
:101C50004265642068656174696E67206661696CBD
:101C600065640048656174696E67206661696C65CA
:101C7000640045312048656174696E67206661695A
:101C80006C65640048656174696E67206661696CA3
:101C900065640070012C0190012701B0012201C090
:101CA000011D01F00118011002130130020E016044
:101CB00002090190020401C002FF000003FA004083
:101CC00003F5008003F000D003EB002004E6007071
:101CD00004E100E004DC004005D700C005D200406C
:101CE00006CD00D006C8008007C3003008BE00F053
:101CF00008B900C009B400B00AAF00B00BAA00D008
:101D00000CA500000EA000500F9B00C010960050C4
:101D100012910000148C00C0158700B0178200B02B
:101D2000197D00D01B7800001E730040206E0090CB
:101D3000226900F024640040275F0090295A00E0E7
:101D40002B5500102E500020304B0010324600E082
:101D500033410090353C001037370070383200A016
:101D6000392D00B03A2800A03B2300603C1E001033
:101D70003D1900903D1400103E0F00703E0A00C057
:101D80003E0500003F0000403FFBFF803FF6FFC0E4
:101D90003FF1FF453120544845524D414C205255AA
:101DA0004E415741590042454420544845524D4107
:101DB0004C2052554E4157415900546865726D612F
:101DC0006C2052756E6177617900453120457272E1
:101DD0003A204D415854454D50004572723A204DBD
:101DE000415854454D5020424544004D41585445BA
:101DF0004D502074726967676572656400453120D3
:101E00004572723A204D494E54454D50004572720C
:101E10003A204D494E54454D5020424544004D49CD
:101E20004E54454D50207472696767657265640051
:101E30004D383420582059205A204500202F0020AA
:101E400042403A0020403A004A3038004A303900D7
:101E500020573A00205A3A0020593A0020436F7523
:101E60006E7420583A0020453A00205A3A00205912
:101E70003A00583A003A004361703A004B6420003F
:101E800023646566696E652044454641554C545F40
:101E9000004B69200023646566696E6520444546F1
:101EA00041554C545F004B70200023646566696E99
:101EB000652044454641554C545F005049442041FB
:101EC00075746F74756E652066696E697368656494
:101ED000212050757420746865206C617374204BE8
:101EE000702C204B6920616E64204B6420636F6E00
:101EF0007374616E74732066726F6D2062656C6FAF
:101F00007720696E746F20436F6E666967757261C2
:101F100074696F6E2E680A00504944204175746FD1
:101F200074756E65206661696C6564212074696DE5
:101F3000656F75740A00453120544845524D414C37
:101F40002052554E4157415900424544205448457E
:101F5000524D414C2052554E4157415900546865ED
:101F6000726D616C2052756E617761790045312028
:101F700048656174696E67206661696C65640042DA
:101F800065642068656174696E67206661696C6567
:101F9000640048656174696E67206661696C656498
:101FA00000504944204175746F74756E65206661F8
:101FB000696C6564212054656D7065726174757219
:101FC0006520746F6F20686967680A00204B643A67
:101FD0002000204B693A2000204B703A20000A2054
:101FE000436C617373696320504944200A00205494
:101FF000753A2000204B753A2000206D61783A2018
:1020000000206D696E3A200020643A200020626949
:1020100061733A2000504944204175746F74756EA5
:1020200065206661696C6564212042616420657881
:10203000747275646572206E756D6265720A005007
:102040004944204175746F74756E652073746172B4
:10205000740A004F66660A00466164652048656937
:102060006768742000426564204C6576656C696E13
:102070006720004661696C656420746F20656E613D
:10208000626C6520426564204C6576656C696E679C
:102090000A004D65736820426564204C6576656C66
:1020A00020646174613A0A004D65736820706F693D
:1020B0006E742063616E6E6F74206265207265734A
:1020C0006F6C7665640A004D34323120696E636F3F
:1020D000727265637420706172616D6574657220DF
:1020E00075736167650A00656E7175657565696E02
:1020F000672022004B494C4C45442E200050726909
:102100006E7465722073746F707065642064756599
:1021100020746F206572726F72732E20466978206A
:10212000746865206572726F7220616E64207573C9
:1021300065204D39393920746F207265737461726E
:10214000742E202854656D706572617475726520F7
:1021500069732072657365742E20536574206974E9
:102160002061667465722072657374617274696E41
:1021700067290A004E6F20436865636B73756D2095
:1021800077697468206C696E65206E756D62657222
:102190002C204C617374204C696E653A20004E6FA0
:1021A00020436865636B73756D2077697468206C74
:1021B000696E65206E756D6265722C204C6173745A
:1021C000204C696E653A2000636865636B73756DBA
:1021D000206D69736D617463682C204C6173742089
:1021E0004C696E653A20004C696E65204E756D62D3
:1021F0006572206973206E6F74204C617374204C7B
:10220000696E65204E756D6265722B312C204C61B4
:102210007374204C696E653A20004D313130004DA9
:1022200033310053442072656164206572726F72AD
:102230000A00446F6E65207072696E74696E672063
:1022400066696C650A0020496E76616C6964206578
:102250007874727564657220000000A0C0000000F0
:102260000000000000000057430000574300004EEC
:1022700043486F6D696E67206661696C6564002014
:102280006E6F7420656E74657265642E0A005072FC
:102290006F7465637465642050696E0A004A303655
:1022A000004A3034004A30370020573A007C3C3E28
:1022B0005E2B3D3F2F5B5D3B2C2A225C00627573D9
:1022C000793A2070617573656420666F7220696E5B
:1022D0007075740A00627573793A20706175736560
:1022E0006420666F7220757365720A006275737977
:1022F0003A2070726F63657373696E670A004A31C2
:1023000035004B494C4C45442E20004B494C4C2049
:10231000636175736564206279204B494C4C20627F
:102320007574746F6E2F70696E0A004B494C4C4582
:10233000442E20004B494C4C20636175736564202A
:10234000627920746F6F206D75636820696E6163B8
:10235000746976652074696D65202D2063757272CD
:10236000656E7420636F6D6D616E643A20004A3152
:1023700031005072696E7465722068616C746564B6
:102380002E206B696C6C28292063616C6C6564215C
:102390000A000000A0C0000000000000000057611B
:1023A000726E696E673A20486F6D696E672042757C
:1023B0006D702044697669736F72203C20310A0089
:1023C0000202040000A0400000A040000000400005
:1023D000005C430000574300004E43FFFFFF000036
:1023E0002100240027002A002D00300033000101C5
:1023F0000000040107010A01000022002500280056
:102400002B002E00310034000201000005010801FC
:102410000B01000020002300260029002C002F00C3
:102420003200000100000301060109010505050550
:10243000070508080808020202020A0A080804043C
:10244000040401010101010101010303030303036A
:102450000303040707070C0C0C0C0C0C0C0C0202F9
:10246000020206060606060606060B0B0B0B0B0BF6
:102470000B0B010210202008081020401020408083
:102480000201020108040201010204081020408038
:1024900080402010080402018004020180402010C6
:1024A000080402010804020101020408102040800F
:1024B000010204081020408000000A0B02090C0DE4
:1024C0000E080703040100000000000000000000E7
:1024D00000000000000000000000000000000000FC
:1024E00000000000121110000000000000000000B9
:1024F0000000000000000000000000000000556E19
:102500006B6E6F776E20636F6D6D616E643A202223
:10251000002066697273740A005A00590058004816
:102520006F6D6520000000484200004842000080B6
:10253000400000000048617264636F646564204479
:10254000656661756C742053657474696E67732079
:102550004C6F616465640A00B80B0000B80B0000A2
:102560003C000000102700000000FA430000FA437E
:102570000000C040000070420000A0420000A042E5
:102580000000C843E17AD24220286D6D2900202046
:102590004D393030204B004C696E656172204164CA
:1025A00076616E63653A0A002044002049002020CD
:1025B0004D33303420500020440020490020204D6D
:1025C0003330312050005049442073657474696E73
:1025D00067733A0A00205A0020204D3636360045EF
:1025E0006E6473746F702061646A7573746D656E68
:1025F000743A0A00205A002059002020473239201E
:102600005333205800205A0020204D3432302053BC
:10261000004D65736820426564204C6576656C6981
:102620006E673A0A00205A0020590020204D3230AF
:1026300036205800486F6D65206F66667365743A82
:102640000A00204500205A0020590020580020543C
:102650000020530020204D32303520510020453CD1
:102660006D61785F655F6A65726B3E0020583C6DF6
:1026700061785F785F6A65726B3E20593C6D617866
:102680005F795F6A65726B3E205A3C6D61785F7A54
:102690005F6A65726B3E00416476616E6365643AA1
:1026A00020513C6D696E5F7365676D656E745F7414
:1026B000696D655F75733E20533C6D696E5F66653D
:1026C0006564726174653E20543C6D696E5F74721E
:1026D0006176656C5F66656564726174653E002055
:1026E000540020520020204D3230342050004163ED
:1026F00063656C65726174696F6E2028756E6974AC
:10270000732F7332293A20503C7072696E745F6186
:102710006363656C3E20523C726574726163745FE2
:10272000616363656C3E20543C74726176656C5FD6
:10273000616363656C3E0A00204500205A00205901
:102740000020204D3230312058004D6178696D7580
:102750006D20416363656C65726174696F6E2028DA
:10276000756E6974732F7332293A0A002045002070
:102770005A0020590020204D3230332058004D613E
:1027800078696D756D206665656472617465732026
:1027900028756E6974732F73293A0A00204500204A
:1027A0005A0020590020204D3932205800537465BA
:1027B00070732070657220756E69743A0A0020206B
:1027C0004D3230302044300A0020204D323030204D
:1027D00044002044697361626C65640A0046696C58
:1027E000616D656E742073657474696E67733A0009
:1027F0002020473231202020203B005452494747B7
:1028000045524544006F70656E003A20007A325F91
:102810006D696E007A5F6D696E00795F6D696E003B
:10282000785F6D696E005265706F7274696E6720B3
:10283000656E6473746F70207374617475730A00CD
:102840000A4D6561737572656420706F696E74738B
:102850003A0A005A206F66667365743A20004E7516
:102860006D20582C593A20352C350A004572726F6C
:10287000722077726974696E6720746F20454550C5
:10288000524F4D210A00526573656E643A20006F05
:102890006B0020746F6F206C6F6E672065787472A8
:1028A0007573696F6E2070726576656E7465640A03
:1028B0000020636F6C6420657874727573696F6E45
:1028C0002070726576656E7465640A00577269746B
:1028D000696E6720746F2066696C653A20006F70BE
:1028E000656E206661696C65642C2046696C653A8A
:1028F00020006F70656E206661696C65642C2046EF
:10290000696C653A200046696C652073656C656387
:102910007465640A002053697A653A200046696C40
:1029200065206F70656E65643A20002066696C658D
:102930003A2000646F696E67006672657368004EC6
:102940006F772000454E4420535542524F5554490D
:102950004E450A002220706F73002220706172655C
:102960006E743A2200535542524F5554494E4520F9
:1029700043414C4C207461726765743A22004B49A4
:102980004C4C45442E2000747279696E6720746F38
:102990002063616C6C207375622D67636F646520C2
:1029A00066696C6573207769746820746F6F206D39
:1029B000616E79206C6576656C732E204D415820D0
:1029C0006C6576656C2069733A00F1D2D2D411241B
:1029D0001FBECFEFD1E2DEBFCDBF00E00CBF14E0E1
:1029E000A0E0B2E0E8E0F3EC01E00BBF02C007902A
:1029F0000D92A431B107D9F727E1A4E1B4E001C0F9
:102A00001D92A63BB207E1F714E1C6EED4E100E067
:102A100006C021970109802FFE010E94DCE0C53E1F
:102A2000D10780E00807A9F70E9451CD0C9473E10B
:102A30000C9400002F923F924F925F926F927F9280
:102A40008F929F92AF92BF92CF92DF92EF92FF92BE
:102A50000F931F93CF93DF93CDB7DEB7C154D10946
:102A60000FB6F894DEBF0FBECDBF21E020939E15B8
:102A70008091C2168D3409F421C5843511F40C946B
:102A80001229873411F00C945E298091C016909120
:102A9000C1168A31910509F405C26CF484309105A0
:102AA00034F4823091055CF597FF22C003C504978A
:102AB00009F4B9C1FFC48A32910509F4F2C344F4A0
:102AC0008C31910509F4F2C14D9709F4F4C1F2C4B7
:102AD0008B35910509F470C48C35910509F470C4E7
:102AE0008A35910509F0E6C4109227040C946029F8
:102AF0008091330281110C9465290C9460292091F6
:102B00003302222311F40C94602911E0029709F09A
:102B100010E00E948C8919821A821B821C821D82FD
:102B20001E821F82188682E50E94243B882309F4B6
:102B30002AC10E94A43A4B015C0120E030E0A901C7
:102B40000E9494D9882309F434C1409132045091F1
:102B5000330460913404709135044EA35FA368A7D9
:102B600079A7609136047091370480913804909170
:102B700039046AA77BA78CA79DA780911316909113
:102B80001416A0911516B09116168EA79FA7A8AB84
:102B9000B9AB4091171650911816609119167091A3
:102BA0001A164AAB5BAB6CAB7DAB9C01AD016EA161
:102BB0007FA188A599A50E9494D981110DC02AA949
:102BC0003BA94CA95DA96AA57BA58CA59DA50E94E2
:102BD00094D9882309F4EDC020E030E0A901C501B3
:102BE000B4010E9494D9881F8827881F181749F0BC
:102BF00060E070E080E89FEB6AAF7BAF8CAF9DAF89
:102C000008C080E090E0A0E8BFE38AAF9BAFACAF24
:102C1000BDAF2EA13FA148A559A56EA57FA588A946
:102C200099A90E94DFDD6EAB7FAB88AF99AF2AA573
:102C30003BA54CA55DA56AA97BA98CA99DA90E946D
:102C4000DFDD6B017C012EA93FA948AD59ADCA015A
:102C5000B9010E94F9D92B013C01A7019601C701D6
:102C6000B6010E94F9D99B01AC01C301B2010E94D7
:102C7000E0DD0E944BE02B013C0120E030E040E031
:102C80005FE30E94F9D922966CAF7DAF8EAF9FAF04
:102C90002297A5019401C501B4010E94F9D94B0105
:102CA0005C0122962CAD3DAD4EAD5FAD2297CA01C1
:102CB000B9010E94F9D99B01AC01C501B4010E9480
:102CC000DFDD0E944BE02AAD3BAD4CAD5DAD0E9417
:102CD000F9D94B015C01C701B6019058A3019201DB
:102CE0000E94BCDEA50194010E94F9D96B017C0110
:102CF0002EA53FA548A959A96EA17FA188A599A590
:102D00000E94E0DD20E030E040E05FE30E94F9D97E
:102D10009B01AC01C701B6010E94E0DD2EA13FA1DD
:102D200048A559A50E94DFDD69837A838B839C8344
:102D30002AA93BA94CA95DA96AA57BA58CA59DA53F
:102D40000E94E0DD20E030E040E05FE30E94F9D93E
:102D50006B017C01A30192016EA97FA988AD99AD99
:102D60000E94BCDEA50194010E94F9D99B01AC012F
:102D7000C701B6010E94E0DD2AA53BA54CA55DA5D3
:102D80000E94DFDD12C089E40E94243B882331F0D9
:102D90000E94A43A69837A838B839C838AE40E948D
:102DA000243B882331F00E94A43A6D837E838F8375
:102DB000988720E030E0A90169817A818B819C812C
:102DC0000E9494D981110EC020E030E0A9016D81EC
:102DD0007E818F8198850E9494D9811103C0E6E895
:102DE000FBE10DC0412FBE016F5F7F4F83E196E194
:102DF0000E94CA9F0C9460290E9488C5F8018491A2
:102E00008F010F5F1F4F8111F7CFEDE1F2E0849149
:102E10008F010F5F1F4F882311F40C9460290E94CB
:102E200088C5F801F4CF80E50E94243B882379F01F
:102E30008091150490911604009749F04AE050E003
:102E400060E070E00E9413D86B017C0103C0C12CCC
:102E5000D12C760183E50E94243B882361F00E94F7
:102E6000A43A20E030E04AE754E40E94F9D90E94F5
:102E700029DF6B017C010E94C4620E94A551C60E2D
:102E8000D71EE81EF91E0E94A551DC01CB018C194A
:102E90009D09AE09BF09B7FD02C00C9460290E94CC
:102EA000099CF1CF0E94C13C0C94602980E00E94F3
:102EB000988E0C94602983E50E94243B882321F19D
:102EC0000E94843A182F863070F0E5EEF2E084918B
:102ED0008F010F5F1F4F882311F40C9460290E940B
:102EE00088C5F801F4CF833009F44AC130F4813049
:102EF00091F1823009F43FC008C0843009F49FC1C9
:102F0000853009F4ACC101C010E00E94108A811123
:102F100003C0E5ECF2E013C08091E115882319F0BD
:102F200063E173E002C067E173E08DEB92E00E9421
:102F3000D9508AE00E9488C50E9420B596C184912C
:102F40007F019FEFE91AF90A882309F48EC10E94D4
:102F500088C5F701F4CF0E94D3B5109201021092F8
:102F6000000282EB92E090938B0C80938A0C0E947B
:102F70005E8B0C946029809100029091010297FF72
:102F80000EC0E9E8F2E084918F010F5F1F4F8823A4
:102F900011F40C9460290E9488C5F801F4CF0097C1
:102FA000A1F4809137028093280419821A821B822F
:102FB0001C8218A219A21AA21BA2BE016F5F7F4F2A
:102FC000CE0180960E946FA727C0815065E00E94C5
:102FD000A8E080FF03C024E0291B922FA5E09A02FD
:102FE000F0011124E80FF11D87FDFA95EE0FFF1F88
:102FF000EE0FFF1FED5CF94E80913A0490913B0477
:10300000A0913C04B0913D0480839183A283B3835B
:1030100080912804809337028091000290910102F0
:10302000893191050CF067C0109237029C012F5F27
:103030003F4F309301022093000265E00E94A8E018
:1030400080FF03C024E0291B922F40913A04509145
:103050003B0460913C0470913D0448A359A36AA3CA
:103060007BA319821A821B821C82B4E08B0290011E
:103070001124F901E053F14F4F0120813181428148
:103080005381F4E09F02C0011124BC016C51714FC7
:103090005B01DB016D917D918D919C91FE013196DB
:1030A0006F01E12CF12C00EA10E40E949FA6198226
:1030B0001A821B821C82B601CE0180960E946FA7E5
:1030C000F50180819181A281B38180933204909334
:1030D0003304A0933404B0933504F40180819181CA
:1030E000A281B3818093360490933704A09338046F
:1030F000B0933904BCC080E090E0A0EAB0E48093D3
:103100003A0490933B04A0933C04B0933D040E9486
:103110005D8A0E94C4628FEF9FEF909301028093BB
:103120000002E5E7F2E084918F010F5F1F4F8823D3
:1031300021F00E9488C5F801F6CF83E992E09A83D6
:10314000898304E610E019A308A3BE016F5F7F4FD7
:10315000CE0180960E948AA88AEB92E09A838983A6
:1031600019A308A3BE016F5F7F4FCE0180960E9416
:103170008AA881E00E94988E81E00E943D8A77C0F3
:1031800088E50E94243B8823A1F00E94743A1FEF37
:10319000160F1530A8F0EEE5F2E084918F010F5F75
:1031A0001F4F882311F40C9460290E9488C5F801F0
:1031B000F4CF88E50E9488C50E94C2D40C9460298F
:1031C00089E50E94243B8823A1F00E94743A0FEF06
:1031D000060F0530A8F0E7E4F2E084918F010F5F5D
:1031E0001F4F882311F40C9460290E9488C5F801B0
:1031F000F4CF89E50E9488C50E94C2D40C9460294E
:103200008AE50E94243B882399F00E94A43A25E095
:10321000129FF0011124E00FF11DEE0FFF1FEE0FC2
:10322000FF1FED5CF94E608371838283938335C009
:103230008AE50E9488C50E94C2D40C9460298AE560
:103240000E94243B8823A1F30E94A43A60932F1686
:103250007093301680933116909332161EC080E022
:103260000E943D8A0E94D3B518C01230B1F460911B
:103270000002709101026931710514F069E170E09A
:1032800088E392E00E94C05069E170E083E392E03D
:103290000E94C0508AE00E9488C50E9400850C945C
:1032A000602980913302882311F40C94602989E409
:1032B0000E94243BE82E882321F00E94743A062FB6
:1032C00001C000E08AE40E94243BF82E882321F00C
:1032D0000E94743A162F01C010E0EE2011F0053064
:1032E00020F4FF2081F0153070F0ECEFF2E08491D3
:1032F0008F010F5F1F4F882311F40C9460290E94E7
:1033000088C5F801F4CF0E94303BEE2091F044E0F4
:103310000402F0011124EC51F14F80819181A281CE
:10332000B3818093131690931416A0931516B0933F
:103330001616FF2091F054E01502F0011124E0531D
:10334000F14F80819181A281B38180931716909370
:103350001816A0931916B0931A1680E50E94243B04
:10336000882319F00E94953A03C080E50E94DB3A59
:1033700086E40E94243B8823D9F00E94A43A6B0182
:103380007C0120E030E0A9010E9406E0181684F4D8
:1033900020E030E040E752E4C701B6010E94BCDE05
:1033A0006093490270934A0280934B0290934C02BF
:1033B0000E9421BC0C946029209327040C9460295E
:1033C00097E5292E92E0392E2CEAE22E25E1F22E05
:1033D00062E374E07FA36EA337E1C32E34E0D32E03
:1033E00000E010E0D1018D911D010E94243B882353
:1033F00009F44BC00E94A43A2B013C01133049F060
:10340000F60120813181428153810E94DFDD2B0151
:103410003C01AEA1BFA12D913D914D915C91C301A5
:10342000B2010E94DFDD4B015C012DEB37E346E882
:1034300055EB0E9406E087FD0AC02DEB37E346E816
:1034400055E3C501B4010E9494D91816F4F4133061
:1034500051F440923E0450923F04609240047092B6
:10346000410401E012C0A5019401F701608171815E
:10347000828193810E94E0DDD7016D937D938D93CE
:103480009C931397812F0E94B48A1F5FB4E0EB0EC8
:10349000F11CEEA1FFA13496FFA3EEA3F4E0CF0E42
:1034A000D11C143009F09ECF002309F4F6CE0E94FF
:1034B0003BA6F3CE0E94BEA80C9460298091C01652
:1034C0009091C1168537910511F40C9460290CF088
:1034D000C5C08C34910509F4D2C40CF05DC08A31AA
:1034E000910509F432C264F58531910509F4EBC107
:1034F000C4F48231910509F456C68431910509F46A
:10350000A2C1419711F00C940F295F988A984798AF
:1035100080910801817080930601479812980C945D
:1035200060298731910509F4D8C10CF4D0C18831E4
:10353000910509F4E8C1499709F4F0C10C940F29E9
:103540008F31910509F48FC384F48C31910509F40E
:10355000A2C20CF408C28D31910511F40C946029BB
:103560004E9709F4A2C20C940F298A32910509F4EE
:103570002DC42CF4809709F42AC30C940F298133AD
:10358000910509F457C48B34910511F00C940F295F
:103590000E94BD770C9460298A36910509F4ACC568
:1035A000B4F58435910509F4FEC5E4F4813591053F
:1035B00009F4D2C54CF48D34910511F00C940F2907
:1035C0000E94DF770C9460298235910509F4E7C5E4
:1035D0008335910511F00C940F2981E08093260426
:1035E0000C9460298C35910509F42DC634F4853589
:1035F000910509F40DC60C940F298836910509F43C
:1036000053C48936910509F417C50C940F298F36D8
:10361000910509F485C484F48C36910509F4D3C46A
:103620000CF488C58D36910509F448C58E36910590
:1036300009F463C40C940F298137910509F4CFC4B0
:103640000CF4C5C48237910509F485C6833791050A
:1036500011F00C940F29E9E0F5E0BCC68E3221E0B0
:10366000920711F40C944B270CF06FC08B3C910522
:1036700009F4CBC7ACF58C38910509F423C5ACF43B
:103680008737910509F44EC70CF4FFC688379105BA
:1036900009F44BC78937910511F00C940F2910924A
:1036A000A90A1092A80A0C9460298E3B910509F48E
:1036B0001FC534F48B39910509F4D9C40C940F2932
:1036C000883C910509F437C7893C910511F00C94A9
:1036D0000F29F7E5EF2EF2E0FF2E00E917E17BC797
:1036E0008C3D910511F40C94DE25ACF48D3C9105D4
:1036F00011F40C9496230CF4A4C78E3C910511F49C
:103700000C942324833D910511F00C940F29EBE9CF
:10371000FBE10C940B25823E910511F40C94592683
:103720003CF48D3D910511F40C94EB250C940F297C
:103730008C3251E0950711F40C9482268D32914021
:1037400011F40C94AB260C940F29853F71E0970778
:1037500011F40C943828E4F58A39B1E09B0709F498
:103760003AC4BCF48033F1E09F0711F40C94A22713
:1037700014F40C949F27833641E0940709F45FC04A
:103780008039914011F00C940F290E94C4620C946E
:103790006029853A61E0960711F40C9435284CF4C1
:1037A000843A914011F00C940F290E94CA850C9420
:1037B00060298C3AB1E09B0711F40C944624843FB5
:1037C000914011F00C940F290E940B690C94602910
:1037D0008A39F2E09F0711F40C947728B4F4873FFC
:1037E00041E0940711F40C943E2814F40C943B2807
:1037F000883F61E0960711F40C944A288C3092407F
:1038000011F40C946E280C940F298B38A3E09A07BE
:1038100011F40C9460293CF48438934011F40C9416
:10382000A4280C940F29803AF3E09F0709F40EC2F4
:10383000873E934011F40C94FC280C940F29E6E881
:10384000FBE10C942228EAE2F3E084918F010F5F00
:103850001F4F882321F00E9488C5F801F6CF1092EF
:10386000961189E49FE00E94B1948BE1E9E4FFE0C6
:10387000DE01159601900D928A95E1F78091470F30
:103880009091480F9C838B838DEE92E09A8389837D
:1038900040E050E0BE016F5F7F4F80E090E00E940B
:1038A0006E71CE0101960E949F9BEBE1F3E0849143
:1038B0008F010F5F1F4F882311F40C9460290E9421
:1038C00088C5F801F4CF0E943D6F0C9460291092D6
:1038D000180F1092190F0C946029E091BE16F09108
:1038E000BF168081882329F0803209F41082319636
:1038F000F8CF40E061E08091BE169091BF160E9423
:1039000012C70C9460298091190F882319F081E067
:103910008093180F0E94BD770C9460291092180FA5
:103920008091B814813011F00C94602982E080936A
:10393000B8140E94A5516093B4147093B514809389
:10394000B6149093B7140C9460298091190F8823B2
:1039500011F40C94602983E50E94243B81110C949E
:103960006A290C94602983E40E94DB3A882309F4D5
:1039700050C0E8E6F3E084918F010F5F1F4F88236A
:1039800021F00E9488C5F801F6CF8091E4108111E2
:1039900003C0EBE3F3E012C0BE016F5F7F4F81EE27
:1039A00090E10E9479938E010F5F1F4FD8018D9196
:1039B0008D01882349F10E9488C5F8CF84918F0139
:1039C0000F5F1F4F882301F10E9488C5F801F6CFD1
:1039D0001CEFC12E13E0D12EE12CF12C20E08091C0
:1039E000820C90E00E2C02C0959587950A94E2F720
:1039F00080FDC6C24FEFE41AF40A52E0C50ED11C96
:103A000065E0E616F10459F78AE00E9488C50C9437
:103A100060298091190F882339F08091180F88232D
:103A200019F0E5E4F3E003C0E7E5F3E028C0849192
:103A30008F010F5F1F4F882321F00E9488C5F80176
:103A4000F6CF6091921170919311809194119091A1
:103A500095114AE00E948FC58FE20E9488C560914F
:103A60008E1170918F1180919011909191114AE077
:103A70000E948FC58AE00E9488C50C9460298491B9
:103A80008F010F5F1F4F882311F40C9460290E944F
:103A900088C5F801F4CF40E060E08091BE169091B7
:103AA000BF160E9412C70C9460298091190F8823B9
:103AB00011F40C94602981EE90E10E9460BA81EECD
:103AC00090E10E9454931092170F1092160F80915C
:103AD000190F882311F40C9460290091BE161091DF
:103AE000BF160E946171B801CE0180960E94757365
:103AF0008C01892B11F40C94602968A179A16115BE
:103B0000710511F06C5F7F4F19821C8222E0A801C1
:103B1000CE0101960E94E098811102C0F12C14C0E0
:103B2000CE0101960E94CF708823C1F361E0CE01DF
:103B300001960E945D93009789F325EEFC01208396
:103B40001C820E9409B8F82ECE0101960E9482C5FF
:103B5000F11003C0E5E8F3E022C0E7E7F3E0849169
:103B60007F012FEFE21AF20A882321F00E9488C514
:103B7000F701F5CFD8018D918D01882319F00E94AE
:103B800088C5F8CF8AE00E9488C5109292111092E1
:103B9000931110929411109295110C9460298491B4
:103BA0007F01BFEFEB1AFB0A882321F00E9488C532
:103BB000F701F5CFF80181918F01882319F00E9458
:103BC00088C5F8CF8EE20E9488C50C946029809148
:103BD000180F81110E94C4628091190F882311F47B
:103BE0000C94602980E50E94243B882319F00E94F0
:103BF000953A03C080E50E94DB3A182F482F61E018
:103C00008091BE169091BF160E9412C783E50E9454
:103C1000243B882381F00E94743AAB01BC0140939D
:103C2000921150939311609394117093951181EEBA
:103C300090E10E946A928091190F882319F081E027
:103C40008093180F11110C94602964CE8091BE16D8
:103C50009091BF1621E02093170F40E060E00E9492
:103C600012C70C9460290E946E777B018C0120E8BA
:103C700031E541E050E00E9482DDC9016DE671E06E
:103C80000E94B5E04B015C01C801B70120E13EE0B4
:103C900040E050E00E9482DDCA01B90128E130E035
:103CA00040E050E00E9482DD762E672EC62ED72E91
:103CB0008CE3282E312C412C512CC801B701A201D4
:103CC00091010E9482DDF62EE72ECA01B901A20100
:103CD00091010E9482DDCB018E010F5F1F4F811485
:103CE0009104D1F0EF92FF927F936F936F927F9246
:103CF000BF92AF929F928F9285EC93E09F938F93A8
:103D00001F930F930E9466D90FB6F894DEBF0FBEC3
:103D1000CDBFEBE9FBE145C0A114B10489F0EF92FE
:103D2000FF927F936F936F927F92BF92AF9285EBDA
:103D300093E09F938F931F930F930E9466D9E4CFD4
:103D4000CD2879F0EF92FF927F936F936F927F92DD
:103D500089EA93E09F938F931F930F930E9466D9F4
:103D6000D3CF892B69F0EF92FF927F936F9381EA13
:103D700093E09F938F931F930F930E9466D9C4CFB4
:103D8000EF92FF928DE993E09F938F931F930F9390
:103D90000E9466D90F900F900F900F900F900F9088
:103DA000B8CF84917F01BFEFEB1AFB0A882321F083
:103DB0000E9488C5F701F5CFB80189ED93E00E9414
:103DC000D9508AE00E9488C50C94602983E50E943E
:103DD000243B882311F40C9460290E94843AE82E35
:103DE00080E50E94243B882339F00E94843A182FF2
:103DF00087FF03C00C9460291DE089E40E94243BE6
:103E0000882341F00E94953A81110C94E329E9E757
:103E1000F6E00BC089E40E94DB3AF6CF319626E04B
:103E2000E93AF20711F40C94E32984911813F6CFC0
:103E30000C94E029F090140481E0F826F092140428
:103E4000E1EFF3E084918F010F5F1F4F882321F092
:103E50000E9488C5F801F6CFFF2019F0E6EEF3E0E6
:103E600002C0EBEEF3E084918F010F5F1F4F8823B8
:103E700011F40C9460290E9488C5F801F4CF809158
:103E8000B814813011F00C94602982E08093B8144A
:103E90000E94A5516093B4147093B5148093B61426
:103EA0009093B7140C94602988E690E00E94F48AFD
:103EB00081110C9460298091820C83FF02C00C94C4
:103EC000602983E50E94243B882399F00E94A43A4C
:103ED0000E9424DFCB010E949A520E94A43A20E063
:103EE00030E044EB52E40E9494D9181614F00E947A
:103EF000DF770E9424510C9460298EE40E94243BB9
:103F0000882311F40C9460290E94743A6093781706
:103F10007093791780937A1790937B170C9460298C
:103F200083E50E94DB3A882359F083E50E94243B15
:103F3000882319F00E94843A01C080E08093820CAB
:103F4000EBE9FBE184918F010F5F1F4F811103C0EB
:103F5000EAE0F4E004C00E9488C5F801F3CF849140
:103F60008F010F5F1F4F882321F00E9488C5F80141
:103F7000F6CF8091820C81112BCDE6E0F4E018C0E1
:103F8000BB24B394B20E222319F08CE20E9488C5A0
:103F9000F60185919491FC0184918F010F5F1F4F71
:103FA000882321F00E9488C5F801F6CF2B2D22CD61
:103FB00084918F010F5F1F4F882309F425CD0E9444
:103FC00088C5F801F5CF10922C020C94602981E18C
:103FD00094E00E94C29B0E942B7F0C94602983E591
:103FE0000E94243B811103C0EBE9FBE10DC00E945C
:103FF000843A8D3320F4809338020C9460298CE34A
:10400000809338020C94602984918F010F5F1F4FB9
:10401000882321F00E9488C5F801F6CF409138022C
:1040200050E060E070E08AE194E00E9486508AE00F
:104030000E9488C50C94602989E690E00E94F48A69
:10404000811111C0E1E2F4E084918F010F5F1F4FF5
:10405000882321F00E9488C5F801F6CF0E94F674EB
:104060008AE00E9488C510929E150C94F82983E579
:104070000E94243B882311F40C9460290E94843A06
:10408000182F8D3308F01CE31093AB150E94A55137
:104090006B017C01212F30E0A8EEB3E00E94D0DD5F
:1040A000C60ED71EE81EF91EC092A715D092A815FD
:1040B000E092A915F092AA150C9460290E945390E1
:1040C0000C9460298091820C83FF02C00C946029BB
:1040D00083E50E94243B882311F40C9460290E94FC
:1040E000A43A0E9424DFCB010E94B33C0C946029C7
:1040F0000E948B870C94602980E50E94243B8111EB
:1041000006C083E50E94243B882361F006C00E941C
:10411000843A81110C946029F4CF0E94743A6F3F65
:10412000710510F06FEF70E07093430460934204E8
:104130000C94602980E50E94243B811106C01092F6
:104140004304109242040C9460290E94743A672B35
:1041500011F00C946029F3CF0E94F4770E9491B083
:10416000109243041092420400E010E062E370E019
:1041700080E090E00E9434AA0E94B47A0F5F1F4F43
:104180000331110599F762E370E080E090E00E944E
:1041900034AA0E94B47A0E94122A0C9460291092C8
:1041A00026040C94602983E50E94243B8823A1F017
:1041B0000E94A43A20E030E04AE754E40E94F9D992
:1041C0000E9429DF6093390270933A0280933B0288
:1041D00090933C020C94602988E50E94DB3A81119F
:1041E0000C947B2989E50E94DB3A81110C947B2990
:1041F0008AE50E94DB3A81110C947B2985E40E94B8
:10420000DB3A81110C947B290E9491B00C946029B7
:1042100083E50E94DB3A882311F40C9460290E9404
:10422000A43A20E030E04AE754E40E94F9D90E9421
:1042300029DF6093A3157093A4158093A51590931F
:10424000A6150C946029A7E5CA2EA2E0DA2EB7EFD6
:10425000EB2EB5E1FB2E10E0D6018D916D010E9491
:10426000DB3A882309F46DC0133009F063C00E9463
:10427000A43A4B015C0120E030E040EA51E40E94A6
:1042800094D987FF4EC0A5019401609103167091E7
:10429000041680910516909106160E94BCDE2B0133
:1042A0003C019B01AC016091510C7091520C8091CA
:1042B000530C9091540C0E94F9D96093510C709357
:1042C000520C8093530C9093540CA3019201609173
:1042D000710C7091720C8091730C9091740C0E940F
:1042E000F9D96093710C7093720C8093730C909356
:1042F000740C60918C1770918D1780918E1790912E
:104300008F170E9498D9A30192010E94F9D90E94A7
:1043100029DF60938C1770938D1780938E1790937D
:104320008F178092031690920416A0920516B092F1
:10433000061607C00E94A43AF70160837183828346
:1043400093831F5FF4E0EF0EF11C143009F084CF6B
:104350000E9473CBB5C70E94C46283E50E94243BD0
:10436000882311F40C944D190E94743A623071053F
:1043700011F00C944D190E94FABF8BE50E9488C57C
:104380006091451770914617809147179091481793
:1043900042E00E9414C64091491750914A1760911B
:1043A0004B1770914C1787E294E00E94A350409104
:1043B0004D1750914E1760914F177091501784E22E
:1043C00094E00E94A3508DE50E9488C58AE00E9477
:1043D00088C576C784918F010F5F1F4F882321F016
:1043E0000E9488C5F801F6CF60E089EF94E00E9452
:1043F000C98461E082EF94E00E94C98461E087EEA5
:1044000094E00E94C98461E087ED94E00E94C98431
:1044100060E08EEC94E00E94C98461E084EC94E05A
:104420000E94C98460E08AEB94E00E94C98460E045
:1044300082EB94E00E94C98461E084EA94E00E94E7
:10444000C98460E086E994E00E94C98460E087E85E
:1044500094E00E94C98460E089E794E00E94C984E6
:1044600060E083E694E00E94C98460E082E594E025
:104470000E94C98460E08DE394E00E94C98461E0F9
:104480008AE294E00E94C9841BC70091BE16109175
:10449000BF1683E0D12C40E08150E9F0D8019C9117
:1044A000292F2B7F2134C1F711962C912133A1F7AD
:1044B000913421F0953421F441E002C0DD24D394FD
:1044C00098012E5F3F4F89012F5F3F4FF801908188
:1044D0009032C9F3E1CF442369F0EBE9FBE1849129
:1044E0007F012FEFE21AF20A882321F00E9488C58B
:1044F000F701F5CFDD2069F0EFECF5E084917F0165
:104500004FEFE41AF40A882321F00E9488C5F701CE
:10451000F5CFD8018D918D01882309F475CA0E94C9
:1045200088C5F7CF0E946BB6CBC681E08093A90AFD
:104530008093A80AC5C688EC90E00E94F48A811195
:10454000BFC684E40E94DB3A882309F441C00E947C
:10455000A43A6B017C0111E020E030E0A9010E9447
:1045600094D9811101C010E01093971620E030E03B
:10457000A901C701B6010E9494D9882349F10E947C
:10458000A43AE091DB14B4E0EB9FF0011124E4566F
:10459000F94E608371838283938320E030E0A90128
:1045A00060919C1670919D1680919E1690919F1619
:1045B0000E9494D981110CC080E090E0A0EEBFE38E
:1045C00080939C1690939D16A0939E16B0939F1671
:1045D0000E94CFB075C6F70181917F010E94DB3A3E
:1045E000882351F00E94A43A0E9429DFD8016D93DC
:1045F0007D938D939C9313970C5F1F4FB7E1003A07
:104600001B0749F70E9402CA5BC6E7E5EE2EE2E00F
:10461000FE2E05E61CE0F70181917F010E94DB3A46
:10462000882341F00E94A43AD8016D937D938D9325
:104630009C9313970C5F1F4FBCE005371B0759F77E
:104640003FC683E50E94243B8823A1F00E94A43A40
:1046500060935D0C70935E0C80935F0C9093600C84
:104660006093590C70935A0C80935B0C90935C0C84
:1046700010E001C011E080E50E94243B882359F03E
:104680000E94A43A60935D0C70935E0C80935F0C63
:104690009093600C10E082E50E94243B882359F03F
:1046A0000E94A43A6093610C7093620C8093630C37
:1046B0009093640C10E084E50E94243B882359F019
:1046C0000E94A43A6093590C70935A0C80935B0C2F
:1046D00090935C0CF5C5112309F4F2C540915D0C73
:1046E00050915E0C60915F0C7091600C89ED95E0CB
:1046F0000E94A3504091610C5091620C6091630C38
:104700007091640C86ED95E00E94A3504091590C85
:1047100050915A0C60915B0C70915C0C83ED95E0AC
:104720000E94A3508AE00E9488C5CAC581E50E9404
:10473000DB3A8823C1F0809115049091160400970C
:1047400039F04AE050E060E070E00E9413D803C006
:1047500060E070E0CB016093750C7093760C8093F1
:10476000770C9093780C83E50E94DB3A882351F014
:104770000E94A43A60937D0C70937E0C80937F0C12
:104780009093800C84E50E94DB3A882351F00E94CC
:10479000A43A6093790C70937A0C80937B0C90937D
:1047A0007C0C88E50E94DB3A882351F00E94A43AF1
:1047B0006093450C7093460C8093470C9093480C83
:1047C00089E50E94DB3A882351F00E94A43A609365
:1047D000490C70934A0C80934B0C90934C0C8AE5D7
:1047E0000E94DB3A8823F1F00E94A43A60934D0CBA
:1047F00070934E0C80934F0C9093500C2DEC3CEC2E
:104800004CEC5DE30E9494D9181664F0E9EEF5E0F3
:1048100084918F010F5F1F4F882321F00E9488C56C
:10482000F801F6CF85E40E94DB3A882309F448C5F5
:104830000E94A43A6093510C7093520C8093530CD5
:104840009093540C3DC567E5C62E62E0D62E7AEAF9
:10485000E72E7AE0F72E10E0F60181916F010E94B9
:10486000DB3A882359F00E94A43AD7016D937D93D7
:104870008D939C931397812F0E94B48A1F5FB4E09D
:10488000EB0EF11C133041F70C944D190E948DA7CB
:10489000811116C502E913E2E2E3F4E0FFA3EEA3FF
:1048A000AE014F5F5F4F5A015BED852E53E2952EAF
:1048B0001501F8016591759185919491AEA1BFA103
:1048C000CD90DD90ED90FD90BFA3AEA3A701960122
:1048D0000E94DFDD2B013C01F10160837183828343
:1048E000938320E030E040EA51EC0E9406E087FD2F
:1048F0000AC020E030E040EA51E4C301B2010E9466
:1049000094D918162CF4F401849118160CF425C5CA
:10491000D101CD90DD90ED90FD901D0120E030E0C3
:1049200040EA51ECC701B6010E9406E087FD0AC0CB
:1049300020E030E040EA51E4C701B6010E9494D97A
:1049400018164CF5E6E8FBE184918F010F5F1F4FCD
:10495000811103C0EBE1F6E004C00E9488C5F801B4
:10496000F3CF84918F010F5F1F4F882321F00E94A6
:1049700088C5F801F6CF88E290E099A388A388EC77
:1049800090E09DA38CA3BE01605E7F4FCE01849614
:104990000E948AA895C40C5F1F4FBFEF8B1A9B0A19
:1049A000E3E20E391E0709F084CF4AEAE42E4AE01A
:1049B000F42E10E0F50181919191A191B1915F01E7
:1049C000F70181939193A193B1937F01812F0E946D
:1049D000B48A1F5F133071F70E94008583E992E06B
:1049E0009DA38CA304E610E019A308A3BE016C5D8F
:1049F0007F4FCE0180960E948AA88AEB92E09DA309
:104A00008CA319A308A3BE016C5D7F4FCE018096D5
:104A10000E948AA855C484918F010F5F1F4F88237D
:104A200021F00E9488C5F801F6CF83E50E94DB3AA9
:104A3000882321F00E94953A80933702E1E6F6E060
:104A400084918F010F5F1F4F882321F00E9488C53A
:104A5000F801F6CF80913702882319F0E9E5F6E0F6
:104A600002C0EDE5F6E084918F010F5F1F4F8111C9
:104A700003C0E1E5F6E004C00E9488C5F801F3CF69
:104A800084918F010F5F1F4F882321F00E9488C5FA
:104A9000F801F6CF40901704509018046090190464
:104AA00070901A042091B8153091B9154091BA153B
:104AB0005091BB15C301B2010E94E0DDAB01BC0106
:104AC0008FE496E00E94A35080901B0490901C04F9
:104AD000A0901D04B0901E042091BC153091BD150E
:104AE0004091BE155091BF15C501B4010E94E0DD93
:104AF000AB01BC018CE496E00E94A350C0901F045F
:104B0000D0902004E0902104F09022042091C01560
:104B10003091C1154091C2155091C315C701B6011E
:104B20000E94E0DDAB01BC0189E496E00E94A35045
:104B3000E1E4F6E084918F010F5F1F4F882321F09D
:104B40000E9488C5F801F6CF20913D0230913E02C7
:104B500040913F0250914002C301B2010E94E0DD4A
:104B6000AB01BC018FE396E00E94A350209141026B
:104B7000309142024091430250914402C501B40178
:104B80000E94E0DDAB01BC018CE396E00E94A350E3
:104B900020914502309146024091470250914802CF
:104BA000C701B6010E94E0DDAB01BC0189E396E0DC
:104BB0000E94A3508AE00E9488C582C383E50E94B8
:104BC000243B882309F47CC30E94743A7093030247
:104BD0006093020275C38DED90E00E94F48A81110A
:104BE0006FC383E50E94243B811103C0EBE9FBE125
:104BF0003AC00091DB1410E00E94743A000F111FBC
:104C0000F801EF5AFD4F718360838091DB1490E0CF
:104C10007C01EE0CFF1CEE0CFF1C8701035D1D4F99
:104C2000880F991FFC01EF5AFD4F60817181072E9B
:104C3000000C880B990B0E949AD92AE037ED43E2C9
:104C40005CE30E94F9D9F701E856F94E20813181E1
:104C5000428153810E94F9D9D8016D937D938D9340
:104C60009C9313972DC384918F010F5F1F4F88234F
:104C700021F00E9488C5F801F6CF85E40E9488C51E
:104C80008091DB14805D0E9488C5E091DB14F0E028
:104C9000EE0FFF1FEF5AFD4F6081718181E796E0B3
:104CA0000E94C05085E20E9488C58AE00E9488C5A3
:104CB00007C380E50E94DB3A882309F401C30E9400
:104CC000743A6B017C0183E50E94243B882321F028
:104CD0000E94743A8B0102C00FEF1FEFC8010196CA
:104CE000039708F0EDC2D7FCEBC28C2DE9E7F6E0A4
:104CF0009491891709F464C33196B6E0E93AFB0749
:104D0000B9F736C383E50E94243B882319F00E943B
:104D1000743A02C064E071E079A368A380E50E9460
:104D2000243B882339F00E94743A6938E3E17E0716
:104D300030F402C068EE73E07A83698304C088E8C7
:104D400093E19A838983BE01605E7F4FCE01019615
:104D50000E948AA8B5C285E40E94243B811110C03C
:104D600080E50E94DB3A882391F00E94A43A609388
:104D7000C9147093CA148093CB149093CC1407C0B9
:104D80000E94843A882361F3E6E8FBE171C089E47C
:104D90000E94DB3A882381F00E94A43A2CEA35EC89
:104DA00047E25EE30E94F9D96093C5147093C6147C
:104DB0008093C7149093C81484E40E94DB3A88233C
:104DC00081F00E94A43A2CEA35EC47E25EE30E94AF
:104DD000BCDE6093CD147093CE148093CF14909367
:104DE000D014EBE9FBE184918F010F5F1F4F882303
:104DF00021F00E9488C5F801F6CF4091C914509166
:104E0000CA146091CB147091CC1481EB96E00E948F
:104E1000A3502CEA35EC47E25EE36091C514709133
:104E2000C6148091C7149091C8140E94BCDEAB01D7
:104E3000BC018DEA96E00E94A3502CEA35EC47E2D3
:104E40005EE36091CD147091CE148091CF14909157
:104E5000D0140E94F9D9AB01BC0189EA96E00E9406
:104E6000A3508AE00E9488C52BC20E9488C5F80121
:104E700084918F010F5F1F4F8111F7CFE5EBF6E0B3
:104E800084918F010F5F1F4F882309F419C20E947C
:104E900088C5F801F5CF83E50E94DB3A182F8823F7
:104EA00071F00E94A43A0E9424DF70933202609352
:104EB000310221E0672B09F020E02093810C80E58E
:104EC0000E94DB3A882359F020913102309132025E
:104ED000232B11F00E94953A8093810CF1C111119E
:104EE000EFC1EBE9FBE184918F010F5F1F4F882336
:104EF00021F00E9488C5F801F6CF8091810C8823AB
:104F000019F06BE173E002C06EE173E08CED96E0A6
:104F10000E94D95060913102709132028BEC96E080
:104F20000E94C050E7ECF6E084918F010F5F1F4FA5
:104F3000882309F4C5C10E9488C5F801F5CF0E94F5
:104F4000687FBEC180E50E94DB3A882351F00E9451
:104F5000A43A6093C1147093C2148093C3149093C5
:104F6000C41489E40E94DB3A882381F00E94A43AA9
:104F70002CEA35EC47E25EE30E94F9D96093BD1458
:104F80007093BE148093BF149093C01484E40E9465
:104F9000DB3A882381F00E94A43A2CEA35EC47E200
:104FA0005EE30E94BCDE6093B9147093BA148093E0
:104FB000BB149093BC14EBE9FBE184918F010F5F6C
:104FC0001F4F882321F00E9488C5F801F6CF409139
:104FD000C1145091C2146091C3147091C41487EF2E
:104FE00096E00E94A3502CEA35EC47E25EE3609124
:104FF000BD147091BE148091BF149091C0140E9492
:10500000BCDEAB01BC0183EF96E00E94A3502CEA0A
:1050100035EC47E25EE36091B9147091BA14809167
:10502000BB149091BC140E94F9D9AB01BC018FEE66
:1050300096E00E94A3508AE00E9488C541C10E9468
:1050400088C5F80184918F010F5F1F4F8111F7CF41
:10505000EBEFF6E084918F010F5F1F4F882309F477
:105060002FC10E9488C5F801F5CF0E94407E28C15B
:105070000E94FF6825C10E9403AF22C183E50E9400
:10508000DB3A882321F00E94953A91E089270E941B
:105090006EAA16C181E08093890C0E94F56210927D
:1050A000890C882309F40CC1EBE9FBE184918F01A1
:1050B0000F5F1F4F811103C0EAE0F7E004C00E94B8
:1050C00088C5F801F3CF84918F010F5F1F4F8823AC
:1050D00009F4F6C00E9488C5F801F5CF8091180F39
:1050E000882309F4EDC081E080931B0FE9C08AE5B5
:1050F0000E94243B811103C0E8E1F7E00BC00E944D
:10510000A43A60932B1670932C1680932D169093CF
:105110002E16D6C084918F010F5F1F4F882321F078
:105120000E9488C5F801F6CF40912B1650912C169D
:1051300060912D1670912E1685E197E00E94A35084
:105140008AE00E9488C5BCC08BE40E94243B811188
:1051500003C0EBE9FBE136C08BE40E94243B8823CB
:10516000C1F00E94A43A6B017C0120E030E0A9016B
:105170000E9406E087FD0AC020E030E040E251E4F2
:10518000C701B6010E9494D9181634F4E7E3F7E09A
:105190000EC0C12CD12C76010E94C462C092550C65
:1051A000D092560CE092570CF092580C89C0849122
:1051B0008F010F5F1F4F882309F482C00E9488C5AA
:1051C000F801F5CF84918F010F5F1F4F882321F0E5
:1051D0000E9488C5F801F6CF4091550C5091560CAD
:1051E0006091570C7091580C86E597E00E94A3508F
:1051F0008AE00E9488C564C081E08093330283E521
:105200000E94243B882339F00E94953A811158C0AE
:105210000E9431C055C083E50E94DB3AF7CF0E945F
:10522000BEA84EC0F090C0160E94C4621091E11555
:1052300080E00E943D8AFF2029F1EBE9FBE18491A7
:105240008F010F5F1F4F882321F00E9488C5F8014E
:10525000F6CF84E50E9488C56F2D70E080E090E075
:105260004AE00E948FC580E20E9488C5E3E7F7E02C
:1052700084918F010F5F1F4F882311F10E9488C511
:10528000F801F6CF10929D15812F0E943D8AEBE91F
:10529000FBE184918F010F5F1F4F882321F00E9453
:1052A00088C5F801F6CF60919D1570E081E697E022
:1052B0000E94C0508AE00E9488C502C00E94BEA819
:1052C00010929E150E9416C093C00E948C890E9465
:1052D00021BCF6CF0E94743AAB01BC0140939211FD
:1052E00050939311609394117093951181EE90E116
:1052F0000E946A92E5CF0E94C46288E50E94DB3A70
:10530000882331F05F9A809131048E7F809331043D
:1053100089E50E94DB3A882339F08A9A479A80917E
:1053200031048D7F809331048AE50E94DB3A882323
:1053300061F0809108018095817080930601479A01
:10534000809131048B7F8093310485E40E94DB3AA5
:10535000882309F4B5CF129AB3CFF7FAF094F7F88F
:10536000F094D101CD92DD92ED92FC921397D0CAC8
:105370000E94C462BC2C60E08C2D0E9431A90F3FBA
:10538000BFEF1B0759F48C2D0E94DBA831E020E011
:10539000892B09F030E0032F122F05C001301105D1
:1053A00061F401E010E08B2D0E94DBA880179107CB
:1053B00009F486CF0E94099CF6CF00E010E0F3CFFD
:1053C0000E94A7D47DCF61E0812F0E9431A96E2D6C
:1053D000812F0E9403A9F12CB701812F0E946DA992
:1053E000193009F06DCFF0924304E092420468CF87
:1053F000CF5BDF4F0FB6F894DEBF0FBECDBFDF919E
:10540000CF911F910F91FF90EF90DF90CF90BF90C1
:10541000AF909F908F907F906F905F904F903F9054
:105420002F9008952F923F924F925F926F927F92AA
:105430008F929F92AF92BF92CF92DF92EF92FF92A4
:105440000F931F93CF93DF93CDB7DEB76F970FB650
:10545000F894DEBF0FBECDBFC0904C04D0904D0479
:10546000E0904E04F0904F0420E030E040EA50E439
:10547000C701B6010E9494D987FD19C120E030E030
:1054800041E953E4C701B6010E9406E018160CF486
:105490000EC110923513109234138091090140917E
:1054A0003313042E000C550B817021E0822790E00D
:1054B0004817590709F433C08091090181702827E2
:1054C0002093331381111BC00E943D6FEDE8FDE076
:1054D00084918F01882351F0082E000C990B0E94B3
:1054E000386F0F5F1F4FF8018491F4CF8DE090E08B
:1054F0000E94386F8AE090E00E94386F10C0E1E9A6
:10550000FDE084918F01882389F3082E000C990B0C
:105510000E94386F0F5F1F4FF8018491F4CF809184
:105520002613833009F44CC02CF4882351F08130C9
:10553000D9F072C0843009F43EC0853009F44DC002
:105540006BC08091180F882309F466C081E08093B6
:1055500026130E94A55160932A1370932B138093F6
:105560002C1390932D1358C08091180F811154C0A3
:105570008091E410882321F082E0809326134CC0B0
:1055800010922613E9E8FDE084918F01882351F001
:10559000082E000C990B0E94386F0F5F1F4FF80107
:1055A0008491F4CF8DE090E00E94386F8AE090E023
:1055B0000E94386F31C0809173138823E9F22CC0A8
:1055C0008091180F811128C080919A0E90919B0EA6
:1055D000891B8F7009F496C01FC08091180F81112C
:1055E0001BC080919A0E90919B0E891B8F7009F4BD
:1055F000ABC012C08DE090E00E94386F8AE090E06E
:105600000E94386F1092261389E69DE090938B0CD0
:1056100080938A0C0E945E8B80911B1390911C13C7
:1056200003974CF57DE9272E79E0372EE0E68E2EA4
:10563000EAEE9E2EA12CB12C81E894E10E94343A2E
:1056400018161906C4F480911B1390911C1304972B
:1056500094F481E894E10E94F83980932113E09159
:105660002213F09123138A3019F08D3009F07DC098
:10567000309709F083C080911B1390911C13009701
:1056800011F40C949239019790931C1380931B137F
:1056900080911D1390911E13019664E070E00E94AA
:1056A000C9E090931E1380931D130C94923980913E
:1056B0003413909135138136FAEE9F07E8F010927B
:1056C000351310923413E5E9FDE084918F018823AE
:1056D00051F0082E000C990B0E94386F0F5F1F4F7E
:1056E000F8018491F4CF8DE090E00E94386F8AE059
:1056F00090E00E94386FD1CE01969093351380933D
:105700003413CBCE85E79DE090938B0C80938A0C6D
:105710000E945E8B80917313882311F082E001C098
:1057200084E080932613E1E7FDE084918F018823D4
:1057300009F438CF082E000C990B0E94386F0F5FC8
:105740001F4FF8018491F3CFEDE6FDE084918F01C6
:10575000882309F44FCF082E000C990B0E94386F54
:105760000F5F1F4FF8018491F3CF8A3309F480CF84
:10577000EF35F10514F40C9426377ACF80911F137E
:105780009091201320E6289F7001299FF00C11248E
:10579000870105561E4EE00FF11F108261E470E094
:1057A000C8010E9430E1009711F40C940A379093DD
:1057B000251380932413801B910B8E0D9F1D60E099
:1057C00070E084569E4E0E9495D50E9424DFCB0146
:1057D000770FAA0BBB0B8232910510F00C940A379D
:1057E000FC018827EE58FF4F8F4F0C94DCE0E4E675
:1057F000FDE084918F01882351F0082E000C990B55
:105800000E94386F0F5F1F4FF8018491F4CF20E0A2
:1058100030E040E05FE360914C0470914D04809172
:105820004E0490914F041EC0EFE5FDE084918F017E
:10583000882351F0082E000C990B0E94386F0F5FDF
:105840001F4FF8018491F4CF60914A0470914B048A
:10585000072E000C880B990B0E949AD920E030E0AB
:1058600040E05FE30E94E0DD0E9424DFCB010E9464
:105870007D3C0E9436C98DE090E00E94386F8AE03E
:1058800090E00E94386F0C940A37EAE5FDE08491BD
:105890008F01882351F0082E000C990B0E94386F5D
:1058A0000F5F1F4FF8018491F4CF20E030E040E01B
:1058B0005FE36091460470914704809148049091A1
:1058C0004904D0CFE5E5FDE084918F01882351F0B4
:1058D000082E000C990B0E94386F0F5F1F4FF801C4
:1058E0008491F4CF6091440470914504B1CF20912C
:1058F00042043091430444E6429FC001439F900D0F
:1059000011246FEF70E00E94C9E08B0165367105CC
:1059100010F004E610E0E0E5FDE084917F018823CB
:1059200059F0082E000C990B0E94386FFFEFEF1A08
:10593000FF0AF7018491F3CFB80180E090E035C70A
:10594000ECE4FDE084918F01882351F0082E000CD7
:10595000990B0E94386F0F5F1F4FF8018491F4CFAD
:1059600080E290E00E94386FE8E4FDE084918F01CE
:10597000882351F0082E000C990B0E94386F0F5F9E
:105980001F4FF8018491F4CF609132047091330479
:1059900080913404909135040E9437C980E290E0F0
:1059A0000E94386FE4E4FDE084918F01882351F078
:1059B000082E000C990B0E94386F0F5F1F4FF801E3
:1059C0008491F4CF6091360470913704809138044B
:1059D000909139040E9437C980E290E00E94386FAC
:1059E000E0E4FDE084918F01882351F0082E000C43
:1059F000990B0E94386F0F5F1F4FF8018491F4CF0D
:105A000060913A0470913B0480913C0490913D0474
:105A10000E9437C980E290E0A0C58091180F8823CA
:105A200009F450C0EBE3FDE084918F01882351F02D
:105A3000082E000C990B0E94386F0F5F1F4FF80162
:105A40008491F4CF8091190F882359F18091E4104B
:105A5000882329F180918E1190918F11A09190113E
:105A6000B09191110097A105B105C1F0BC01CD0124
:105A70006D597F4F8F4F9F4F24E630E040E050E05C
:105A80000E9482DD60919211709193118091941126
:105A9000909195110E9482DD822F01C080E090E0FC
:105AA000E6CEE7E3FDE084918F01882309F4E3CE9D
:105AB000082E000C990B0E94386F0F5F1F4FF801E2
:105AC0008491F3CFEFE2FDE084918F01882309F404
:105AD000D2CE082E000C990B0E94386F0F5F1F4F1B
:105AE000F8018491F3CFEAE2FDE084918F018823ED
:105AF00051F0082E000C990B0E94386F0F5F1F4F5A
:105B0000F8018491F4CF80912A1390912B13A091E6
:105B10002C13B0912D13892B8A2B8B2B09F477C072
:105B20000E94A551A50194010E9482DD69017A01BC
:105B300060912A1370912B1380912C1390912D1347
:105B4000A50194010E9482DD8601021B130BC8018E
:105B50006CE370E00E94B5E0CB019927EAE0F0E049
:105B6000BF010E94C9E0282FCB01BF010E94C9E0FC
:105B7000805D80932904205D20932A0410922B04D9
:105B800089E294E00E9436C980E290E00E94386F7A
:105B9000E8E2FDE084917F01882359F0082E000C93
:105BA000990B0E94386FFFEFEF1AFF0AF7018491FB
:105BB000F3CF80E290E00E94386FC8016CE370E0A0
:105BC0000E94B5E06AE070E00E94C9E0605D609309
:105BD0002904805D80932A0410922B0489E294E0CA
:105BE0000E9436C980E290E00E94386FE6E2FDE054
:105BF00084918F01882309F43ECE082E000C990B66
:105C00000E94386F0F5F1F4FF8018491F3CF80E23D
:105C100090E00E94386FEEE1FDE084918F018823CF
:105C200009F429CE082E000C990B0E94386F0F5FE3
:105C30001F4FF8018491F3CF109254138091090102
:105C400080FF11C0EAE1FDE084918F01882309F40F
:105C500012CE082E000C990B0E94386F0F5F1F4F59
:105C6000F8018491F3CF83E50E94D2C8882341F0E4
:105C70000E94EDC80E9429DF7093291360932813B6
:105C8000E6E1FDE084918F01882351F0082E000C9D
:105C9000990B0E94386F0F5F1F4FF8018491F4CF6A
:105CA0008DE090E00E94386F8AE090E00E94386FAB
:105CB00080917213882309F442C280912813909135
:105CC00029138430910509F4C8C08830910509F47E
:105CD0007DC1892B09F0E7C3EAE3FBE084918F01E2
:105CE000882351F0082E000C990B0E94386F0F5F2B
:105CF0001F4FF8018491F4CF8DE090E00E94386F3F
:105D00008AE090E00E94386FEFE2FBE084918F011F
:105D1000882351F0082E000C990B0E94386F0F5FFA
:105D20001F4FF8018491F4CF8DE090E00E94386F0E
:105D30008AE090E00E94386FE3E2FBE084918F01FB
:105D4000882351F0082E000C990B0E94386F0F5FCA
:105D50001F4FF8018491F4CF8DE090E00E94386FDE
:105D60008AE090E00E94386FE7E1FBE084918F01C8
:105D7000882351F0082E000C990B0E94386F0F5F9A
:105D80001F4FF8018491F4CF8DE090E00E94386FAE
:105D90008AE090E00E94386FE9E0FBE084918F0197
:105DA000882351F0082E000C990B0E94386F0F5F6A
:105DB0001F4FF8018491F4CF8DE090E00E94386F7E
:105DC0008AE090E00E94386FEBEFFAE084918F0157
:105DD000882351F0082E000C990B0E94386F0F5F3A
:105DE0001F4FF8018491F4CF8DE090E00E94386F4E
:105DF0008AE090E00E94386FEEEEFAE084918F0125
:105E0000882351F0082E000C990B0E94386F0F5F09
:105E10001F4FF8018491F4CF8DE090E00E94386F1D
:105E20008AE090E00E94386FE1EEFAE084918F0101
:105E3000882351F0082E000C990B0E94386F0F5FD9
:105E40001F4FF8018491F4CF8DE090E00E94386FED
:105E50008AE090E00E94386F26C3E3EDFAE0849177
:105E60008F01882351F0082E000C990B0E94386F87
:105E70000F5F1F4FF8018491F4CF8DE090E00E94F6
:105E8000386F8AE090E00E94386FE5ECFAE0849188
:105E90008F01882351F0082E000C990B0E94386F57
:105EA0000F5F1F4FF8018491F4CF8DE090E00E94C6
:105EB000386F8AE090E00E94386FEFEAFAE0849150
:105EC0008F01882351F0082E000C990B0E94386F27
:105ED0000F5F1F4FF8018491F4CF8DE090E00E9496
:105EE000386F8AE090E00E94386FE9E9FAE0849127
:105EF0008F01882351F0082E000C990B0E94386FF7
:105F00000F5F1F4FF8018491F4CF8DE090E00E9465
:105F1000386F8AE090E00E94386FE7E8FAE08491F9
:105F20008F01882351F0082E000C990B0E94386FC6
:105F30000F5F1F4FF8018491F4CF8DE090E00E9435
:105F4000386F8AE090E00E94386FE5E7FAE08491CC
:105F50008F01882351F0082E000C990B0E94386F96
:105F60000F5F1F4FF8018491F4CF8DE090E00E9405
:105F7000386F8AE090E00E94386FE7E6FAE084919B
:105F80008F01882351F0082E000C990B0E94386F66
:105F90000F5F1F4FF8018491F4CF8DE090E00E94D5
:105FA000386F8AE090E00E94386FE9E5FAE084916A
:105FB0008F01882309F448CF082E000C990B0E940A
:105FC000386F0F5F1F4FF8018491F3CFE2E5FAE0DD
:105FD00084918F01882351F0082E000C990B0E94A8
:105FE000386F0F5F1F4FF8018491F4CF8DE090E080
:105FF0000E94386F8AE090E00E94386FEBE4FAE08C
:1060000084918F01882351F0082E000C990B0E9477
:10601000386F0F5F1F4FF8018491F4CF8DE090E04F
:106020000E94386F8AE090E00E94386FE4E3FAE063
:1060300084918F01882351F0082E000C990B0E9447
:10604000386F0F5F1F4FF8018491F4CF8DE090E01F
:106050000E94386F8AE090E00E94386FEDE1FAE02C
:1060600084918F01882351F0082E000C990B0E9417
:10607000386F0F5F1F4FF8018491F4CF8DE090E0EF
:106080000E94386F8AE090E00E94386FE6E0FAE004
:1060900084918F01882351F0082E000C990B0E94E7
:1060A000386F0F5F1F4FF8018491F4CF8DE090E0BF
:1060B0000E94386F8AE090E00E94386FEFEEF9E0BE
:1060C00084918F01882351F0082E000C990B0E94B7
:1060D000386F0F5F1F4FF8018491F4CF8DE090E08F
:1060E0000E94386F8AE090E00E94386FE1EEF9E09C
:1060F00084918F01882351F0082E000C990B0E9487
:10610000386F0F5F1F4FF8018491F4CF8DE090E05E
:106110000E94386F8AE090E00E94386FE3EDF9E06A
:1061200084918F01882309F48FCE082E000C990BDF
:106130000E94386F0F5F1F4FF8018491F3CF809159
:10614000190F882309F486C181E08093961110927B
:1061500098111092971188E69FE00E94B1948BE10C
:10616000E8E6FFE0DE01159601900D928A95E1F7D1
:106170008091660F9091670F9C838B838DEE92E0E8
:106180009A83898340E050E0BE016F5F7F4F80E0DB
:1061900090E00E946E71CE0101960E949F9BC0907C
:1061A0009711D09098110091281310912913C601CE
:1061B000801B910B049720F06801F3E0CF0ED11CF7
:1061C00054EC452E59E0552E65EB662E69E0762E8F
:1061D000C016D10608F467C10115110509F0A1C068
:1061E0006CE17FE088E69FE00E94799362E273E0D1
:1061F0008CE19FE00E943BE1892B09F04AC0F2014B
:10620000849144ECE42E49E0F42E882359F0082EC2
:10621000000C990B0E94386FFFEFEF1AFF0AF7018D
:106220008491F3CF8DE090E00E94386F8AE090E097
:106230000E94386FF301849135EBE32E39E0F32EA1
:10624000882359F0082E000C990B0E94386FFFEF3D
:10625000EF1AFF0AF7018491F3CF8DE090E00E94DE
:10626000386F8AE090E00E94386F4AE060E070E0AA
:10627000CB010E948FC5E5EAF9E084917F012FEF01
:10628000E21AF20A882309F4E2C00E9488C5F701E5
:10629000F4CFE1EAF9E084917F01882359F0082ED8
:1062A000000C990B0E94386FFFEFEF1AFF0AF701FD
:1062B0008491F3CF8DE090E00E94386F8AE090E007
:1062C0000E94386FF10184912DE9E22E29E0F22E2F
:1062D000882359F0082E000C990B0E94386FFFEFAD
:1062E000EF1AFF0AF7018491F3CF8DE090E00E944E
:1062F000386F8AE090E00E94386F4AE060E070E01A
:10630000CB010E948FC5E8E9F9E084917F012FEF6E
:10631000E21AF20A882309F49AC00E9488C5F7019C
:10632000F4CF60E070E0C80101970E94347380915F
:106330001A0F882309F45FC0E6E9F9E084917F0130
:10634000882359F0082E000C990B0E94386FFFEF3C
:10635000EF1AFF0AF7018491F3CF8CE19FE00E94CE
:1063600036C98DE090E00E94386F8AE090E00E948C
:10637000386FE4E9F9E084917F01882359F0082E11
:10638000000C990B0E94386FFFEFEF1AFF0AF7011C
:106390008491F3CF89E29FE00E9436C98DE090E0BE
:1063A0000E94386F8AE090E00E94386FC801A0E038
:1063B000B0E04AE0BC01CD010E948FC5E2E9F9E0FE
:1063C00084917F012FEFE21AF20A882321F00E94C4
:1063D00088C5F701F5CF99E2E92E9FE0F92EF70184
:1063E00081917F01882319F00E9488C5F8CF8AE047
:1063F0000E9488C52CC08CE19FE00E9436C98DE0C8
:1064000090E00E94386F8AE090E00E94386F89E245
:106410009FE00E9436C98DE090E00E94386F8AE0CC
:1064200090E00E94386FC801A0E0B0E04AE0BC01F3
:10643000CD010E948FC589E2E82E8FE0F82EF7018A
:1064400081917F01882399F20E9488C5F8CF0F5F60
:106450001F4FBECEE3E8F9E084918F01882351F00D
:10646000082E000C990B0E94386F0F5F1F4FF80128
:106470008491F4CF8DE090E00E94386F8AE090E044
:106480000E94386FE4E7F9E084918F01882309F4D2
:10649000DBCC082E000C990B0E94386F0F5F1F4F4A
:1064A000F8018491F3CFE2E1FDE084918F0188232C
:1064B00009F4E1C9082E000C990B0E94386F0F5F98
:1064C0001F4FF8018491F3CF8091180F882339F082
:1064D0000E94A0709FC48091180F8823E9F00E9449
:1064E00032A498C480912613823019F0833609F0C3
:1064F00091C40E947F70EEE0FDE084918F018823BB
:1065000009F4B9C9082E000C990B0E94386F0F5F6F
:106510001F4FF8018491F3CF80912613833609F041
:1065200079C4DDCF85E09DE00E94C29B80919A0EE8
:1065300090919B0E891B8F7009F06CC4809126137B
:10654000823009F467C4833609F098C463C48DE0CF
:1065500090E00E94386F8AE090E00E94386F8BC90B
:1065600080919A0E90919B0E891B8F7009F052C4F6
:1065700080912613823009F44DC4833609F44AC44D
:106580008091E4108111CEC445C483E50E94D2C835
:10659000811126C083E40E94D2C8882309F43AC43A
:1065A00080919A0E90919B0E891B8F7009F032C4D6
:1065B00020E030E040E251E460913A0470913B0405
:1065C00080913C0490913D040E9494D987FF08C0BB
:1065D00082EF9CE090938B0C80938A0C0E945E8BE0
:1065E0000E94EDC820E030E0A9010E9494D987FD07
:1065F00010C00E94EDC820E030E849E853E40E9452
:1066000006E018164CF00E94EDC80E9429DFCB016D
:1066100005C080E090E002C083E191E00E949A52C0
:10662000F9C383E50E94D2C8882309F4F3C30E940A
:10663000EDC820E030E0A9010E9494D987FD10C088
:106640000E94EDC820E030E046E153E40E9406E0FD
:1066500018164CF00E94EDC80E9429DFCB0105C03E
:1066600080E090E002C086E990E00E94B33CD2C393
:1066700083E50E94D2C88823D9F00E94EDC820E0AB
:1066800030E04FE753E40E94F9D920E030E048ECD5
:1066900052E40E94BCDE0E9429DF6F3F710519F0B1
:1066A00010F06FEF70E07093430460934204E3C80E
:1066B0008FEF90E09093430480934204DCC8809174
:1066C0009A0E90919B0E891B8F7009F0D4C880910F
:1066D000180F8111D0C80E942B7F5F9A80913104DE
:1066E0008E7F809331048A9A479A809131048D7FFE
:1066F0008093310480910801809581708093060118
:10670000479A809131048B7F80933104129AB3C8E9
:1067100083E50E94D2C8882319F10E94EDC820E0C9
:1067200030E040E252E40E9494D987FD0FC00E94FD
:10673000EDC820E030EC49E754E40E9406E018166A
:1067400044F00E94EDC80E9424DF05C068E270E0BA
:1067500002C067EE73E070930302609302025AC3B3
:10676000ECEEFCE084918F01882351F0082E000CA0
:10677000990B0E94386F0F5F1F4FF8018491F4CF7F
:10678000C0900202D09003020D2C000CEE08FF080E
:10679000F7FE0DC06DE281E894E1DDD5662777272D
:1067A000CB016C197D098E099F094AE003C04AE0BC
:1067B000C701B6010E94F6C85EC880919A0E9091FA
:1067C0009B0E891B8F7009F025C3809126138230A0
:1067D00009F420C3833609F0EBC21CC380919A0EE2
:1067E00090919B0E891B8F7009F045C880912613EC
:1067F000823009F440C8833609F0B6C33CC88091A2
:106800009A0E90919B0E891B8F7009F003C38091A3
:106810002613823009F4FEC2833609F0FBC4FAC2A3
:1068200080919A0E90919B0E891B8F7009F0F2C295
:1068300080912613823009F4EDC2833609F020C519
:10684000E9C280919A0E90919B0E891B8F7009F07E
:10685000E1C280912613823009F4DCC2833609F04C
:1068600045C5D8C280915413811103C00E943D6F69
:10687000C4C18E3271F5809155138E3209F046C134
:106880008091B910882309F4B8C181508093B91060
:10689000882361F090E001974FE1489F9001499F64
:1068A000300D1124C9018D57904F02C085E49FE03F
:1068B0002BE1FC013496A8E6BFE001900D922A95E9
:1068C000E1F7FC01828193819093670F8093660FBB
:1068D00094C18C3309F01AC164E273E084E593E15A
:1068E0000E943BE1892B21F481E08093721385C1E2
:1068F00063E373E084E593E10E943BE1892B79F443
:10690000E0E5F9E084918F010F5F1F4F882321F0AC
:106910000E9488C5F801F6CF83E399E0E4C06AE4F9
:1069200073E084E593E10E943BE1892B79F4EFE089
:10693000F9E084918F010F5F1F4F882321F00E949F
:1069400088C5F801F6CF8CEF98E0CDC061E673E022
:1069500084E593E10E943BE1892B79F4E1EEF8E0D4
:1069600084918F010F5F1F4F882321F00E9488C5FB
:10697000F801F6CF8CED98E0B6C06FE673E084E5E1
:1069800093E10E943BE1892B79F4E1ECF8E08491FA
:106990008F010F5F1F4F882321F00E9488C5F801E7
:1069A000F6CF8CEB98E09FC06DE773E084E593E150
:1069B0000E943BE1892B79F4E1EAF8E084918F01B0
:1069C0000F5F1F4F882321F00E9488C5F801F6CF82
:1069D00088E998E088C06BE873E084E593E10E9461
:1069E0003BE1892B71F405E718E0F80184918823D5
:1069F00029F00F5F1F4F0E9488C5F7CF8EE698E001
:106A000072C061EA73E084E593E10E943BE1892B67
:106A100079F4EFE4F8E084918F010F5F1F4F882332
:106A200021F00E9488C5F801F6CF88E498E05BC0A9
:106A300063EB73E084E593E10E943BE1892B79F4F9
:106A4000E0E3F8E084918F010F5F1F4F882321F06E
:106A50000E9488C5F801F6CF8FE198E044C06EEB44
:106A600073E084E593E10E943BE1892B79F4E6E051
:106A7000F8E084918F010F5F1F4F882321F00E945F
:106A800088C5F801F6CF84EF97E02DC06AEC73E07B
:106A900084E593E10E943BE1892B79F4E9EDF7E08D
:106AA00084918F010F5F1F4F882321F00E9488C5BA
:106AB000F801F6CF87EC97E016C068ED73E084E547
:106AC00093E10E943BE1892BA9F4EDEAF7E0849180
:106AD0008F010F5F1F4F882321F00E9488C5F801A6
:106AE000F6CF8BE997E090938B0C80938A0C0E94F1
:106AF0005E8B83C065EE73E084E593E10E943BE129
:106B0000892B09F07AC01092721377C01D82188603
:106B10001C821B828DEE92E09A83898380916B0F99
:106B2000811103C065E47FE002C064E67FE0611587
:106B3000710519F06C5F7F4F02C060E070E021E0EA
:106B400044E553E1CE0105960E94E098882361F167
:106B50008BE1FE013596A8E6BFE001900D928A9583
:106B6000E1F72B813C813093670F2093660F809172
:106B7000B9108A3008F03DC091E0980F9093B91099
:106B8000FFE18F9FC0011124DC01A957B04F4BE1F9
:106B9000E8E6FFE001900D924A95E1F7FC01ED5720
:106BA000F04F3383228325C0EBE9FBE184918F0111
:106BB0000F5F1F4F882321F00E9488C5F801F6CF90
:106BC000E5E8F7E084918F010F5F1F4F882321F0E4
:106BD0000E9488C5F801F6CF04E513E1F801819120
:106BE0008F01882319F00E9488C5F8CF8AE00E949F
:106BF00088C5CE0101960E949F9B109254138091EC
:106C0000090180FF07C1E0E3FCE084918F01882344
:106C100011F40C943B2C082E000C990B0E94386F39
:106C20000F5F1F4FF8018491F2CF8FE40E94D2C80A
:106C300081110C943B2C83E40E94D2C80C943B2C11
:106C400083E50E94D2C8811159C08FE40E94D2C846
:106C5000882319F088EF9BE007C084E50E94D2C822
:106C6000882349F080ED9BE090938B0C80938A0CF5
:106C70000E945E8B43C083E40E94D2C8882319F02F
:106C800087EA9BE0F1CF81E50E94D2C8882319F002
:106C90008FE79BE0E9CF88E40E94D2C88823C9F03F
:106CA000EBE7FBE084918F01882351F0082E000C64
:106CB000990B0E94386F0F5F1F4FF8018491F4CF3A
:106CC0008DE090E00E94386F8AE090E00E94386F7B
:106CD00015C08CE40E94D2C8882381F0E7E7FBE06E
:106CE00084918F01882361F3082E000C990B0E9478
:106CF000386F0F5F1F4FF8018491F4CFEFE3FCE092
:106D000084918F01882311F40C943B2C082E000CE5
:106D1000990B0E94386F0F5F1F4FF8018491F2CFDB
:106D200080919A0E80919B0E0C943B2C83E50E94DF
:106D3000D2C8882309F46EC08FE49BE090938B0C3B
:106D400080938A0C0E945E8BEFE3FCE084918F01BC
:106D5000882311F40C943B2C082E000C990B0E94F4
:106D6000386F0F5F1F4FF8018491F2CFEAE4FBE028
:106D700084918F01882351F0082E000C990B0E94FA
:106D8000386F0F5F1F4FF8018491F4CFE5E4FBE00B
:106D900084918F01882311F40C943B2C082E000C55
:106DA000990B0E94386F0F5F1F4FF8018491F2CF4B
:106DB00088E50E94D2C8811106C089E50E94D2C828
:106DC000882309F4C3C088E50E94D2C8882341F013
:106DD00086EE9CE090938B0C80938A0C0E945E8BD5
:106DE00089E50E94D2C8882341F080EE9CE0909310
:106DF0008B0C80938A0C0E945E8B8AE50E94D2C81D
:106E0000882341F08AED9CE090938B0C80938A0C50
:106E10000E945E8B80911F1390912013019664E075
:106E200070E00E94C9E09093201380931F1380911B
:106E30001B1390911C13019690931C1380931B13AA
:106E400010922313109222130C941C2B40911F13A9
:106E5000509120139F012F5F3F4F309323132093B6
:106E6000221390E6949F9001959F300D1124255692
:106E70003E4EE20FF31F80830C941C2B00912413D1
:106E800010912513780124E0E20EF11C6AE270E013
:106E9000C7010E9430E1F80124812F3221F4B801AA
:106EA0006B5F7F4F03C02C3339F4B70184E593E166
:106EB0000E9444E10C943B2C10925413009719F05B
:106EC000FC0131971082809124139091251340E0AA
:106ED00061E004960E9412C78091E410882389F033
:106EE000E1E0FDE084918F01882309F430CB082E86
:106EF000000C990B0E94386F0F5F1F4FF8018491AF
:106F0000F3CFEDEFFCE084918F01882309F41FCBD0
:106F1000082E000C990B0E94386F0F5F1F4FF8016D
:106F20008491F3CF0E947F70E9EFFCE084918F01A0
:106F3000882311F40C943B2C082E000C990B0E9412
:106F4000386F0F5F1F4FF8018491F2CF8AE50E94DE
:106F5000D2C8811138CF83E40E94D2C8882309F4B3
:106F600059CF86ED9CE050CF86E40E94D2C888239A
:106F700009F44DC10E94EDC80E9429DF8B0182ED0A
:106F80009CE090938B0C80938A0C0E945E8B88E52A
:106F90000E94D2C8882309F451C00E94EDC82B0179
:106FA0003C012DEC3CEC4CE45EE30E9494D99E0144
:106FB0002F5F3F4F7901181674F020E030E0A901EF
:106FC000C301B2010E9406E018162CF41F930F9320
:106FD00087EC9CE005C12DEC3CEC4CEC5DEBC30177
:106FE000B2010E9494D918167CF020E030E040E80D
:106FF0005FEBC301B2010E9406E018162CF41F9348
:107000000F938BEB9CE0ECC01F930F93C301B20175
:107010000E9424DF7F936F9381EB9CE09F938F937B
:10702000FF92EF920E9466D90FB6F894DEBF0FBEB2
:10703000CDBFCE0101960E94368BDFC089E50E944C
:10704000D2C8882309F441C00E94EDC82B013C013D
:107050002DEC3CEC4CE45EE30E9494D9FE013196A9
:107060007F01181674F020E030E0A901C301B201DD
:107070000E9406E018162CF41F930F9386EA9CE0FA
:10708000AFC02DEC3CEC4CEC5DEBC301B2010E94B7
:1070900094D918167CF020E030E040E85FEBC301A3
:1070A000B2010E9406E018162CF41F930F938AE990
:1070B0009CE096C01F930F93C301B2010E9424DF8E
:1070C0007F936F9380E99CE0A9CF8AE50E94D2C8A4
:1070D000882309F441C00E94EDC82B013C012DEC2E
:1070E0003CEC4CE45EE30E9494D9FE0131967F01B2
:1070F000181674F020E030E0A901C301B2010E942B
:1071000006E018162CF41F930F9385E89CE068C0E6
:107110002DEC3CEC4CEC5DEBC301B2010E9494D928
:1071200018167CF020E030E040E85FEBC301B201CC
:107130000E9406E018162CF41F930F9389E79CE039
:107140004FC01F930F93C301B2010E9424DF7F93AE
:107150006F938FE69CE062CF85E40E94D2C88823BB
:1071600009F44BC00E94EDC82B013C012DEC3CEC16
:107170004CE45EE30E9494D9FE0131967F0118161B
:1071800074F020E030E0A901C301B2010E9406E0E2
:1071900018162CF41F930F9384E69CE021C02DEC6D
:1071A0003CEC4CEC5DEBC301B2010E9494D9181683
:1071B0007CF020E030E040E85FEBC301B2010E94C8
:1071C00006E018162CF41F930F9388E59CE008C086
:1071D000C301B2010E9424DF7F936F938DE49CE092
:1071E0009F938F93FF92EF920E9466D90F900F901A
:1071F0000F900F900F900F901CCF89E49CE090931C
:107200008B0C80938A0C0E945E8B0C943B2C00E0CC
:1072100010E0B5CE20E030E040E251E460913A0465
:1072200070913B0480913C0490913D040E9494D95C
:1072300087FF08C082E49CE090938B0C80938A0CBB
:107240000E945E8B82E390E0909345048093440417
:107250000E94B07588EC90E00E949A52EFE3FCE047
:1072600084918F01882311F40C943B2C082E000C80
:10727000990B0E94386F0F5F1F4FF8018491F2CF76
:1072800020E030E040E251E460913A0470913B0428
:1072900080913C0490913D040E9494D987FF08C0DE
:1072A00088E39CE090938B0C80938A0C0E945E8B09
:1072B00080E590E090934504809344040E94B0756B
:1072C00080EF90E00E949A52EFE3FCE084918F01FE
:1072D000882311F40C943B2C082E000C990B0E946F
:1072E000386F0F5F1F4FF8018491F2CF80E090E07C
:1072F0000E949A5210924504109244040E94B07564
:10730000E4E3FCE084918F01882311F40C943B2C7E
:10731000082E000C990B0E94386F0F5F1F4FF80169
:107320008491F2CF6F960FB6F894DEBF0FBECDBF3B
:10733000DF91CF911F910F91FF90EF90DF90CF9051
:10734000BF90AF909F908F907F906F905F904F9085
:107350003F902F9008950F931F93CF93DF93FC01DD
:10736000A685B7858D0100581F4FE8018881998156
:1073700001968F779927AD014E575F4FEA0128811B
:10738000398128173907D1F3E80128813981A20F03
:10739000B31F6C93A685B785A058BF4F11969C93D9
:1073A0008E93A689B7892C9181E090E0078C02C06A
:1073B000880F991F0A94E2F7822B8C9381E081A3B6
:1073C0000488F589E02D80818064808381E090E0ED
:1073D000DF91CF911F910F910895FC0181A1882326
:1073E00029F0A489B5898C9186FFFBCF11A208955D
:1073F000FC01A485B585FD01E058FF4F2081318156
:107400003296808191812817390779F080819181A6
:10741000A80FB91F8C91208131812F5F3F4F2F77AB
:1074200033273183208390E008958FEF9FEF0895F5
:10743000DC011C96ED91FC911D97DF01A058BF4F18
:107440002D913C91119712968D919C91119728172F
:10745000390739F08D919C91E80FF91F808190E0F8
:1074600008958FEF9FEF0895FC0124853585F9017C
:10747000E058FF4F80819181329620813181805880
:107480009F4F821B930B60E870E00C94C9E0089555
:10749000089580E090E00895CF92DF92EF92FF92FE
:1074A000C0904902D0904A02E0904B02F0904C020A
:1074B000FC0180819181A281B381809349029093E4
:1074C0004A02A0934B02B0934C020E9421BCC0928E
:1074D0004902D0924A02E0924B02F0924C02FF9095
:1074E000EF90DF90CF90089580911504909116044D
:1074F000009731F04AE050E060E070E00C94E8D68C
:1075000060E070E0CB010895EFDF97FD0AC0ECDF8B
:107510006F3F71058105910509F02CF4E5DF862F99
:10752000089580E008958FEF08958091150490915B
:107530001604892B31F0E8DF91E0811103C090E05F
:1075400001C091E0892F08950F931F93CF938091ED
:10755000150490911604009711F1FC018F01C1915F
:107560002C2F2F7DA9F0C53411F0C536B9F7F801DD
:10757000108260E070E080911504909116040E94E2
:1075800095D5F801C083562F472F382F292F0BC0D0
:1075900060E070E0CF911F910F910C9495D550E071
:1075A00040E030E020E0652F742F832F922FCF91A1
:1075B0001F910F91089581548A3108F042C0E82F3D
:1075C000F0E04091BA165091BB166091BC167091D4
:1075D000BD1604C076956795579547958A95D2F75D
:1075E000842F817040FF2FC0E056F94E908199237F
:1075F00009F1E091D715F091D815E90FF11D9081AF
:1076000020ED290F2A3098F09E3211F491810CC0A0
:107610009D3211F09B3271F4918120ED290F2A30B7
:1076200030F09E3239F4928190539A3018F42E2F14
:107630009F2F02C020E090E0209315049093160441
:10764000089580E008950895B6DF882341F081E031
:107650002091150430911604232B09F480E008953D
:1076600080E1E2E3F4E0A3E1B6E101900D928A95B6
:10767000E1F708952F923F924F925F926F927F921F
:107680008F929F92AF92BF92CF92DF92EF92FF9232
:107690000F931F93CF93DF9300D01F921F92CDB70C
:1076A000DEB77C018B016A01190180903204909051
:1076B0003304A0903404B0903504A5019401FC017A
:1076C00060817181828193810E9494D9F1E0FD8370
:1076D000811112C020913604309137044091380452
:1076E00050913904F80160817181828193810E94F7
:1076F00094D9811101C01D82F601408051806280C1
:10770000738020910402309105024091060250914D
:107710000702C301B2010E9494D9882309F453C01F
:107720004092040250920502609206027092070293
:1077300020E030E040E450E460916D0C70916E0CFC
:1077400080916F0C9091700C0E94BCDE69837A83EB
:107750008B839C838092131690921416A092151618
:10776000B09216168091360490913704A091380497
:10777000B09139048093171690931816A093191698
:10778000B0931A16F60180819181A281B381809312
:107790001B1690931C16A0931D16B0931E16809175
:1077A0003E0490913F04A0914004B0914104809325
:1077B0001F1690932016A0932116B0932216CE0187
:1077C00001966ADE4DDFFD81FF2309F16090690CAF
:1077D00070906A0C80906B0C90906C0CA090650C73
:1077E000B090660CC090670CD090680C9501A60113
:1077F000B301C4010E9406E0181614F0530164019D
:1078000020E030E040E251E4B501C6010CC020E0C8
:1078100030E040EC5FE36091710C7091720C8091EC
:10782000730C9091740C0E94BCDE69837A838B8305
:107830009C8320911404222349F0AB01BC0189E907
:107840009DE00E94A3508AE00E9488C5F7018081D4
:107850009181A281B3818093131690931416A09303
:107860001516B0931616F80180819181A281B3811B
:107870008093171690931816A0931916B0931A16A2
:10788000F101208131814281538160911F167091F5
:10789000201680912116909122160E94E0DD6093BF
:1078A0001F16709320168093211690932216CE01F6
:1078B0000196F2DDD5DE0F900F900F900F900F9094
:1078C000DF91CF911F910F91FF90EF90DF90CF90BC
:1078D000BF90AF909F908F907F906F905F904F90F0
:1078E0003F902F90089580E1E3E1F6E1A2E3B4E058
:1078F00001900D928A95E1F708959C0197FD0EC0C5
:107900008436910584F064E670E00E94C9E0CB0102
:107910006AE070E00E94C9E0805D06C03195219563
:1079200031098DE201C080E280932D042A303105B7
:1079300064F0EAE0F0E0C901BF010E94C9E0CB01B8
:10794000BF010E94C9E0805D01C080E280932E04E7
:10795000C9016AE070E00E94C9E0805D80932F0455
:107960008DE294E008958E3691051CF02EE680E0BD
:1079700002C0282F892F20934404809345040C943F
:10798000B0752F923F924F925F926F927F928F923B
:107990009F92AF92BF92CF92DF92EF92FF920F939E
:1079A0001F93CF93DF93CDB7DEB7C455D1090FB680
:1079B000F894DEBF0FBECDBFE8E5F0E184918F0102
:1079C0000F5F1F4F882321F00E9488C5F801F6CF72
:1079D0000E948DA781110C94A74680E090E0A0E85A
:1079E000BFE380930B1690930C16A0930D16B093E3
:1079F0000E1680930F1690931016A0931116B09345
:107A000012168DEC9CECACE4BEE3809307169093C9
:107A10000816A0930916B0930A1680E090E0A0E241
:107A2000B1E48093C1049093C204A093C304B093C3
:107A3000C4048CE390E09093C0048093BF048DEC69
:107A400090E09093BE048093BD041092BC048FE438
:107A5000FBDD882311F078DD04C06AE979E989E962
:107A60009EE36BAF7CAF8DAF9EAF83E4EDDD8823EB
:107A700011F05BDD02C083E49EDD61968FAF6197FC
:107A80008BE4E2DD882311F050DD02C08BE493DD4E
:107A900060968FAF609782E4D7DD8823E9F054DDEC
:107AA0000E9424DF7093C0046093BF0461157105C8
:107AB00099F0685271096536710570F0E3E2F0E102
:107AC00084918F010F5F1F4F882311F40C94A746F8
:107AD0000E9488C5F801F4CF8CE4B6DD882351F10B
:107AE00033DD6B017C016093071670930816809359
:107AF000091690930A1620E030E0A9010E9406E0E2
:107B000087FD0AC020E030E040E050E4C701B60144
:107B10000E9494D9181674F4EBEFFFE084918F0162
:107B20000F5F1F4F882311F40C94A7460E9488C54D
:107B3000F801F4CF81E53FDD882309F440C080914E
:107B4000150490911604892B19F4E0EDFFE02BC089
:107B5000FBDC6B017C0160930F1670931016809311
:107B60001116909312162DEC3CEC4CE45DE30E9450
:107B700006E087FD0AC020E030E040E751E4C7019D
:107B8000B6010E9494D91816D4F4EFE9FFE084916D
:107B90008F010F5F1F4F882311F40C94A7460E949A
:107BA00088C5F801F4CF84918F010F5F1F4F8823A0
:107BB00011F40C94A7460E9488C5F801F4CF83E520
:107BC00043DD882319F1C0DC4B015C012DEC3CEC5A
:107BD0004CEC5DE30E9406E087FD0AC020E030E047
:107BE00040E85FE3C501B4010E9494D91816ACF4D3
:107BF000E8E7FFE084918F010F5F1F4F882311F4A6
:107C00000C94A7460E9488C5F801F4CF5DEC852E40
:107C10005CEC952EA92C5EE3B52E80E5CCDC8823A8
:107C200009F443C08091150490911604892B71F4D6
:107C3000E0E4FFE084918F010F5F1F4F882311F470
:107C40000C94A7460E9488C5F801F4CF8091BC042B
:107C50008F5F8093BC0478DC6B017C016093C1046E
:107C60007093C2048093C3049093C40420E030E076
:107C7000A9010E9406E087FD0AC020E030E048EC40
:107C800051E4C701B6010E9494D9181674F4E8E1D2
:107C9000FFE084918F010F5F1F4F882311F40C9434
:107CA000A7460E9488C5F801F4CF86E4CDDC88237E
:107CB00019F14ADC6B017C0120E030E040E85FE331
:107CC0000E9406E087FD0AC020E030E040E850E472
:107CD000C701B6010E9494D91816A4F4EFEEFEE095
:107CE00084918F010F5F1F4F882311F40C94A746D6
:107CF0000E9488C5F801F4CFC12CD12C40EEE42EAF
:107D00004FE3F42EA7019601C701B6010E94F9D9ED
:107D10009B01AC0160E070E084E490E40E94BCDE72
:107D200020910B1630910C1640910D1650910E16A5
:107D30000E94F9D92B013C01A5019401C501B401B0
:107D40000E94F9D9A70196010E94F9D92CEE31E5DC
:107D500048EB5DE30E94BCDE9B01AC01C301B201B4
:107D60000E94F9D960930B1670930C1680930D1630
:107D700090930E1688E468DC8823C9F0E5DB0E9446
:107D800024DF7093BE046093BD04655A71096437A3
:107D9000710568F0E1ECFEE084918F010F5F1F4FE9
:107DA000882309F4D4C70E9488C5F801F5CF85E57A
:107DB00002DC8823E9F00E94A55161157105810557
:107DC000910511F00E948CD58091150490911604B4
:107DD000892B11F0B9DB04C060E070E088E492E424
:107DE0006093B8047093B9048093BA049093BB0471
:107DF00082E5E1DB81110DC0EDE8FEE084918F01A9
:107E00000F5F1F4F882309F4A2C70E9488C5F8019D
:107E1000F5CF8091150490911604892BA9F064DBAD
:107E20002F967FAF6EAF2F97161617069CF0E9E5D9
:107E3000FEE084918F010F5F1F4F882309F487C7ED
:107E40000E9488C5F801F5CF8AE190E02F969FAF98
:107E50008EAF2F9788E5F8DB882361F075DB2091E2
:107E60001704309118044091190450911A040E948B
:107E7000DFDD08C0609132047091330480913404D6
:107E8000909135046093B4047093B5048093B60464
:107E90009093B70489E5D8DB882361F055DB209106
:107EA0001B0430911C0440911D0450911E040E943B
:107EB000DFDD08C06091360470913704809138048A
:107EC000909139046093B0047093B1048093B2042C
:107ED0009093B3046091B4047091B5048091B6049A
:107EE0009091B70440EB54E00E94C3C681110DC0CD
:107EF000EFE2FEE084918F010F5F1F4F882309F4AA
:107F000026C70E9488C5F801F5CF84E454DB91E0D0
:107F100089270E943D8A20E030E040EA50E46091E9
:107F20003A0470913B0480913C0490913D040E947E
:107F300094D987FF14C0198A1A8A1B8A1C8A80E088
:107F400090E0A0EAB0E489839A83AB83BC83BE014E
:107F50006F5E7F4FCE0101960E946FA7C4DC0E9426
:107F6000A5516B017C01A8E8CA0EA3E1DA1EE11C51
:107F7000F11C8091BF049091C004F5DC6091BF04B6
:107F80007091C004072E000C880B990B0E949AD99F
:107F90009B01AC01609146047091470480914804B4
:107FA000909149040E94DFDD4B015C0120E030E04C
:107FB000A9010E9406E087FF04C0B7FAB094B7F8A1
:107FC000B09420E030E040E450E4C501B4010E94E8
:107FD00006E0181604F50E94A551DC01CB018C19AE
:107FE0009D09AE09BF09B7FD0FC00E94A5516B01E5
:107FF0007C01B8E8CB0EB3E1DB1EE11CF11C0E9452
:10800000F6748AE00E9488C50E94099C80914317FB
:1080100080934417B3CF8091BD049091BE040E9419
:108020009A526091BD047091BE04072E000C880B1B
:10803000990B0E949AD99B01AC0160914C047091FC
:108040004D0480914E0490914F040E94DFDD4B015E
:108050005C0120E030E0A9010E9406E087FF04C037
:10806000B7FAB094B7F8B09420E030E040E450E4C0
:10807000C501B4010E9406E0181604F50E94A5513E
:10808000DC01CB018C199D09AE09BF09B7FD0FC0FA
:108090000E94A5516B017C01E8E8CE0EE3E1DE1EF3
:1080A000E11CF11C0E94F6748AE00E9488C50E94BF
:1080B000099C8091431780934417B3CF10923E04DC
:1080C00010923F0410924004109241040E943BA67B
:1080D0008091BC04882399F1C3DA2091C1043091C6
:1080E000C2044091C3045091C40460911F16709162
:1080F000201680912116909122160E94E0DD609357
:108100001F1670932016809321169093221620E05C
:1081100030E040E751E46091710C7091720C8091F5
:10812000730C9091740C0E94BCDE69837A838B83FC
:108130009C83CE010196B0D993DA0E9448A480E2D4
:10814000E0E9F4E0DF01282F1D922A95E9F7E0E746
:10815000F4E0DF01282F1D922A95E9F7E0E5F4E02D
:10816000DF011D928A95E9F77BDA809107169091DD
:108170000816A0910916B0910A1680931B169093C9
:108180001C16A0931D16B0931E1619821A821B820C
:108190001C829E012F5F3F4F4BE156E167E176E184
:1081A00083E196E167DA9E01255C3F4F4BE156E1A2
:1081B00067E176E183E196E15DDA6196BFAD6197B3
:1081C000BB2329F066E374E082E394E004C060EB33
:1081D00074E084EB94E00E94E4CB298F3A8F4B8FBC
:1081E0005C8F6D8F7E8F3FAF2D962FAF2D972D9685
:1081F000EFAD2D97E7FD82C4FFADF7FD7FC424E00E
:10820000E202F0011124EC51F14F40805180628074
:1082100073803FAD84E03802F0011124E053F14F48
:10822000D080C180328023808D2D9C2DA32DB22D36
:108230008FAB98AFA9AFBAAFAE01495C5F4FB20147
:10824000C3010E94C3C6882309F45CC420E030E067
:1082500040EA50E4B201C3010E94E0DDF62E072F90
:10826000182FE92E862F902FA12FBE2D8BAB9CAB04
:10827000ADABBEAB8D2D9C2DA32DB22D8FA798AB92
:10828000A9ABBAAB2D969FAD2D97911152C0AFAD52
:10829000A11105C05F2D402F312F2E2D04C0542D6C
:1082A000452D362D272D852F942FA32FB22F8BAB45
:1082B0009CABADABBEABBFADB43034F4F42C052DEC
:1082C000162DE72CBB2369F020E030E040EA50E4B3
:1082D0006D2D7C2D832D922D0E94DFDD362F272FD3
:1082E00003C09601832D922D432F522FBC014FA71F
:1082F00058AB69AB7AABEFADE4300CF0A7C020E02F
:1083000030E040EA50E46D2D7C2D832D922D0E94AB
:10831000E0DD21966FAF219723967FAF23972596B7
:108320008FAF259727969FAF2797FFADF11185C097
:1083300099C02D962FAD2D9724300CF453C03FAD2E
:1083400034305CF020E030E040EA50E4B201C30198
:108350000E94DFDD362F272F03C0342D252DC301CA
:10836000432F522FBC014BAB5CAB6DAB7EAB8FADE3
:108370008111E4C420E030E040EA50E4B201C301DE
:108380000E94DFDDF62E072F182FE92E20E030E0C7
:1083900040EA50E46D2D7C2D832D922D0E94E0DD6E
:1083A0006FA778AB89AB9AAB9FAD992309F44EC008
:1083B00020E030E040EA50E46D2D7C2D832D922D9D
:1083C0000E94DFDD21966FAF219723967FAF239721
:1083D00025968FAF259727969FAF2797AFADA430EF
:1083E00064F140C0BFADB1110DC020E030E040EA03
:1083F00050E4B201C3010E94DFDDF62E072F182FD3
:10840000E92E0FC0EFADE430B4F120E030E040EAF7
:1084100050E4B201C3010E94DFDD6BAB7CAB8DABDE
:108420009EAB2196DFAE21972396CFAE239725965C
:108430003FAE259727962FAE279732ED832E33E553
:10844000932E3BE7A32E31E4B32E29C02196DFAE55
:1084500021972396CFAE239725963FAE2597279653
:108460002FAE279722ED822E23E5922E2BEFA22E00
:1084700020E4B22E14C02196DFAE21972396CFAE12
:10848000239725963FAE259727962FAE279792EDF7
:10849000892E93E5992E9BEFA92E91E4B92E8BA9F5
:1084A0009CA9ADA9BEA92C968CAF9DAFAEAFBFAFB6
:1084B0002C979C01AD01B201C3010E94DFDD698BE5
:1084C0007A8B8B8B9C8B4FA458A869A87AA8A301A0
:1084D00092016D2D7C2D832D922D0E94DFDD6D8B01
:1084E0007E8B8F8B988F2C962CAD3DAD4EAD5FADB6
:1084F0002C976091320470913304809134049091F0
:1085000035040E94DFDD2C966CAF7DAF8EAF9FAF40
:108510002C97A301920160913604709137048091E9
:108520003804909139040E94DFDD2B013C018F2D2E
:10853000902FA12FBE2D89839A83AB83BC83219674
:108540008FAD219723969FAD23972596AFAD2597A5
:108550002796BFAD27978D839E83AF83B887809181
:10856000071690910816A0910916B0910A168987EE
:108570009A87AB87BC872DEC3CEC4CEC5CE3C501E7
:10858000B4010E94F9D920910B1630910C1640913C
:108590000D1650910E160E94F9D920913E0430918B
:1085A0003F0440914004509141040E94E0DD6D87FA
:1085B0007E878F87988B2C962CAD3DAD4EAD5FADF1
:1085C0002C97CA01B9010E94F9D96B017C01A30162
:1085D0009201C301B2010E94F9D99B01AC01C7010C
:1085E000B6010E94E0DD20E030E040E050E40E946F
:1085F00006E018160CF046C00E9448A41BA21CA25C
:108600001DA21EA220E030E040E05FE360913A044A
:1086100070913B0480913C0490913D040E94E0DD08
:108620006F8F78A389A39AA39E012D5D3F4FAE0162
:10863000415E5F4F66E374E082E394E01BD81BA2C7
:108640001CA21DA21EA220E030E040E05FE360918A
:108650000716709108168091091690910A160E94CB
:10866000E0DD6F8F78A389A39AA39E012D5D3F4F14
:10867000AE01415E5F4FBE01615D7F4FCE01C3968B
:108680000E943A3B1F8E18A219A21AA29E01215ED7
:108690003F4F47E056E1BE01615D7F4FCE01C3967B
:1086A0000E943A3B0E9474A44090490250904A02B2
:1086B00060904B0270904C02E090690CF0906A0C54
:1086C00000916B0C10916C0CA090650CB090660C36
:1086D000C090670CD090680C9501A601B701C80145
:1086E0000E9406E0181614F47501860120E030E0BF
:1086F00040E251E4B701C8010E94BCDE6093490228
:1087000070934A0280934B0290934C0240E0BE016A
:108710006F5E7F4FCE0101960E94CA9F4092490230
:1087200050924A0260924B0270924C020E94303B7F
:10873000A4EEBEE02496BFAFAEAF249722961FAE44
:108740001EAE229701E010E021960FAC219702C0E7
:10875000000F111F0A94E2F72296EEADFFAD2297AB
:1087600031962296FFAFEEAF229721E030E02196BE
:108770000FAC219702C0220F331F0A94E2F76396D1
:108780003FAF2EAF639780E5282E84E0382E80E936
:1087900094E02A969FAF8EAF2A97A0E7B4E0289680
:1087A000BFAFAEAF2897E0EDFEE02696FFAFEEAF8D
:1087B00026972A962EAD3FAD2A9765963FAF2EAFEE
:1087C0006597D9018D919C919C0120233123232B06
:1087D00009F4ADC06396EEADFFAD63978E239F2382
:1087E000892B09F4A4C02896AEADBFAD28978D9112
:1087F0009C9180239123892B09F099C020E030E0DF
:1088000040E050E42496AEADBFAD24976D917D91CC
:108810008D919C910E94E0DD6B017C0120E030E0B5
:1088200040E050E42496EEADFFAD2497648175815D
:10883000868197810E94DFDD4B015C0120E030E002
:1088400040E850ECC701B6010E9494D987FD70C181
:1088500020E030E046E553E4C701B6010E9406E09F
:10886000181634F4C12CD12CB6E5EB2EB3E4FB2E54
:10887000CBA6DCA6EDA6FEA62696AEADBFAD26978E
:108880004D905D906D907C9020E030E040E85FE39B
:10889000C301B2010E9494D987FD51C120E030E0AC
:1088A00046E553E4C301B2010E9406E0181634F411
:1088B000412C512CF6E56F2EF3E47F2E4F8E58A2FB
:1088C00069A27AA24FA258A669A67AA620E030E053
:1088D00040E850ECC501B4010E9494D987FD36C12F
:1088E00020E030E046E553E4C501B4010E9406E013
:1088F000181634F4812C912C76E5A72E73E4B72E4C
:108900008BA29CA2ADA2BEA2AE01495D5F4FC70182
:10891000B6010E94C3C6811120C12896EEADFFADFD
:10892000289780819181802B912B918380832A9637
:108930002EAD3FAD2A972E5F3F4F2A963FAF2EAF09
:108940002A976596AEADBFAD65978D919C918023BA
:108950009123892B09F4A6C0F9018081918180239C
:108960009123892B09F49EC0F1018081918180239C
:108970009123892B09F096C020E030E040E050E4DC
:108980002696AEADBFAD26976D917D918D919C9150
:108990000E94E0DD2B013C0120E030E040E050E4AB
:1089A0002696EEADFFAD269764817581868197810D
:1089B0000E94DFDD4B015C012496AEADBFAD249774
:1089C000CD90DD90ED90FC9020E030E040E850EC60
:1089D000C701B6010E9494D987FDFFC020E030E0B6
:1089E00046E553E4C701B6010E9406E0181634F4C8
:1089F000C12CD12C56E5E52E53E4F52ECBA2DCA2FA
:108A0000EDA2FEA2CBA6DCA6EDA6FEA620E030E0FD
:108A100040E85FE3C301B2010E9494D987FDE4C03E
:108A200020E030E046E553E4C301B2010E9406E0D5
:108A3000181634F4412C512C36E5632E33E4732E92
:108A40004FA258A669A67AA620E030E040E85FE38E
:108A5000C501B4010E9494D987FDCDC020E030E06B
:108A600046E553E4C501B4010E9406E0181634F44B
:108A7000812C912C96E5A92E93E4B92E8F8E98A285
:108A8000A9A2BAA2AE01495D5F4FC701B6010E941B
:108A9000C3C68111B7C0F10180819181802B912BD8
:108AA00091838083F2E02F0E311C28962EAD3FADCE
:108AB00028972E5F3F4F28963FAF2EAF28972696D8
:108AC0008EAD9FAD2697049626969FAF8EAF2697C4
:108AD0009AE5291694E0390609F06BCE2496AEADDE
:108AE000BFAD249714962496BFAFAEAF24972296BD
:108AF000EEADFFAD2297359709F024CE8091431754
:108B0000809344172F962EAD3FAD2F9721503109FA
:108B10002F963FAF2EAF2F97232B09F4B3C02D967E
:108B20003FAD2D9737FDAEC08FAD87FF46CBAAC0B6
:108B3000C12CD12CA0E8EA2EA0ECFA2E99CE412C23
:108B4000512CE0E86E2EEFE37E2EB8CE812C912CD6
:108B500060E8A62E60ECB62ED3CEAE01415E5F4F2C
:108B6000C501B4010E94C3C6882309F4D6CE809102
:108B70001404882321F1B701A60189E09EE00E9438
:108B8000A3504FA158A569A57AA583E09EE00E9455
:108B9000A3504BA15CA16DA17EA189EF9DE00E9435
:108BA000A3504F8D58A169A17AA183EF9DE00E9447
:108BB000A35089E20E9488C58AE00E9488C59E0170
:108BC000215E3F4FAE014D5D5F4FBE01695D7F4F3E
:108BD000CE018B960E94A4A4A0CEC12CD12C40E83B
:108BE000E42E40ECF42E0ACF412C512C20E8622ECA
:108BF0002FE3722E25CF812C912C80E8A82E8FE3B5
:108C0000B82E3CCFAE01415E5F4FC701B6010E9456
:108C1000C3C6882309F43FCF80911404882321F12F
:108C2000B701A6018FEC9DE00E94A3504FA158A56B
:108C300069A57AA589EC9DE00E94A3504BA15CA197
:108C40006DA17EA18FEB9DE00E94A3504F8D58A196
:108C500069A17AA189EB9DE00E94A35089E20E945C
:108C600088C58AE00E9488C59E01215E3F4FAE0103
:108C70004D5D5F4FBE01695D7F4FCE018B960E94B7
:108C8000A4A409CF0E9448A480E090E0A0EAB0E448
:108C900080931B1690931C16A0931D16B0931E165E
:108CA00019821A821B821C829E012F5F3F4F4BE16B
:108CB00056E167E176E183E196E10E943A3B8091DB
:108CC000B4049091B504A091B604B091B704809318
:108CD000131690931416A0931516B0931616809140
:108CE000B0049091B104A091B204B091B304809308
:108CF000171690931816A0931916B0931A16198286
:108D00001A821B821C829E012F5F3F4F4BE156E16E
:108D100067E176E183E196E10E943A3B6096FFAD20
:108D20006097F11114C010924504109244040E94FF
:108D3000B07580E090E00E949A5209C02FADF42CEB
:108D4000052D162DE72C24300CF032CB1FCBCC5A3E
:108D5000DF4F0FB6F894DEBF0FBECDBFDF91CF91CE
:108D60001F910F91FF90EF90DF90CF90BF90AF9049
:108D70009F908F907F906F905F904F903F902F903B
:108D800008951F920F920FB60F9211240BB60F92F7
:108D90002F933F938F939F93EF93FF932091F9131A
:108DA0003091FA138091FB139091FC132817390727
:108DB00031F4809131018F7D8093310114C0E091B5
:108DC000FB13F091FC13E758FC4E20818091FB13BC
:108DD0009091FC1301968F7799279093FC138093C1
:108DE000FB1320933601FF91EF919F918F913F915B
:108DF0002F910F900BBE0F900FBE0F901F901895E4
:108E00001F920F920FB60F9211240BB60F922F9351
:108E10004F935F938F939F93EF93FF9380913001D4
:108E200082FD1CC02091360180917D1490917E14AA
:108E300040917F145091801401968F77992748179D
:108E4000590771F0E0917D14F0917E14E350FC4ECF
:108E5000208390937E1480937D1402C0809136010C
:108E6000FF91EF919F918F915F914F912F910F9073
:108E70000BBE0F900FBE0F901F90189580919A0E09
:108E800090919B0E891B8F7019F480E090E00895FB
:108E90009091970E992351F0833030F48FEF890F22
:108EA00019F08093970EF1CF1092970EE0919B0EE0
:108EB00088E5E89FF0011124EB53FB4F808180FD92
:108EC000E4CF80919B0E8F5F8F708093980E90916E
:108ED0009B0E8091990E981304C08091980E8093F8
:108EE000990ECF0108950F930FB70F9300916E0065
:108EF0000F930B7F00936E0000916F000D7F009326
:108F00006F000F930BB70F930CB70F921F922F9315
:108F10003F934F935F936F937F938F939F93AF9301
:108F2000BF93EF93FF9311244AD0FF91EF91BF912C
:108F3000AF919F918F917F916F915F914F913F91F1
:108F40002F911F900F900CBF0F910BBF0F910260DC
:108F5000F89400936F000F9100936E000F910FBF74
:108F60000F91189580914A0A80FF03C089988FEF6E
:108F700002C0899A81E08093140280914A0A81FF9D
:108F800003C08F9A8FEF02C08F9881E08093150203
:108F900080914A0A82FF09C080910B0180958270FE
:108FA00080930901439A8FEF07C080910B01827073
:108FB00080930901439881E08093160208952F92CF
:108FC0003F924F925F926F927F928F929F92AF9259
:108FD000BF92CF92DF92EF92FF920F931F93CF93A6
:108FE000DF93CDB7DEB72D970FB6F894DEBF0FBE77
:108FF000CDBFF8948FEF9FEF909389008093880006
:109000002AE02987212C312C44244A94542C320103
:1090100078948091960A9091970AA091980AB091BD
:10902000990A892B8A2B8B2B09F010C28091A714E7
:109030008823E1F01092A7148091A5149091A614B2
:10904000892B09F403C210924B0A1092A6141092B5
:10905000A51490919A0E80919B0E981709F4F6C171
:1090600080919B0E8F5F8F7080939B0E8091A514D3
:109070009091A614892B09F4E9C1C090920AD0906E
:10908000930AE090940AF090950A40918E0A5091CC
:109090008F0A6091900A7091910A0091810A10E004
:1090A00020E030E0DB01CA018C199D09AE09BF093F
:1090B000081719072A073B0710F4D901C801482FE0
:1090C0008C0D9D1DAE1DBF1D8093920A9093930A37
:1090D000A093940AB093950A209184003091850062
:1090E000245E3F4FC090670AD090680AE090690AFA
:1090F000F0906A0A8091570A9091580AA091590AF3
:10910000B0915A0A8C0D9D1DAE1DBF1D8093670A3C
:109110009093680AA093690AB0936A0AB7FD1CC0CD
:10912000889AC090E715D090E815E090E915F09086
:10913000EA1580911402082E000C990BAA0BBB0BA8
:109140008C0D9D1DAE1DBF1D8093E7159093E815F6
:10915000A093E915B093EA15C0906B0AD0906C0A01
:10916000E0906D0AF0906E0A80915B0A90915C0A23
:10917000A0915D0AB0915E0A8C0D9D1DAE1DBF1DB4
:1091800080936B0A90936C0AA0936D0AB0936E0A59
:10919000B7FD1CC08E9AC090EB15D090EC15E090F6
:1091A000ED15F090EE1580911502082E000C990B2C
:1091B000AA0BBB0B8C0D9D1DAE1DBF1D8093EB1527
:1091C0009093EC15A093ED15B093EE15C0906F0A37
:1091D000D090700AE090710AF090720A80915F0A54
:1091E0009091600AA091610AB091620A8C0D9D1D58
:1091F000AE1DBF1D80936F0A9093700AA093710AF1
:10920000B093720AB7FD3EC09091490A8091160250
:109210009923C1F09091470A92FF02C087FD05C0D3
:109220009091460A992309F4BEC56091470A70914E
:10923000480A73FF02C087FD0CC09091450A911146
:1092400008C006C090910B01909598709093090109
:10925000419AC090EF15D090F015E090F115F09084
:10926000F215082E000C990BAA0BBB0B8C0D9D1D43
:10927000AE1DBF1D8093EF159093F015A093F115CF
:10928000B093F215C090730AD090740AE090750AFA
:10929000F090760A8091630A9091640AA091650A21
:1092A000B091660A8C0D9D1DAE1DBF1D8093730A83
:1092B0009093740AA093750AB093760AB7FD3AC0EA
:1092C0008090F3159090F415A090F515B090F615D8
:1092D000C09017020C2C000CDD08EE08FF08C80C2B
:1092E000D91CEA1CFB1CC092F315D092F415E09235
:1092F000F515F092F615C090530AD090540AE090FC
:10930000550AF090560A8C199D09AE09BF09809341
:10931000730A9093740AA093750AB093760A909199
:109320004A0A80917F0A93FF02C0815001C08F5F7B
:1093300080937F0A8091670A9091680AA091690AD8
:10934000B0916A0AB7FD15C0C090530AD090540A74
:10935000E090550AF090560A8C199D09AE09BF0994
:109360008093670A9093680AA093690AB0936A0A87
:10937000889880916B0A90916C0AA0916D0AB091C7
:109380006E0AB7FD15C0C090530AD090540AE09001
:10939000550AF090560A8C199D09AE09BF098093B1
:1093A0006B0A90936C0AA0936D0AB0936E0A8E9824
:1093B00080916F0A9091700AA091710AB091720A1F
:1093C000B7FD3AC0C090530AD090540AE090550AB5
:1093D000F090560A8C199D09AE09BF0980936F0A57
:1093E0009093700AA093710AB093720A8091490A0F
:1093F0008823E1F08091470A82FF04C08091160221
:1094000087FD05C08091460A882309F4D3C4809162
:10941000470A9091480A93FF04C08091160287FD85
:109420000BC08091450A811107C005C080910B01D6
:109430008870809309014198415041F080918400E7
:109440009091850082179307C8F34CCE809121023A
:1094500090912202A0912302B0912402892B8A2BA1
:109460008B2B09F08AC08091800A882309F452C0AE
:109470008090920A9090930AA090940AB090950AD6
:10948000C0907B0AD0907C0AE0907D0AF0907E0A22
:1094900080917F0AC814D904EA04FB0488F420915F
:1094A0004C0A30914D0A4091500A5091510A42178E
:1094B000530730F4815080937F0A2150310915C041
:1094C0008C149D04AE04BF04E8F420914C0A309142
:1094D0004D0A40914E0A50914F0A2417350790F4D7
:1094E0008F5F80937F0A2F5F3F4F30934D0A209309
:1094F0004C0A40911D0250911E0260911F02709112
:1095000020020BC040921D0250921E0260921F0268
:10951000709220024FEF5FEFBA0180917F0A87FDC2
:1095200002C0169801C0169A2091840030918500DF
:10953000245E3F4F80917F0A8823B9F0149A80916E
:109540007F0A87FF02C08F5F01C0815080937F0A2E
:10955000149880917F0A882369F380918400909108
:10956000850082179307C8F3E5CF409321025093FB
:10957000220260932302709324028091960A9091B4
:10958000970AA091980AB091990A892B8A2B8B2B64
:1095900009F08FC3A091A514B091A614109709F4F7
:1095A000AEC5C090920AD090930AE090940AF090D1
:1095B000950A40918E0A50918F0A6091900A70919D
:1095C000910AC416D506E606F706D0F010924B0AAB
:1095D0001092A6141092A51490919A0E80919B0E51
:1095E000981709F48CC580919B0E8F5F8F708093C4
:1095F0009B0E00ED802E07E0902EA12CB12C8AC18D
:1096000040918A0A50918B0A60918C0A70918D0A60
:109610004C155D056E057F0508F46DC04091860A06
:109620005091870A6091880A7091890AD2960D91AB
:109630001D912D913C91D597EE27419FF12D529F81
:10964000C001629F900D619F800D911D429FF00DA2
:10965000811D9E1F519FF00D811D9E1F609FF00D6B
:10966000811D9E1F509FF10D8E1F9E1FF6958E1F10
:109670009E1F349F800D911D359F900D1124FD017B
:10968000EA5BFF4F0081118122813381080F191F8E
:10969000211D311D0093820A1093830A2093840AAE
:1096A0003093850A3497C080D180E280F380C01661
:1096B000D106E206F30640F4C092820AD092830AF1
:1096C000E092840AF092850AC090820AD090830AC0
:1096D000E090840AF090850A85E898E121E0FC0199
:1096E00085909590A590B4908C149D04AE04BF0411
:1096F00008F466C370C320917B0A30917C0A4091C4
:109700007D0A50917E0A29833A834B835C832C1512
:109710003D054E055F0508F070C04091770A5091F5
:10972000780A6091790A70917A0A4A875B876C8718
:109730007D87D2960D911D912D913C91D597EE2765
:10974000419FF12D529FC001629F900D619F800D3E
:10975000911D429FF00D811D9E1F519FF00D811D97
:109760009E1F609FF00D811D9E1F509FF10D8E1F4B
:109770009E1FF6958E1F9E1F349F800D911D359F55
:10978000900D11248C0120E030E08090820A9090AE
:10979000830AA090840AB090850AFD01E65BFF4F22
:1097A000081519052A053B05A0F440815181628105
:1097B00073814D835E836F837887801A910AA20A32
:1097C000B30A84169506A606B70638F44A015B016B
:1097D00004C080809180A280B38085E898E151E048
:1097E0005D83FC01059115912591349108151905AA
:1097F0002A053B0508F473C380C380917F0A882340
:10980000D9F0D8964D915C91D99760E070E00091C5
:109810001D0210911E0220911F023091200240175C
:1098200051076207730741F0109221021092220241
:1098300010922302109224024091190250911A02B0
:1098400060911B0270911C0277FF5CC0AE5BBF4F42
:109850008D919D910D90BC91A02D25E838E141E0BE
:10986000F901C590D590E590F490C816D906EA069E
:10987000FB0658F4B695A79597958795440F2C5FEE
:109880003F4F78E1213A370759F74093810A8032F8
:109890009105A105B10520F480E290E0A0E0B0E0E0
:1098A0008097A109B109811538E09307A105B10599
:1098B00008F4DFC344E0949F900111242B573B4EE2
:1098C000F901329645915491EE27859FB001849F0E
:1098D000610D7E1F06946E1F7E1F1124CB01A0E038
:1098E000B0E0F9014591549160E070E0481B590BDC
:1098F0006A0B7B0B4093190250931A0260931B0270
:1099000070931C028090190290901A02A0901B0282
:10991000B0901C028091A5149091A614892B09F097
:10992000C0C1ACDA9093A6148093A514892B09F4D6
:10993000B8C1E091A514F091A614808183FF3EC0C8
:1099400085899689A789B08D8093E7159093E8154E
:10995000A093E915B093EA15818D928DA38DB48DF6
:109960008093EB159093EC15A093ED15B093EE1545
:10997000858D968DA78DB0A18093EF159093F015EE
:10998000A093F115B093F21581A192A1A3A1B4A166
:109990008093F3159093F415A093F515B093F615F5
:1099A00090919A0E80919B0E981709F4BACF8091EE
:1099B0009B0E8F5F8F7080939B0EB3CFC588D68828
:1099C000E788F08C81E0C114D104E104F10409F4CA
:1099D00080E0018D128D238D348D01151105210537
:1099E000310509F08260458D568D678D70A1411556
:1099F00051056105710509F0846080934B0A10924E
:109A0000770A1092780A1092790A10927A0A1092C4
:109A1000860A1092870A1092880A1092890A85A1F4
:109A200096A1A7A1B0A580938E0A90938F0AA093C8
:109A3000900AB093910A882499245401881A990AAB
:109A4000AA0ABB0A8092730A9092740AA092750ABD
:109A5000B092760A80926F0A9092700AA092710A70
:109A6000B092720A80926B0A90926C0AA0926D0A70
:109A7000B0926E0A8092670A9092680AA092690A70
:109A8000B0926A0ACC0CDD1CEE1CFF1CC092570A77
:109A9000D092580AE092590AF0925A0A000F111F08
:109AA000221F331F00935B0A10935C0A20935D0A08
:109AB00030935E0A440F551F661F771F40935F0A5D
:109AC0005093600A6093610A7093620A41A152A1A7
:109AD00063A174A1440F551F661F771F4093630A4B
:109AE0005093640A6093650A7093660A880F991F01
:109AF000AA1FBB1F8093530A9093540AA093550A40
:109B0000B093560A1092920A1092930A1092940AF5
:109B10001092950A82A593A5A4A5B5A580938A0A5B
:109B200090938B0AA0938C0AB0938D0A86A597A573
:109B3000A0A9B1A980937B0A90937C0AA0937D0A87
:109B4000B0937E0A81A58093520A97A99093800AC8
:109B5000992309F124AD35AD3093510A2093500A71
:109B600022AD33AD30934F0A20934E0A109221025A
:109B700010922202109223021092240240AD51ADA5
:109B800060E070E040931D0250931E0260931F023C
:109B90007093200208C040921D0250921E026092F3
:109BA0001F027092200296A920914A0A92130AC0BD
:109BB0002091180230E0482F082E000C550B421758
:109BC000530729F090934A0A80931802CBD98091C9
:109BD000A90A81110E94E3B54092190250921A021B
:109BE00060921B0270921C02E091A514F091A614E1
:109BF000EA5BFF4F80819181A281B3818093820AC9
:109C00009093830AA093840AB093850A25E838E1EB
:109C100041E0F901C590D590E590F490C816D906B9
:109C2000EA06FB0660F4B695A79597958795440FCD
:109C30002C5F3F4FE1EAF8E1E217F30751F7409359
:109C4000810A80329105A105B10520F480E290E0FF
:109C5000A0E0B0E08097A109B109811558E095070F
:109C6000A105B10508F428C264E0969F9001112473
:109C70002B573B4EF901329645915491EE27859F23
:109C8000B001849F610D7E1F06946E1F7E1F1124FC
:109C9000F90185909490A12CB12C861A970AA108FD
:109CA000B1088092960A9092970AA092980AB09270
:109CB000990A0091960A1091970A2091980A30917A
:109CC000990A4091210250912202609123027091E1
:109CD0002402F02E1983F22FE32F40175107620759
:109CE000730720F4F42E5983F62FE72F8F2D9981D7
:109CF000AF2FBE2F0097E1E0AE07B10520F08FEF48
:109D00009FEFA0E0B0E0081B190B2A0B3B0B009360
:109D1000960A1093970A2093980A3093990A4F3F16
:109D2000FFEF5F076F077F0761F0481B590B6A0B56
:109D30007B0B409321025093220260932302709385
:109D40002402F8942091840030918500205F3F4FD9
:109D5000498541504987442339F0280E391E22167F
:109D6000330608F455C901C01901309289002092C8
:109D7000880078942D960FB6F894DEBF0FBECDBF45
:109D8000DF91CF911F910F91FF90EF90DF90CF90D7
:109D9000BF90AF909F908F907F906F905F904F900B
:109DA0003F902F90089590910B019095987090930B
:109DB00009013BCA80910B0188708093090127CB70
:109DC000F694E794D794C794220F0496E8E1813A79
:109DD0009E0709F084CC2093810AF0E2CF16D104CB
:109DE000E104F10428F410E2C12ED12CE12CF12C75
:109DF00030E2C31AD108E108F108C11488E0D8069E
:109E0000E104F104F8F0E4E0DE9EC00111248B5778
:109E10009B4EFC01329625913491FC2DEE27F39F49
:109E20008001F29F010D1E1F06940E1F1E1F11249C
:109E3000FC0185909490A12CB12C801A910AA10864
:109E4000B10822C097018601369527951795079589
:109E5000F801EC7F9F012B573F4EF90185909490BC
:109E6000F901329685919491EC2DE770E89F90016D
:109E7000E99F300D1124F3E036952795FA95E1F727
:109E8000821A930AA12CB12C480D591D6A1D7B1D05
:109E90004093860A5093870A6093880A7093890AD0
:109EA0009091800A80917F0A992309F474C08823D5
:109EB00009F430CDD8968D919C91D997A0E0B0E06F
:109EC00040911D0250911E0260911F02709120026C
:109ED00084179507A607B70709F060C01BCDB69495
:109EE000A794979487944D81440F4D83049661EA1B
:109EF00078E16817790709F074CC2D812093810AE5
:109F000030E283169104A104B10428F450E2852EB6
:109F1000912CA12CB12C60E2861A9108A108B108FD
:109F2000811478E09706A104B10408F440C0E4E08D
:109F30009E9EC00111248B579B4EFC0132962591A9
:109F40003491F82DEE27F39F8001F29F010D1E1F23
:109F500006940E1F1E1F1124FC0185909490A12CC5
:109F6000B12C801A910AA108B1084A855B856C85DD
:109F70007D85480D591D6A1D7B1D4093770A5093BE
:109F8000780A6093790A70937A0A8091800A811125
:109F900032C080917F0A882309F4BCCC1092210240
:109FA000109222021092230210922402B3CC950147
:109FB00084013695279517950795F801EC7F9F0149
:109FC0002B573F4EF90185919491F90132960591F5
:109FD0001491E82DE770E09F9001E19F300D11246E
:109FE00043E0369527954A95E1F74C01821A930A8A
:109FF000A12CB12CBACF49815A816B817C812D81F2
:10A00000420F511D611D711D4C155D056E057F05CB
:10A01000C8F480917F0A882309F47CCCD8964D91AE
:10A020005C91D99760E070E000911D0210911E02D2
:10A0300020911F02309120024017510762077307D9
:10A0400009F468CC1092210210922202109223028D
:10A0500010922402D8968D919C91D997A0E0B0E0FF
:10A0600080931D0290931E02A0931F02B0932002C2
:10A0700051CCAC01BD017695679557954795FA018E
:10A08000EC7F9F012B573F4EF90145915491F90107
:10A090003296659174918770869F9001879F300DED
:10A0A0001124C901F3E096958795FA95E1F7481BCD
:10A0B000590B60E070E01ECCAC01BD017695679550
:10A0C00057954795FA01EC7F9F012B573F4EF901B9
:10A0D00085909490F9013296459154918770849FB0
:10A0E0009001859F300D1124C901A3E096958795B5
:10A0F000AA95E1F7881A990AA12CB12CD2CD80ED4E
:10A10000882E87E0982EA12CB12C0BCCCF92DF9219
:10A11000EF92FF92CF93DF936A017B01FC01849160
:10A12000EF012196882321F00E9488C5FE01F7CF18
:10A130004AE0C701B601DF91CF91FF90EF90DF9029
:10A14000CF900C948FC5CF92DF92EF92FF92CF9376
:10A15000DF936A017B01FC018491EF012196882342
:10A1600021F00E9488C5FE01F7CF42E0C701B60189
:10A17000DF91CF91FF90EF90DF90CF900C9414C6B9
:10A180000F931F93CF93DF938B01FC018491EF0119
:10A190002196882321F00E9488C5FE01F7CFB801DF
:10A1A000110F880B990BDF91CF911F910F910C9498
:10A1B000FAC50F931F93CF93DF938B01FC0184911A
:10A1C000EF012196882321F00E9488C5FE01F7CF78
:10A1D000E8018991882319F00E9488C5FACFDF91A0
:10A1E000CF911F910F9108950F931F93CF93DF93FA
:10A1F00000D01F92CDB7DEB78C0108960E946CB4D8
:10A2000069837A838B839C83B8016C5F7F4FAE0137
:10A210004F5F5F4FC8010E940BB39B01AC01F80177
:10A2200060857185828593850E94DFDDF8016087F6
:10A230007187828793870F900F900F900F90DF9117
:10A24000CF911F910F91089586E40E94DB3A80938D
:10A25000D514882351F00E94A43A609310027093A1
:10A260001102809312029093130283E50E94DB3A5D
:10A27000882351F00E94A43A60930C0270930D025F
:10A2800080930E0290930F0282E40E94DB3A8823AF
:10A2900051F00E94A43A60930802709309028093DF
:10A2A0000A0290930B020895CF92DF92EF92FF92F1
:10A2B0000F931F93CF93DF936C017A018B01C0E062
:10A2C000D0E0CE15DF0581F0D8016D918D01D6016A
:10A2D000ED91FC910190F081E02DC6011995892B3B
:10A2E00011F02196EECF7E01C701DF91CF911F9132
:10A2F0000F91FF90EF90DF90CF9008950E94F0E0D3
:10A300003FB7F8948091410C9091420CA091430C7E
:10A31000B091440C26B5A89B05C02F3F19F00196BB
:10A32000A11DB11D3FBFBA2FA92F982F8827820FDB
:10A33000911DA11DB11DBC01CD0142E0660F771F2B
:10A34000881F991F4A95D1F708952FB7F894609107
:10A350003D0C70913E0C80913F0C9091400C2FBFB2
:10A3600008951F920F920FB60F9211242F933F93CF
:10A370008F939F93AF93BF9380913D0C90913E0C30
:10A38000A0913F0CB091400C30913C0C23E0230F86
:10A390002D3720F40196A11DB11D05C026E8230F1D
:10A3A0000296A11DB11D20933C0C80933D0C90930F
:10A3B0003E0CA0933F0CB093400C8091410C9091C7
:10A3C000420CA091430CB091440C0196A11DB11D0B
:10A3D0008093410C9093420CA093430CB093440C97
:10A3E000BF91AF919F918F913F912F910F900FBE91
:10A3F0000F901F9018951F920F920FB60F92112475
:10A400000BB60F922F933F934F935F936F937F936E
:10A410008F939F93AF93BF93EF93FF9380919D0A88
:10A4200090919E0AA0919F0AB091A00A892B8A2B35
:10A430008B2B59F190919C0AE0919A0AF0919B0A1A
:10A4400080818927808380919D0A90919E0AA091A6
:10A450009F0AB091A00A181619061A061B060CF0DE
:10A4600056C080919D0A90919E0AA0919F0AB0913A
:10A47000A00A0197A109B10980939D0A90939E0AB1
:10A48000A0939F0AB093A00A42C080912502E5EAFA
:10A49000F8E1E4919FEF90932502E230C9F050F487
:10A4A000EE2399F0E13081F590916F009D7F9093BC
:10A4B0006F002AC0E43019F1E0F0E53029F5909101
:10A4C00073009D7F909373001FC010926E001CC09C
:10A4D000909170009D7F9093700091E09093B000F8
:10A4E0009091B100987F94609093B1001092B30066
:10A4F0000BC0909171009D7F9093710005C0909169
:10A5000072009D7F9093720060E00E9403A9FF910A
:10A51000EF91BF91AF919F918F917F916F915F91DB
:10A520004F913F912F910F900BBE0F900FBE0F9048
:10A530001F90189590934B0480934A0480E00C94EC
:10A54000FC752F923F924F925F926F927F928F9203
:10A550009F92AF92BF92CF92DF92EF92FF920F93B2
:10A560001F93CF93DF93CDB7DEB7C857D1090FB68E
:10A57000F894DEBF0FBECDBFE091D714F091D81490
:10A58000EF2B11F00C946A5B2896DFAECEAE2897C5
:10A590006E2C79016A015B01FC01208131814281CD
:10A5A00053816C962CAF3DAF4EAF5FAF6C9720914F
:10A5B000F7153091F8154091F9155091FA156C96F0
:10A5C0006CAD7DAD8EAD9FAD6C970E94F9D90E94A8
:10A5D00011E0E0966CAF7DAF8EAF9FAFE097D501F5
:10A5E0008D919D910D90BC91A02DA0968CAF9DAFAB
:10A5F000AEAFBFAFA0972091FB153091FC154091F5
:10A60000FD155091FE15BC01CD010E94F9D90E94A3
:10A6100011E0E4966CAF7DAF8EAF9FAFE497D601AB
:10A620002D913D914D915C91A4962CAF3DAF4EAFD5
:10A630005FAFA4972091FF1530910016409101164D
:10A6400050910216A4966CAD7DAD8EAD9FADA497D2
:10A650000E94F9D90E9411E0E8966CAF7DAF8EAFF1
:10A660009FAFE897D7012D913D914D915C91229636
:10A670002CAF3DAF4EAF5FAF2297209103163091C4
:10A680000416409105165091061622966CAD7DADCC
:10A690008EAD9FAD22970E94F9D90E9411E060967D
:10A6A0006CAF7DAF8EAF9FAF60978091820C83FFC0
:10A6B0001CC060962CAD3DAD4EAD5FAD6097209354
:10A6C000CC0E3093CD0E4093CE0E5093CF0E2296EB
:10A6D0008CAD9DADAEADBFAD22978093BC0E909377
:10A6E000BD0EA093BE0EB093BF0ED801BC91BDA30A
:10A6F000F801F181F9ABD8011296BC91BEABF8011B
:10A70000F381FAAF80919A0E90919B0E891B8F7006
:10A710008F3019F40E94099CF5CF00919A0EE996AA
:10A720000FAFE99780919A0E082F10E01CA30BA39E
:10A730008091C00E9091C10EA091C20EB091C30E37
:10A74000E0968CAC9DACAEACBFACE097881A990A91
:10A75000AA0ABB0A8091C40E9091C50EA091C60EA4
:10A76000B091C70EE4962CAC3DAC4EAC5FACE49718
:10A77000281A390A4A0A5B0A8091C80E9091C90EBC
:10A78000A091CA0EB091CB0EE8962CAD3DAD4EAD6A
:10A790005FADE897281B390B4A0B5B0B2DA73EA733
:10A7A0004FA758AB8091CC0E9091CD0EA091CE0EBC
:10A7B000B091CF0E60960CAD1DAD2EAD3FAD609744
:10A7C000081B190B2A0B3B0B09A71AA72BA73CA7A1
:10A7D000012B022B032B09F4BCC08091810C811149
:10A7E0004BC060914C0470914D0480914E04909147
:10A7F0004F040E9424DF209131023091320262170F
:10A8000073070CF039C060962CAD3DAD4EAD5FAD19
:10A8100060972093CC0E3093CD0E4093CE0E509384
:10A82000CF0E22968CAD9DADAEADBFAD229780937D
:10A83000BC0E9093BD0EA093BE0EB093BF0EEBE97D
:10A84000FBE184918F010F5F1F4F811103C0E9E18C
:10A85000FAE104C00E9488C5F801F3CF84918F010A
:10A860000F5F1F4F882321F00E9488C5F801F6CFA3
:10A8700019A61AA61BA61CA694E0699E80011124A5
:10A88000035D1D4F69A57AA58BA59CA50E949AD949
:10A89000D8012D913D914D915C910E94F9D96B01A8
:10A8A0007C0120E030E0A9010E9406E087FF04C09F
:10A8B000F7FAF094F7F8F09460910316709104168B
:10A8C00080910516909106160E9424DF9B01AC0131
:10A8D000A8ECB0E00E94C0DD0E949AD9A7019601C1
:10A8E0000E9494D987FF39C060960CAD1DAD2EAD86
:10A8F0003FAD60970093CC0E1093CD0E2093CE0EFB
:10A900003093CF0E22962CAD3DAD4EAD5FAD22976C
:10A910002093BC0E3093BD0E4093BE0E5093BF0EDD
:10A92000EBE9FBE184918F010F5F1F4F811103C0A1
:10A93000EAEFF9E104C00E9488C5F801F3CF8491E1
:10A940008F010F5F1F4F882321F00E9488C5F801F7
:10A95000F6CF19A61AA61BA61CA6D501C4018827E6
:10A96000B7FD83959927AA27BB27782E57FE03C0EA
:10A97000382F3260732E8DA59EA5AFA5B8A9B7FF5D
:10A9800003C0972D9460792E09A51AA52BA53CA587
:10A9900037FF03C0172D1860712E24E0629E8001DE
:10A9A0001124035D1D4F69A57AA58BA59CA50E9466
:10A9B0009AD9D8012D913D914D915C910E94F9D980
:10A9C0006B017C0120E030E0A9010E9406E087FFD6
:10A9D00004C0C701B601905802C0C701B60120E00B
:10A9E00030E040E05FE30E94E0DD0E9429DF6AABD7
:10A9F0007BAB8CAB9DAB88E50BA11CA1809FF001CC
:10AA0000819FF00D1124EB53FB4F108276AAB50104
:10AA1000A401B7FE07C044275527BA0148195909B0
:10AA20006A097B0988E50BA11CA1809FF001819F29
:10AA3000F00D1124EB53FB4F458B568B678B708FBA
:10AA40002C962CAE3DAE4EAE5FAE2C9757FE0DC091
:10AA500088279927DC0182199309A409B5092C9646
:10AA60008CAF9DAFAEAFBFAF2C9728E50BA11CA15B
:10AA7000209FF001219FF00D1124EB53FB4F2C96EA
:10AA80008CAD9DADAEADBFAD2C97818F928FA38F56
:10AA9000B48F0DA51EA52FA538A937FF07C0309587
:10AAA0002095109501951F4F2F4F3F4FE8E57E2EC3
:10AAB000ABA1BCA17A9EF0017B9EF00D1124EB535B
:10AAC000FB4F058F168F278F30A38AA99BA9ACA9AE
:10AAD000BDA981A392A3A3A3B4A323964FAF2397A9
:10AAE000752EF62FE72F2C968CAD9DADAEADBFAD7C
:10AAF0002C97481759076A077B0778F429969FAD6A
:10AB0000299723969FAF23972A967FAC2A972B9657
:10AB1000FFAD2B972C96EFAD2C9723968FAD2397F7
:10AB2000972DAF2FBE2F80179107A207B30710F400
:10AB3000D901C8010AA91BA92CA93DA98017910711
:10AB4000A207B30710F4D901C80128E50BA11CA185
:10AB5000209FF001219FF00D1124EB53FB4F85A3A3
:10AB600096A3A7A3B0A70697A105B10508F4ABC5A6
:10AB7000DF01AE5ABF4F80914204909143048D9300
:10AB80009C9361A6452B462B472B09F05F9888E5DF
:10AB90000BA11CA1809FF001819FF00D1124EB53AC
:10ABA000FB4F818D928DA38DB48D892B8A2B8B2B9E
:10ABB00011F08A98479888E50BA11CA1809FF001AD
:10ABC000819FF00D1124EB53FB4F858D968DA78D42
:10ABD000B0A1892B8A2B8B2B31F0809108018170D9
:10ABE0008093060147982AA93BA94CA95DA9232B6C
:10ABF000242B252B09F470C58091870C882319F02C
:10AC000081508093870C611004C0129880E2809379
:10AC1000870C60907D0C70907E0C00917F0C1091E1
:10AC2000800C9301A8016DA179A98EA99AAD0E940B
:10AC300094D987FF04C06DA279AA0EAB1AAFC501E3
:10AC4000B4010E949AD92091A0173091A117409188
:10AC5000A2175091A3170E94F9D926966CAF7DAF29
:10AC60008EAF9FAF2697698B7A8B8B8B9C8BC201A3
:10AC7000B1010E949AD92091A4173091A517409153
:10AC8000A6175091A7170E94F9D92B013C016D8B93
:10AC90007E8B8F8B988F6DA57EA58FA598A90E941E
:10ACA0009AD92091A8173091A9174091AA175091CD
:10ACB000AB170E94F9D94B015C01698F7A8F8B8F9A
:10ACC0009C8F2091AC173091AD174091AE175091E9
:10ACD000AF17C701B6010E94F9D96B017C016D8FD6
:10ACE0007E8F8F8F98A388E50BA11CA1809FF00118
:10ACF000819FF00D1124EB53FB4F2589368947893D
:10AD0000508D2DA73EA74FA758AB263031054105E2
:10AD1000510508F4EAC42896AEADBFAD2897CD9092
:10AD2000DD90ED90FC9020E030E0A901C701B60174
:10AD30000E9494D98111F8C426962CAD3DAD4EAD3C
:10AD40005FAD2697CA01B9010E94F9D96B017C0158
:10AD5000A3019201C301B2010E94F9D99B01AC0188
:10AD6000C701B6010E94E0DD6B017C01A5019401E1
:10AD7000C501B4010E94F9D99B01AC01C701B6011C
:10AD80000E94E0DD0E944BE028E50BA11CA1209F62
:10AD9000F001219FF00D1124EB53FB4F658776875F
:10ADA0008787908B88E50BA11CA1809FF001819F74
:10ADB000F00D1124EB53FB4F458456846784708853
:10ADC000A301920160E070E080E89FE30E94BCDE96
:10ADD00064966CAF7DAF8EAF9FAF64972DA139A9FC
:10ADE0004EA95AAD0E94F9D94B015C0180919A0E8F
:10ADF0009091980E891B8F7027968FAF2797A5018A
:10AE0000940160E074E284E799E40E94BCDE0E9451
:10AE100011E06B017C0127968FAD27978250863019
:10AE200008F491C4A5019401C301B2010E94F9D9AB
:10AE30009B01AC010E94F9D968966CAF7DAF8EAFD3
:10AE40009FAF689788E5ABA1BCA18A9F80018B9FCB
:10AE5000100D11240B531B4F68962CAD3DAD4EAD1C
:10AE60005FAD6897D80111962D933D934D935C93F8
:10AE7000149795962D913D914D915C9198972EAB9D
:10AE80003FAB48AF59AFCA01B9010E9498D96AAF28
:10AE90007BAF8CAF9DAF9B01AC01C501B4010E949B
:10AEA000F9D90E94A6DE0E9429DFA8966CAF7DAF7B
:10AEB0008EAF9FAFA897F801EE5BFF4F6083718361
:10AEC000828393838E010F5E1F4F2A961FAF0EAFB2
:10AED0002A970051110924961FAF0EAF249705E65B
:10AEE0001CE0AC961FAF0EAFAC978E010F5D1F4FED
:10AEF0001AA309A324960EAD1FAD2497AA961FAFDF
:10AF00000EAFAA97312C212C10E81DA30FE309AB3B
:10AF10002A96AEADBFAD2A972D913D914D915D9191
:10AF20002A96BFAFAEAF2A97C501B4010E94F9D9E6
:10AF30006B017C01AA96EEADFFADAA976193719368
:10AF400081939193AA96FFAFEEAFAA9720E030E0ED
:10AF5000A9010E9406E087FF04C0F7FAF094F7F811
:10AF6000F094AC96AEADBFADAC974D905D906D904A
:10AF70007D90AC96BFAFAEAFAC97A7019601C30171
:10AF8000B2010E9494D987FD18C409A11AA12A967A
:10AF90002EAD3FAD2A970217130709F0B9CF20E075
:10AFA00030E040E85FE3632D722D8DA199A90E94E6
:10AFB00094D987FF58C07E0131E1E30EF11C24963D
:10AFC0000EAD1FAD2497232D322D4DA159A9D801C7
:10AFD0006D917D918D919C910E94F9D9F8016193B9
:10AFE0007193819391938F01EE16FF0661F728E527
:10AFF0000BA11CA1209FC001219F900D11249C0139
:10B000002B533B4F790189010E5B1F4FA8966CAD06
:10B010007DAD8EAD9FADA8970E9498D9232D322D7E
:10B020004DA159A90E94F9D90E9429DFD8016D9339
:10B030007D938D939C931397232D322D4DA159A968
:10B04000632D722D8DA199A90E94F9D968962CAD16
:10B050003DAD4EAD5FAD68970E94F9D9F7016183B0
:10B060007283838394832AAD3BAD4CAD5DAD649612
:10B070006CAD7DAD8EAD9FAD64970E94F9D96DA387
:10B080007EA38FA398A70DA51EA52FA538A9012BD8
:10B09000022B032B09F0A9C388E52BA13CA1829FB9
:10B0A0008001839F100D11240B531B4FF801818DDC
:10B0B000928DA38DB48D892B8A2B8B2B09F095C390
:10B0C000858D968DA78DB0A1892B8A2B8B2B09F0AE
:10B0D0008CC32091610C3091620C4091630C5091B3
:10B0E000640C6DA17EA18FA198A50E94F9D90E9440
:10B0F000A6DE0E9429DF2B013C01D801D7961C92C5
:10B1000088E52BA13CA1829F8001839F100D112413
:10B110000B531B4FF801E25BFF4F4082518262826A
:10B120007382C301B2010E9498D96B017C012DA1E9
:10B130003EA14FA158A50E94BCDE6AAF7BAF8CAF89
:10B140009DAFD80151966D937D938D939C935497A9
:10B150002DEB37E346E051E4C701B6010E94F9D96F
:10B160000E9429DFF80162AB73AB84AB95AB87A972
:10B17000882371F1FE962091550C3091560C409128
:10B18000570C5091580C60817181828193810E948B
:10B19000F9D92AAD3BAD4CAD5DAD0E94F9D92091F6
:10B1A00003163091041640910516509106160E9420
:10B1B000F9D99B01AC0160E074E284EF99E40E944C
:10B1C000BCDE0E9429DFD801D9967C936E93D89774
:10B1D00088E50BA11CA1809FF001819FF00D112437
:10B1E000EB53FB4F21813281438154812C962CAF4C
:10B1F0003DAF4EAF5FAF2C97CA01B9010E944BE043
:10B20000362E272E8C0145E45CE062965FAF4EAF90
:10B2100062973E0151E1650E711C85E49CE09FAB95
:10B220008EAB24964EAC5FAC249739A62DA60DA309
:10B2300019AB1AAAD201CD90DD90ED90FD902D01B1
:10B2400020E030E0A901C701B6010E9406E087FFB7
:10B2500004C0F7FAF094F7F8F094EEA9FFA98190F2
:10B260009190A190B190FFABEEABA7019601C50103
:10B27000B4010E9494D987FDD4C564147504D1F635
:10B2800027965FAD2797552309F444C6C0909C0EBE
:10B29000D0909D0EE0909E0EF0909F0E2DEB37E328
:10B2A00046E855E3C701B6010E9494D987FD32C62E
:10B2B000C701B6010E944BE06B017C019B01AC0110
:10B2C000632D722DC8010E9494D987FD03C03C2CC8
:10B2D0002D2C87019601A701632D722DC8010E94B4
:10B2E000BCDE68966CAF7DAF8EAF9FAF689780EA8B
:10B2F0009EE028969FAF8EAF289720E030E040E890
:10B300005FE32AAB3BAB4CAB5DAB1EAA2896AEAD60
:10B31000BFAD28972D913D914D915D912896BFAF7E
:10B32000AEAF289768966CAD7DAD8EAD9FAD68973A
:10B330000E94F9D94B015C012496EEADFFAD249734
:10B34000C190D190E190F1902496FFAFEEAF249799
:10B35000FEA9FF2391F02AA93BA94CA95DA90E944F
:10B36000F9D94B015C012AA93BA94CA95DA9C701E8
:10B37000B6010E94F9D96B017C01A7019601C501B4
:10B38000B4010E9406E020E030E0A90118160CF09C
:10B390008EC5C701B6010E9406E018160CF482C5DE
:10B3A00020E030E0A901C501B4010E9494D987FDD5
:10B3B00079C52601370177FA709477F87094A30164
:10B3C0009201C501B4010E9406E0181614F424018C
:10B3D00035016296AEADBFAD6297CD90DD90ED9038
:10B3E000FD906296BFAFAEAF6297A3019201C70115
:10B3F000B6010E9494D987FF15C0A3019201C7012D
:10B40000B6010E94BCDE9B01AC016AA97BA98CA994
:10B410009DA90E94F9D96AAB7BAB8CAB9DABBEA951
:10B42000BF5FBEABE0EBFEE028962EAD3FAD2897A8
:10B43000E217F30709F06ACF3EA9332361F02AA986
:10B440003BA94CA95DA9632D722DC8010E94F9D9B1
:10B45000362E272E8C0124EA30E74DE75FE3632D7B
:10B46000722DC8010E94F9D96B017C012091830CD7
:10B470003091840C4091850C5091860C0E9494D997
:10B4800087FD3EC589A59DA5ADA1B9A98093830C73
:10B490009093840CA093850CB093860C28E54BA167
:10B4A0005CA1249FC001259F900D1124DC01AB53AA
:10B4B000BB4F7D01232D322DA801632D722DC801B4
:10B4C0000E94F9D9F70161877287838794876AADF3
:10B4D0007BAD8CAD9DAD90589B01AC010E94E0DD31
:10B4E000D7011D962D913D914D915C9150970E94F1
:10B4F000F9D99B01AC016BE077ED83E29BE30E94FD
:10B50000DFDD9B01AC018BE097EDA3E2BBE3F7012C
:10B5100085839683A783B08710812C966CAD7DAD13
:10B520008EAD9FAD2C970E9494D918160CF4F7C4D9
:10B5300083E0182B88E52BA13CA1829FF001839F1B
:10B54000F00D1124EB53FB4F108380E1FE01319687
:10B55000A0EABEE001900D928A95E1F72C968CADA1
:10B560009DADAEADBFAD2C9780939C0E90939D0E7C
:10B57000A0939E0EB0939F0EE0960CAD1DAD2EAD28
:10B580003FADE0970093C00E1093C10E2093C20E02
:10B590003093C30EE4962CAD3DAD4EAD5FADE49758
:10B5A0002093C40E3093C50E4093C60E5093C70E21
:10B5B000E8968CAD9DADAEADBFADE8978093C80E5B
:10B5C0009093C90EA093CA0EB093CB0E60960CADAB
:10B5D0001DAD2EAD3FAD60970093CC0E1093CD0EF8
:10B5E0002093CE0E3093CF0E6C962CAD3DAD4EAD6C
:10B5F0005FAD6C972093B00E3093B10E4093B20EB6
:10B600005093B30EA0968CAD9DADAEADBFADA097DF
:10B610008093B40E9093B50EA093B60EB093B70E70
:10B62000A4960CAD1DAD2EAD3FADA4970093B80E02
:10B630001093B90E2093BA0E3093BB0E22962CAD08
:10B640003DAD4EAD5FAD22972093BC0E3093BD0E45
:10B650004093BE0E5093BF0E90919A0E80919B0E18
:10B66000981303C084E68093970EE9968FADE9970F
:10B670008F5F8F7080939A0E80919A0E9091990EA1
:10B6800081508F7089134DC410919B0E1BA30091A4
:10B690009A0E09A728E51BA109A51013CDC4812C7A
:10B6A000912CA12CB12C1DA61DA219AA1EAE212CD5
:10B6B000312C00E010E029A53BA12313CAC42114BA
:10B6C000310409F079C580916F00826080936F002A
:10B6D00081E0E2C680E0E0C66090790C70907A0C60
:10B6E00000917B0C10917C0C9CCA818D928DA38D56
:10B6F000B48D0697A105B10508F00DCB858D968D0B
:10B70000A78DB0A10697A105B10508F004CB20E0F4
:10B7100030E0A901C701B6010E9406E087FF04C01E
:10B72000F7FAF094F7F8F09488E50BA11CA1809F3C
:10B73000F001819FF00D1124EB53FB4FC586D68697
:10B74000E786F08A2FCB8091750C9091760CA091B2
:10B75000770CB091780CC816D906EA06FB0608F0FB
:10B7600061CB8C199D09AE09BF09BC01CD01660FE3
:10B77000771F881F991F27964FAD2797042F10E03A
:10B7800020E030E0A90198010E9482DDCA01B901E0
:10B790000E9498D90E9411E06C0D7D1D8E1D9F1D89
:10B7A0000E9498D99B01AC0160E074E284E799E4BF
:10B7B0000E94BCDE4B015C0135CBA7019601C301A1
:10B7C000B2010E94BCDE7B018C019B01AC01632DA8
:10B7D000722D8DA199A90E9406E018160CF0D5CB08
:10B7E0003E2C2F2C0DA319ABD0CB0AA91BA92CA939
:10B7F0003DA9012B022B032B49F020915D0C3091C8
:10B800005E0C40915F0C5091600C08C02091590C67
:10B8100030915A0C40915B0C50915C0C6DA17EA153
:10B820008FA198A50E94F9D90E94A6DE0E9429DF67
:10B830002B013C012AA93BA94CA95DA9232B242B50
:10B84000252BC9F020E030E0A9016091550C7091E2
:10B85000560C8091570C9091580C0E9494D98823D3
:10B8600051F081E009A51AA52BA53CA510161106DB
:10B87000120613060CF080E098E52BA13CA1929FE4
:10B880008001939F100D11240B531B4FD801D796A5
:10B890008C93882309F4B2C02091B00E3091B10E80
:10B8A0004091B20E5091B30E6C966CAD7DAD8EADE5
:10B8B0009FAD6C970E94DFDD69A77AA78BA79CA735
:10B8C0002091B40E3091B50E4091B60E5091B70E46
:10B8D000A0966CAD7DAD8EAD9FADA0970E94DFDDD3
:10B8E0004B015C012091B80E3091B90E4091BA0E17
:10B8F0005091BB0EA4966CAD7DAD8EAD9FADA4975F
:10B900000E94DFDD6B017C0129A53AA54BA55CA552
:10B91000CA01B9010E94F9D969A77AA78BA79CA788
:10B92000A5019401C501B4010E94F9D99B01AC01A4
:10B9300069A57AA58BA59CA50E94E0DD4B015C0161
:10B94000A7019601C701B6010E94F9D99B01AC017C
:10B95000C501B4010E94E0DD0E944BE06B017C0157
:10B960002091BC0E3091BD0E4091BE0E5091BF0E85
:10B9700022966CAD7DAD8EAD9FAD22970E94DFDD2E
:10B98000A70196010E94BCDE6B017C01F801FE96C6
:10B99000608371838283938320E030E040E450E44D
:10B9A0000E9406E018161CF4F80117AA27C020917F
:10B9B000550C3091560C4091570C5091580CC701C2
:10B9C000B6010E94F9D99B01AC016091510C7091B4
:10B9D000520C8091530C9091540C0E94BCDE2DA10E
:10B9E0003EA14FA158A50E94F9D90E9429DF6415F4
:10B9F00075058605970510F42B013C0180917C1795
:10BA000090917D17A0917E17B0917F170EA91FA965
:10BA100028AD39AD80179107A207B30708F4DFC03E
:10BA20002DA53EA54FA558A9232B242B252B41F14D
:10BA30006091801770918117809182179091831780
:10BA40006415750586059705D8F42EA93FA948AD5C
:10BA500059AD0E9473DD6B017C012DA53EA54FA55C
:10BA600058A9C301B2010E9473DDC616D706E806C5
:10BA7000F90630F4C701B6010E9482DD29013A01BE
:10BA800088E50BA11CA1809FF001819FF00D11247E
:10BA9000EB53FB4FC18CD28CE38CF48CC114D104DA
:10BAA000E104F10431F16091841770918517809160
:10BAB0008617909187176415750586059705C8F454
:10BAC0002EA93FA948AD59AD0E9473DD4B015C0121
:10BAD000A7019601C301B2010E9473DD8616970685
:10BAE000A806B90630F4C501B4010E9482DD29011F
:10BAF0003A0188E50BA11CA1809FF001819FF00D08
:10BB00001124EB53FB4FC58CD68CE78CF0A0C114ED
:10BB1000D104E104F10431F1609188177091891723
:10BB200080918A1790918B17641575058605970586
:10BB3000C8F42EA93FA948AD59AD0E9473DD4B0151
:10BB40005C01A7019601C301B2010E9473DD861654
:10BB50009706A806B90630F4C501B4010E9482DD3B
:10BB600029013A0188E50BA11CA1809FF001819F6A
:10BB7000F00D1124EB53FB4FC1A0D2A0E3A0F4A021
:10BB8000C114D104E104F10409F4BACA60918C171C
:10BB900070918D1780918E1790918F176415750590
:10BBA0008605970508F0ACCA2EA93FA948AD59AD46
:10BBB0000E9473DD4B015C01A7019601C301B20134
:10BBC0000E9473DD86169706A806B90608F098CA83
:10BBD000C501B4010E9482DD29013A0191CA2DA557
:10BBE0003EA54FA558A9232B242B252BC9F16091E5
:10BBF0008017709181178091821790918317641537
:10BC000075058605970560F50E9498D92AAD3BAD6C
:10BC10004CAD5DAD0E94F9D96B017C016DA57EA58F
:10BC20008FA598A90E9498D94B015C01C301B2016C
:10BC30000E9498D9A50194010E94F9D99B01AC01F9
:10BC4000C701B6010E9494D987FF0AC0A5019401DB
:10BC5000C701B6010E94BCDE0E9429DF2B013C0116
:10BC600088E50BA11CA1809FF001819FF00D11249C
:10BC7000EB53FB4F818C928CA38CB48C8114910478
:10BC8000A104B104B9F16091841770918517809176
:10BC9000861790918717641575058605970550F5E9
:10BCA0000E9498D92AAD3BAD4CAD5DAD0E94F9D94B
:10BCB0006B017C01C501B4010E9498D94B015C0164
:10BCC000C301B2010E9498D9A50194010E94F9D93B
:10BCD0009B01AC01C701B6010E9494D987FF0AC03D
:10BCE000A5019401C701B6010E94BCDE0E9429DFB4
:10BCF0002B013C0188E50BA11CA1809FF001819FD5
:10BD0000F00D1124EB53FB4F858C968CA78CB0A0C3
:10BD100081149104A104B104B9F160918817709164
:10BD2000891780918A1790918B1764157505860580
:10BD3000970550F50E9498D92AAD3BAD4CAD5DAD4D
:10BD40000E94F9D96B017C01C501B4010E9498D908
:10BD50004B015C01C301B2010E9498D9A501940175
:10BD60000E94F9D99B01AC01C701B6010E9494D988
:10BD700087FF0AC0A5019401C701B6010E94BCDE7D
:10BD80000E9429DF2B013C0188E50BA11CA1809FAB
:10BD9000F001819FF00D1124EB53FB4FC1A0D2A005
:10BDA000E3A0F4A0C114D104E104F10409F4A8C98A
:10BDB00060918C1770918D1780918E1790918F17CD
:10BDC000641575058605970508F09AC90E9498D9EB
:10BDD0002AAD3BAD4CAD5DAD0E94F9D94B015C0184
:10BDE000C701B6010E9498D96B017C01C301B20161
:10BDF0000E9498D9A70196010E94F9D99B01AC0134
:10BE0000C501B4010E9494D987FF7AC9A7019601A0
:10BE1000C501B4010E94BCDE0E9429DF2B013C0158
:10BE20006FC9FAA9FF2331F1A5019401632D722D89
:10BE3000C8010E94F9D94B015C0129A53DA54DA17E
:10BE400059A9C701B6010E94F9D99B01AC01C501EE
:10BE5000B4010E9494D987FF22C0A7019601C501B1
:10BE6000B4010E94BCDE69A77DA78DA399AB21E038
:10BE70002AAB03CAA7019601C501B4010E94BCDE2A
:10BE80009B01AC0169A57DA58DA199A90E94F9D955
:10BE900069A77DA78DA399AB31E03AABEEC941E02C
:10BEA0004AABEBC9A7019601C501B40113C0C70194
:10BEB000B6010E9494D987FD09C020E030E0A901B5
:10BEC000C501B4010E9406E018164CF4A5019401C6
:10BED000C701B6010E94DFDD2B013C017ACA2401B3
:10BEE000350177FA709477F87094A3019201C70135
:10BEF000B6010E9494D987FD6CCA2601370169CA30
:10BF000029A53DA54DA159A9C701B6010E9494D903
:10BF100087FFB8CA39A42DA40DA119A9B3CA81E01D
:10BF200008CBF0909A0E8FEF8F0D8F708BA3B0908F
:10BF3000990E80919A0EB81609F454C0C12CD12CD8
:10BF40000BA10B1509F44EC0602E712C28E5269D1F
:10BF50008001279D100D11240B531B4FD8018C918C
:10BF600083FD2BC00EAF1AAB0115110541F11996D7
:10BF7000BC91B9A7F801F285FDA7D8011B96BC9129
:10BF8000BDA3F801F485F9ABD80115962D903D902D
:10BF90004D905C901897A201910169A57DA58DA196
:10BFA0009F2F0E9494D9811180C1C114D10439F00E
:10BFB000F601808180FD79C102C0CEAEDAAA8BA1E4
:10BFC00081508F708BA38091990E8B1103C0CEACE2
:10BFD000DAA8B6CF0BA10B1529F081E08B0D8F707D
:10BFE000B82EF1CF1091990E1BA3C12CD12C8091AA
:10BFF0009A0E0BA1801709F447CB802E912C28E5CF
:10C00000289D8001299D100D11240B531B4FD80131
:10C010008C9183FD0AC05801C114D10439F0C601C6
:10C020000E942C7E811102C0BFC156018BA18F5F7F
:10C030008F708BA36501DBCF802F81508F70289F7D
:10C04000F0011124EB53FB4F908193FF28CB89A77C
:10C0500022CB48E5439FC0011124DC01AB53BB4F09
:10C060001D018C9183FD19C015966D917D918D9167
:10C070009C9118970E944BE0F62EE72ED82EC92EE1
:10C080000115110509F48AC0F801808180FD0AC0FC
:10C09000D1018C9180FD06C081C0FDA4EDA0D9A87E
:10C0A000CEAC81C0F801808181608083C8010E948C
:10C0B0002C7E81116FC0F80161817281838194812E
:10C0C0000E944BE02B013C019B01AC0160E070E061
:10C0D00080E89FE30E94BCDE4B015C019B01AC0148
:10C0E0006F2D7E2D8D2D9C2D0E94F9D969837A8329
:10C0F0008B839C832DA53DA149A95EADC501B401EB
:10C100000E94F9D9698B7A8B8B8B9C8BAE014F5F28
:10C110005F4FBE016F5E7F4FC8010E9434B1D801EE
:10C12000D7968C918823B1F12091550C3091560C03
:10C130004091570C5091580CF801FE966081718126
:10C14000828193810E94F9D92091031630910416BF
:10C1500040910516509106160E94F9D94B015C01D9
:10C160009B01AC01C301B2010E94F9D90E9429DFF1
:10C17000F80173AF62AFA50194016F2D7E2D8D2D57
:10C180009C2D0E94F9D90E9429DFD801DD967C936D
:10C190006E93DC97F80180818E7F80838F2C9E2C9C
:10C1A000AD2CBC2C81018BA18F5F8F708BA3FDA662
:10C1B000EDA2D9AACEAE7FCAD1018C9181608C93B9
:10C1C000C8010E942C7E81116BC0F10161817281D6
:10C1D000838194810E944BE06B017C019B01AC0147
:10C1E00060E070E080E89FE30E94BCDE2B013C0130
:10C1F0002DEC3CEC4CE45DE30E94F9D969837A8331
:10C200008B839C839401A501C301B2010E94F9D9DB
:10C21000698B7A8B8B8B9C8BAE014F5F5F4FBE011E
:10C220006F5E7F4FC1010E9434B1D101D7968C91CE
:10C230008823B1F12091550C3091560C4091570C48
:10C240005091580CF101FE96608171818281938139
:10C250000E94F9D9209103163091041640910516D9
:10C26000509106160E94F9D94B015C019B01AC016B
:10C27000C701B6010E94F9D90E9429DFF10173AF0D
:10C2800062AF2DEC3CEC4CE45DE3C501B4010E94CF
:10C29000F9D90E9429DFD101DD967C936E93DC975A
:10C2A000F10180818E7F80830ECA28E5269DF001F2
:10C2B000279DF00D1124EB53FB4F808181FD43C07E
:10C2C000C114D10441F0D6011596CD90DD90ED90CA
:10C2D000FC90189708C08BE0C82E87EDD82E83E21B
:10C2E000E82E8BE3F82EB8E5B69DF001B79DF00D72
:10C2F0001124EB53FB4F81899289A389B489BC0136
:10C30000CD0190589B01AC010E94E0DDF80125852C
:10C310003685478550890E94F9D99B01AC01C70138
:10C32000B6010E94DFDDE62E872E982EA92E262F3D
:10C33000372F482F592F69A57DA58DA199A90E9456
:10C3400094D987FF04C0E9A48DA49DA0A9A82E2D8F
:10C35000382D492D5A2DC201B1010E9494D988234C
:10C3600009F42DCEF8E5F69DC001F79D900D11243E
:10C370009C012B533B4F6901D9018C9181608C93B7
:10C38000C8010E942C7E882329F0F60180818E7FCF
:10C39000808315CE8E2D982DA92DBA2DF60185837B
:10C3A0009683A783B0870BCED6018C9181FD52C0B6
:10C3B000D60115962D913D914D915C91189729A725
:10C3C0003AA74BA75CA71501B5E02B0E311CF8016D
:10C3D0004580568067807084A301920169A57AA583
:10C3E0008BA59CA50E9494D987FF34C0F601818952
:10C3F0009289A389B489BC01CD0190589B01AC01FD
:10C400000E94E0DDD6011D962D913D914D915C91EC
:10C4100050970E94F9D99B01AC0169A57AA58BA51B
:10C420009CA50E94DFDD6B017C019B01AC01C30177
:10C43000B2010E9406E018166CF4D8018C9181605C
:10C440008C93C5010E942C7E8823E1F0F801808145
:10C450008E7F808318E5189DF001199DF00D112441
:10C46000EB53FB4F21853285438554856581768169
:10C47000878190850E9494D98111D8CD0BA100931A
:10C48000990ED4CDD101CD92DD92ED92FC9213970D
:10C490000BA10093990EDECFC858DF4F0FB6F8946A
:10C4A000DEBF0FBECDBFDF91CF911F910F91FF90E7
:10C4B000EF90DF90CF90BF90AF909F908F907F9044
:10C4C0006F905F904F903F902F90089580919A0EBB
:10C4D00090919B0E891B8F708F3019F40E94099CDC
:10C4E000F5CF80919A0E8F5F8F70E0919A0E98E54C
:10C4F0009E9FF0011124EB53FB4FDF011D929A9593
:10C50000E9F798E090834091C00E5091C10E609180
:10C51000C20E7091C30E458B568B678B708F409106
:10C52000C40E5091C50E6091C60E7091C70E418F1A
:10C53000528F638F748F4091C80E5091C90E6091D5
:10C54000CA0E7091CB0E458F568F678F70A34091A6
:10C55000CC0E5091CD0E6091CE0E7091CF0E41A3B6
:10C5600052A363A374A320919A0E90919B0E29135A
:10C5700003C094E69093970E80939A0E80916F007B
:10C58000826080936F00089590919A0E80919B0E27
:10C59000981306C08091D7149091D814892B19F064
:10C5A0000E94099CF1CF0895CF93DF938B3D924079
:10C5B000B1F0E6E8FBE18491EF012196882321F0B8
:10C5C0000E9488C5FE01F7CFE4E3FAE18491EF0110
:10C5D0002196882331F00E9488C5FE01F7CF80E0C4
:10C5E00001C081E0DF91CF9108952F923F924F9249
:10C5F0005F926F927F928F929F92AF92BF92CF92F3
:10C60000DF92EF92FF920F931F93CF93DF93CDB7FB
:10C61000DEB7C757D1090FB6F894DEBF0FBECDBF46
:10C620002DB63EB6A7961FAE1EAEA79784E690E045
:10C63000A9969FAF8EAFA99701E09E012B593F4F5E
:10C6400044E050E0BE01655A7F4FCE0189599F4FAB
:10C650000E94A0B69E012B593F4F42E050E0BE0120
:10C6600067597F4FCE0189599F4F0E94A0B643E082
:10C6700050E0BE01655A7F4F8FED92E00E944BE182
:10C68000892B09F43FC06F968FAD6F97882339F0DF
:10C690008FE36C968FAF6C976D961FAE6D97EBE93D
:10C6A000FBE184917F012FEFE21AF20A811103C0AE
:10C6B000E7EFFAE104C00E9488C5F701F2CF849148
:10C6C0007F013FEFE31AF30A882321F00E9488C517
:10C6D000F701F5CFBE01655A7F4F8EEE9AE10E94B9
:10C6E000D950E0EEFAE184917F019FEFE91AF90A4F
:10C6F000882321F00E9488C5F701F5CF81E080935F
:10C70000880C54C5EDB7FEB7E696FFAFEEAFE697DF
:10C710006B961CAE1DAE1EAE1FAE6B97A7961FAEDE
:10C720001EAEA79701E09E012B593F4F41E050E01C
:10C73000BE0160597F4FCE0189599F4F0E94A0B61C
:10C7400080E1EBE5F2E0DE01919601900D928A9591
:10C75000E1F780E1EBE6F2E0DE01519601900D9207
:10C760008A95E1F780E1EBE7F2E0DE0111960190B6
:10C770000D928A95E1F7E1964FADE19750E04D5F5C
:10C780005F4F440F551F440F551F2DB73EB7241B55
:10C79000350B0FB6F8943EBF0FBE2DBF8DB79EB7B9
:10C7A00001967C0100E09E012B593F4FBC01CE0158
:10C7B00089599F4F0E94A0B69E012B593F4F44E0DC
:10C7C00050E065E77CE0CE0189599F4F0E94A0B6FA
:10C7D000E1968FACE197912C93E0890E911C880C27
:10C7E000991C880C991CEDB7FEB7E819F9090FB62A
:10C7F000F894FEBF0FBEEDBF2DB73EB72F5F3F4F82
:10C8000069018DB79EB7881999090FB6F8949EBF34
:10C810000FBE8DBFEDB7FEB731965F019E012B595C
:10C820003F4FA401B601CE0189599F4F0E94A0B687
:10C830009E012B593F4FA401B501CE0189599F4F4D
:10C840000E94A0B61091890C112309F4A7C000E042
:10C850009E012B593F4F44E050E06DE57CE0CE0156
:10C8600089599F4F0E94A0B69E012B593F4F44E02B
:10C8700050E061E67CE0CE0189599F4F0E94A0B64E
:10C880009E012B593F4F44E050E069E57CE0CE012A
:10C8900089599F4F0E94A0B69E012B593F4F44E0FB
:10C8A00050E06DE77CE0CE0189599F4F0E94A0B611
:10C8B0009E012B593F4F44E050E069E77CE0CE01F8
:10C8C00089599F4F0E94A0B69E012B593F4F40E1CE
:10C8D00050E065E47CE0CE0189599F4F0E94A0B6EC
:10C8E0009E012B593F4F44E050E0BE01695A7F4FF3
:10C8F000CE0189599F4F0E94A0B69E012B593F4FF0
:10C900004CE050E06AEA7AE0CE0189599F4F0E94DC
:10C91000A0B69E012B593F4F44E050E067E276E11C
:10C92000CE0189599F4F0E94A0B69E012B593F4FBF
:10C9300044E050E0BE01695A7F4FCE0189599F4FB4
:10C940000E94A0B601E09E012B593F4F41E050E00C
:10C95000BE0161597F4FCE0189599F4F0E94A0B6F9
:10C960009E012B593F4F41E050E0BE0162597F4F7D
:10C97000CE0189599F4F0E94A0B611118AC06B96B3
:10C980008CAD9DADAEADBFAD6B9780932F169093E0
:10C990003016A0933116B09332167BC0E1968FAD5E
:10C9A000E19790E0029625E63CE0E4963FAF2EAF9B
:10C9B000E497B501DE011196E7EF8E2EE5E19E2E9C
:10C9C000AE014F5E5F4FF0E9AF2EF7E1BF2EE89664
:10C9D000FFAEEEAEE8977E0131E2E30EF11C20E0FF
:10C9E00030E0821793072CF0E896EEADFFADE897A4
:10C9F00001C0F7014080518062807380F50141924F
:10CA00005192619271925F018217930714F0F601BF
:10CA100001C0FA014080518062807380F40141922C
:10CA20005192619271924F018217930734F0FB018A
:10CA3000408051806280738005C04D905D906D9004
:10CA40007C901397E496EEADFFADE497419251923E
:10CA500061927192E496FFAFEEAFE4972F5F3F4F84
:10CA60006C5F7F4F1496F4E0CF0ED11C4C5F5F4F8C
:10CA7000E896EEADFFADE8973496E896FFAFEEAFDF
:10CA8000E897F4E0EF0EF11C2430310509F0A9CF4E
:10CA9000DECEE0968FADE097853099F4AF968FADFE
:10CAA000AF97853071F400E09E012B593F4F44E66B
:10CAB00050E063E376E1CE0189599F4F0E94A0B612
:10CAC00024C0111102C00E94D3B5E0968FADE0974B
:10CAD000AF96CFACAF978C9D60011124E12CF12C67
:10CAE000EC14FD0491F000E09E012B593F4F44E00F
:10CAF00050E0BE01695A7F4FCE0189599F4F0E9475
:10CB0000A0B62FEFE21AF20AEBCF00E09E012B59FC
:10CB10003F4F44E050E0BE016D5A7F4FCE0189592E
:10CB20009F4F0E94A0B61AE0115079F000E09E01DC
:10CB30002B593F4F44E050E0BE01695A7F4FCE0170
:10CB400089599F4F0E94A0B6EFCF01E09E012B595B
:10CB50003F4F41E050E0BE0163597F4FCE018959FC
:10CB60009F4F0E94A0B69E012B593F4F41E050E0DD
:10CB7000BE0164597F4FCE0189599F4F0E94A0B6D4
:10CB800000E09E012B593F4F44E050E0BE01635C42
:10CB90007F4FCE0189599F4F0E94A0B69E012B590D
:10CBA0003F4F44E050E0BE016F5C7F4FCE0189599A
:10CBB0009F4F0E94A0B6AE968FADAE97AD96CFAC0C
:10CBC000AD978C9D60011124E12CF12C00E09E01B9
:10CBD0002B593F4FCE14DF0471F044E050E0BE010A
:10CBE000695A7F4FCE0189599F4F0E94A0B63FEFEF
:10CBF000E31AF30AEBCF41E050E0BE016F587F4FDC
:10CC0000CE0189599F4F0E94A0B69E012B593F4FDC
:10CC100041E050E0BE0165597F4FCE0189599F4FD9
:10CC20000E94A0B69E012B593F4F44E050E0BE0148
:10CC3000695A7F4FCE0189599F4F0E94A0B69E012D
:10CC40002B593F4F44E050E0BE01695A7F4FCE015F
:10CC500089599F4F0E94A0B69E012B593F4F44E037
:10CC600050E06BE276E1CE0189599F4F0E94A0B659
:10CC70009E012B593F4F44E050E0BE01615B7F4F66
:10CC8000CE0189599F4F0E94A0B69E012B593F4F5C
:10CC900044E050E0BE01655B7F4FCE0189599F4F54
:10CCA0000E94A0B69E012B593F4F44E050E0BE01C8
:10CCB000695B7F4FCE0189599F4F0E94A0B610E05B
:10CCC00000E09E012B593F4F44E050E0BE01695AFD
:10CCD0007F4FCE0189599F4F0E94A0B6111110C0FD
:10CCE0006B96CCACDDACEEACFFAC6B9720E030E8E3
:10CCF0004BE355E4C701B6010E9494D9811103C0EA
:10CD000054E0F52E33C08091890C811108C0C09287
:10CD1000C914D092CA14E092CB14F092CC1400E063
:10CD20009E012B593F4F44E050E065EC74E1CE0189
:10CD300089599F4F0E94A0B69E012B593F4F44E056
:10CD400050E06DEC74E1CE0189599F4F0E94A0B66E
:10CD50009E012B593F4F44E050E0BE01695A7F4F7E
:10CD6000CE0189599F4F0E94A0B612C0FA94FF20AD
:10CD700079F000E09E012B593F4F44E050E0BE01A6
:10CD8000695A7F4FCE0189599F4F0E94A0B6EECFBE
:10CD90001F5F153009F094CF00E09E012B593F4FE3
:10CDA00042E050E0BE016D597F4FCE0189599F4F3F
:10CDB0000E94A0B69E012B593F4F44E050E0BE01B7
:10CDC000695A7F4FCE0189599F4F0E94A0B66B963A
:10CDD000CCACDDACEEACFFAC6B9720E030E84BE3C5
:10CDE00055E4C701B6010E9494D9882329F18091A6
:10CDF000890C811108C0C092C114D092C214E09273
:10CE0000C314F092C41400E09E012B593F4F44E03C
:10CE100050E06DEB74E1CE0189599F4F0E94A0B69E
:10CE20009E012B593F4F44E050E069EB74E1CE0185
:10CE300089599F4F0E94A0B600E09E012B593F4F99
:10CE400042E050E0BE016F597F4FCE0189599F4F9C
:10CE50000E94A0B69E012B593F4F41E050E0BE0119
:10CE60006F587F4FCE0189599F4F0E94A0B619E09D
:10CE7000115000E09E012B593F4F112359F044E01F
:10CE800050E0BE01695A7F4FCE0189599F4F0E94E1
:10CE9000A0B6EECF41E050E067E976E1CE018959D6
:10CEA0009F4F0E94A0B6F12C00E09E012B593F4FEE
:10CEB00044E050E0BE01695A7F4FCE0189599F4F2F
:10CEC0000E94A0B61091890C111110C0F1100EC073
:10CED0006B968CAD9DADAEADBFAD6B9780939C1640
:10CEE00090939D16A0939E16B0939F16F39485E0A1
:10CEF000F812DACF111102C00E94B2474CE0F42EB2
:10CF0000FA94F11003C03CE0F32E0FC000E09E0144
:10CF10002B593F4F42E050E0BE01615A7F4FCE0196
:10CF200089599F4F0E94A0B6EBCFFA9400E09E0172
:10CF30002B593F4FFF2059F044E050E0BE016D5B9C
:10CF40007F4FCE0189599F4F0E94A0B6EECF46E099
:10CF500050E0BE01635C7F4FCE0189599F4F0E9414
:10CF6000A0B69E012B593F4F44E050E065E57CE0C0
:10CF7000CE0189599F4F0E94A0B69E012B593F4F69
:10CF80004CE050E0BE016F5C7F4FCE0189599F4F4E
:10CF90000E94A0B62CE1F22EFA94F11003C094E0A6
:10CFA000F92E1DC000E09E012B593F4F44E050E098
:10CFB000BE01695A7F4FCE0189599F4F0E94A0B68A
:10CFC000EBCF00E09E012B593F4F44E050E0BE0103
:10CFD000695A7F4FCE0189599F4F0E94A0B6FA949B
:10CFE000F110EFCF8BE0F82EFA94FF2079F000E0FB
:10CFF0009E012B593F4F44E050E0BE01695A7F4FDC
:10D00000CE0189599F4F0E94A0B6EECFA9968EAD52
:10D010009FADA99784569109C7DA8093880C88231D
:10D0200009F1EBE9FBE184917F019FEFE91AF90A2D
:10D03000882321F00E9488C5F701F5CFA9966EAD2F
:10D040007FADA9976456710988ED9AE10E94C0509E
:10D050006BED72E080ED9AE10E94C0508AE00E9480
:10D0600088C599C0A7962EAD3FADA797AB968EAD5C
:10D070009FADAB972817390709F44BC081E0809327
:10D08000880CE6E8FBE184917F012FEFE21AF20AB7
:10D09000811103C0E0EBFAE104C00E9488C5F701EA
:10D0A000F2CF84917F013FEFE31AF30A882321F046
:10D0B0000E9488C5F701F5CFAB966EAD7FADAB97FB
:10D0C00080E090E04AE00E948FC5EBEAFAE18491AB
:10D0D0007F019FEFE91AF90A882321F00E9488C591
:10D0E000F701F5CFA7966EAD7FADA79780E090E0F2
:10D0F0004AE00E948FC5EBE9FAE184917F012FEFAE
:10D10000E21AF20A882309F446C00E9488C5F70192
:10D11000F4CF111142C0EBE9FBE184917F013FEFB5
:10D12000E31AF30A811103C00FED12E004C00E945C
:10D1300088C5F701F2CFF80181918F01882319F09A
:10D140000E9488C5F8CFA9966EAD7FADA9976456A9
:10D1500071098EE79AE10E94C050A7964EAD5FAD6F
:10D16000A79760E070E081E79AE10E948650EEE6C2
:10D17000FAE184917F012FEFE21AF20A811107C0D0
:10D180008091880C811109C00E9461B706C00E947D
:10D1900088C5F701EECF112399F3E6968EAD9FADCA
:10D1A000E6970FB6F8949EBF0FBE8DBF8091890C95
:10D1B000811102C00E946EAA9091880C81E089279B
:10D1C0000FB6F8943EBE0FBE2DBEC958DF4F0FB646
:10D1D000F894DEBF0FBECDBFDF91CF911F910F91AD
:10D1E000FF90EF90DF90CF90BF90AF909F908F9087
:10D1F0007F906F905F904F903F902F90089581E0C7
:10D200008093890CF2D91092890C8111EEC90E9489
:10D2100003AF81E008958F929F92AF92BF92CF9219
:10D22000DF92EF92FF920F931F93CF93DF93CDB7CF
:10D23000DEB7CA5AD1090FB6F894DEBF0FBECDBF14
:10D24000E9961CAE1DAE1EAE1FAEE9978091EC03B1
:10D250009091ED03A091EE03B091EF03ED968CAFAA
:10D260009DAFAEAFBFAFED97C556DF4F19821882A5
:10D27000CB59D04084E690E0C356DF4F9983888332
:10D28000CD59D0401092880C9E0125563F4F44E066
:10D2900050E0BE0167587F4FCE0183569F4F0E94DA
:10D2A000EDB6C356DF4F88819981CD59D0400296A3
:10D2B000C356DF4F99838883CD59D040C556DF4F81
:10D2C00019821882CB59D04081E0CD55DF4F888339
:10D2D000C35AD0409E0125563F4F41E050E0BE0169
:10D2E0006D557F4FCE0183569F4F0E94EDB69E0134
:10D2F00025563F4F40E150E060E977E1CE0183568B
:10D300009F4F0E94EDB69E0125563F4F44E050E0EE
:10D3100065E77CE0CE0183569F4F0E94EDB69E01EB
:10D3200025563F4F40E150E067EF75E1CE0183564F
:10D330009F4F0E94EDB69E0125563F4F40E150E0C1
:10D3400065E67CE0CE0183569F4F0E94EDB69E01BC
:10D3500025563F4F44E050E06DE57CE0CE0183561A
:10D360009F4F0E94EDB69E0125563F4F44E050E08E
:10D3700061E67CE0CE0183569F4F0E94EDB69E0190
:10D3800025563F4F44E050E069E57CE0CE018356EE
:10D390009F4F0E94EDB69E0125563F4F44E050E05E
:10D3A0006DE77CE0CE0183569F4F0E94EDB69E0153
:10D3B00025563F4F44E050E069E77CE0CE018356BC
:10D3C0009F4F0E94EDB69E0125563F4F40E150E031
:10D3D00065E47CE0CE0183569F4F0E94EDB68AE063
:10D3E00097EDA3EABCE3E9968CAF9DAFAEAFBFAFBC
:10D3F000E9979E0125563F4F44E050E0BE016B582F
:10D400007F4FCE0183569F4F0E94EDB69E01255659
:10D410003F4F4CE050E06AEA7AE0CE0183569F4FDE
:10D420000E94EDB68091E2159091E315A091E4156C
:10D43000B091E515C358DF4F88839983AA83BB83D6
:10D44000CD57D0409E0125563F4F44E050E0BE01ED
:10D4500063587F4FCE0183569F4F0E94EDB685E003
:10D46000CC55DF4F8883C45AD040CB55DF4F8883DB
:10D47000C55AD0409E0125563F4F44E050E06FE230
:10D4800076E1CE0183569F4F0E94EDB69E01255650
:10D490003F4F41E050E0BE016C557F4FCE018356B7
:10D4A0009F4F0E94EDB69E0125563F4F41E050E050
:10D4B000BE016B557F4FCE0183569F4F0E94EDB644
:10D4C0009E0125563F4F44E650E063E376E1CE01EE
:10D4D00083569F4F0E94EDB6CF57DF4F18821982B7
:10D4E0001A821B82C158D0409E0125563F4F44E00E
:10D4F00050E0BE016F577F4FCE0183569F4F0E9471
:10D50000EDB6E9961CAE1DAE1EAE1FAEE9971AE051
:10D51000115071F09E0125563F4F44E050E0BE018E
:10D520006B587F4FCE0183569F4F0E94EDB6F0CFD0
:10D5300083E0CA55DF4F8883C65AD040C955DF4FB4
:10D540008883C75AD040CB57DF4F188219821A827E
:10D550001B82C558D040C757DF4F188219821A82E4
:10D560001B82C958D040E9961CAE1DAE1EAE1FAE40
:10D57000E9979E0125563F4F41E050E0BE016A55B4
:10D580007F4FCE0183569F4F0E94EDB69E012556D8
:10D590003F4F41E050E0BE0169557F4FCE018356B9
:10D5A0009F4F0E94EDB69E0125563F4F44E050E04C
:10D5B000BE0167577F4FCE0183569F4F0E94EDB645
:10D5C0009E0125563F4F44E050E0BE016B577F4F10
:10D5D000CE0183569F4F0E94EDB60AE010E0015045
:10D5E000110971F09E0125563F4F44E050E0BE0105
:10D5F0006B587F4FCE0183569F4F0E94EDB6EFCF01
:10D60000C855DF4F1882C85AD0408FEFC755DF4F3B
:10D610008883C95AD0409E0125563F4F41E050E0D3
:10D62000BE0168557F4FCE0183569F4F0E94EDB6D5
:10D630009E0125563F4F41E050E0BE0167557F4FA8
:10D64000CE0183569F4F0E94EDB6E9961CAE1DAEEB
:10D650001EAE1FAEE9979E0125563F4F44E050E0B5
:10D66000BE016B587F4FCE0183569F4F0E94EDB68F
:10D670009E0125563F4F44E050E0BE016B587F4F5E
:10D68000CE0183569F4F0E94EDB69E0125563F4F17
:10D6900044E050E06BE276E1CE0183569F4F0E945A
:10D6A000EDB680918B0290918C02A0918D02B09189
:10D6B0008E02C357DF4F88839983AA83BB83CD58DB
:10D6C000D04080918F0290919002A0919102B091F0
:10D6D0009202CF56DF4F88839983AA83BB83C159B7
:10D6E000D040CB56DF4F19821882C559D040C95659
:10D6F000DF4F19821882C759D0409E0125563F4FEF
:10D7000044E050E0BE0163577F4FCE0183569F4FE8
:10D710000E94EDB69E0125563F4F44E050E0BE0109
:10D720006F567F4FCE0183569F4F0E94EDB69E01EC
:10D7300025563F4F44E050E0BE016B567F4FCE016F
:10D7400083569F4F0E94EDB610E0C12C80E8D82E82
:10D750008BE3E82E85E4F82E812C912C90E8A92EFD
:10D760009FE3B92E111138C09E0125563F4F44E06A
:10D7700050E069EC74E1CE0183569F4F0E94EDB6F4
:10D780009E0125563F4F44E050E065EC74E1CE0128
:10D7900083569F4F0E94EDB69E0125563F4F44E0B1
:10D7A00050E06DEC74E1CE0183569F4F0E94EDB6C0
:10D7B000E9968CAE9DAEAEAEBFAEE9979E01255602
:10D7C0003F4F44E050E0BE016B587F4FCE0183567F
:10D7D0009F4F0E94EDB62AC0E996CCAEDDAEEEAE0C
:10D7E000FFAEE9979E0125563F4F44E050E0BE0151
:10D7F0006B587F4FCE0183569F4F0E94EDB6E9963E
:10D800001CAE1DAE1EAE1FAEE99704E0015071F0D4
:10D810009E0125563F4F44E050E0BE016B587F4FBC
:10D82000CE0183569F4F0E94EDB6F0CF1F5F15309B
:10D8300009F098CF84E190E0C156DF4F9983888347
:10D84000CF59D0409E0125563F4F42E050E0BE01E7
:10D8500061567F4FCE0183569F4F0E94EDB69E01C9
:10D8600025563F4F44E050E061EC74E1CE01835611
:10D870009F4F0E94EDB69E0125563F4F44E050E079
:10D880006DEB74E1CE0183569F4F0E94EDB69E0171
:10D8900025563F4F44E050E069EB74E1CE018356DA
:10D8A0009F4F0E94EDB680E290E0CF55DF4F998305
:10D8B0008883C15AD0409E0125563F4F42E050E038
:10D8C000BE016F557F4FCE0183569F4F0E94EDB62C
:10D8D000C655DF4F1882CA5AD04080E2E3E9F2E031
:10D8E000DE019D9601900D928A95E1F79E012556E5
:10D8F0003F4F41E050E0BE0166557F4FCE01835659
:10D900009F4F0E94EDB69E0125563F4F40E250E0EA
:10D91000BE01635D7F4FCE0183569F4F0E94EDB6DF
:10D920009E0125563F4F41E050E067E976E1CE0188
:10D9300083569F4F0E94EDB610E011110EC08091EA
:10D940009C1690919D16A0919E16B0919F16E996F7
:10D950008CAF9DAFAEAFBFAFE9979E0125563F4F4D
:10D9600044E050E0BE016B587F4FCE0183569F4F7D
:10D970000E94EDB61F5F153001F7BE01635B7F4F5C
:10D9800086E1FB0111928A95E9F79E0125563F4FEA
:10D9900046E150E0CE0183569F4F0E94EDB68CE2E7
:10D9A000E3EBF2E0DE01119601900D928A95E1F72A
:10D9B0009E0125563F4F4CE250E0BE016F5F7F4F06
:10D9C000CE0183569F4F0E94EDB6BE0161597F4F35
:10D9D00086E0FB0111928A95E9F79E0125563F4F9B
:10D9E00046E050E0CE0183569F4F0E94EDB69E0167
:10D9F00025563F4F44E050E065E57CE0CE0183567C
:10DA00009F4F0E94EDB6BE016D597F4F8CE0FB0128
:10DA100011928A95E9F79E0125563F4F4CE050E060
:10DA2000CE0183569F4F0E94EDB6E9961CAE1DAE07
:10DA30001EAE1FAEE9971CE1115071F09E012556F4
:10DA40003F4F44E050E0BE016B587F4FCE018356FC
:10DA50009F4F0E94EDB6F0CFE9961CAE1DAE1EAEF4
:10DA60001FAEE99714E0115071F09E0125563F4F0B
:10DA700044E050E0BE016B587F4FCE0183569F4F6C
:10DA80000E94EDB6F0CFE9961CAE1DAE1EAE1FAEE5
:10DA9000E9971BE0115071F09E0125563F4F44E07D
:10DAA00050E0BE016B587F4FCE0183569F4F0E94BE
:10DAB000EDB6F0CF8091880C811167C0C356DF4F5F
:10DAC000E880F980CD59D040F4E6EF1AF108C55648
:10DAD000DF4F88819981CB59D040C756DF4F99835A
:10DAE0008883C959D04084E690E0C356DF4F9983BC
:10DAF0008883CD59D0409E0125563F4F44E050E0E9
:10DB00006FED72E0CE0183569F4F0E94EDB69E01ED
:10DB100025563F4F42E050E0BE0167567F4FCE0191
:10DB200083569F4F0E94EDB6EBE9FBE184918F0194
:10DB30000F5F1F4F882321F00E9488C5F801F6CFA0
:10DB4000B7018CE59AE10E94C050C756DF4F48816B
:10DB50005981C959D04060E070E08FE49AE10E9499
:10DB60008650ECE4FAE184918F010F5F1F4F882308
:10DB700021F00E9488C5F801F6CFC7010E94D46247
:10DB80009091880C892B8093880C9091880C81E06F
:10DB90008927C655DF4F0FB6F894DEBF0FBECDBF45
:10DBA000DF91CF911F910F91FF90EF90DF90CF9079
:10DBB000BF90AF909F908F9008958F929F92AF9259
:10DBC000BF92CF92DF92EF92FF921F93CF93DF939A
:10DBD000C82F8AEB90E19093960E8093950E109249
:10DBE000D61082E090E0A0E0B0E08093BF10909368
:10DBF000C010A093C110B093C2101092940E109256
:10DC0000900E1092910E1092920E1092930E8FEF32
:10DC10009FEFDC0180938C0E90938D0EA0938E0E5F
:10DC2000B0938F0ECC2379F1C53008F0F8C040E0F6
:10DC300060E070E0CB010E9449B8882309F4EFC08E
:10DC400020E1C29FC00111248458934FFC01E2548B
:10DC5000FE4F20812F7709F0E2C03C964081518130
:10DC600062817381443651056105710508F4D7C09E
:10DC70003497C080D180E280F380C114D104E104E4
:10DC8000F10421F4CCC0C12CD12C760140E0C701B5
:10DC9000B6010E9449B8182F882309F4C0C08091AA
:10DCA000970C9091980C8115924009F0B8C0A09102
:10DCB0009C0CAA2309F4B3C060919A0C70919B0C40
:10DCC0006115710509F4ABC02091990C222309F468
:10DCD000A6C0A093D1102093C31080E030E041E0B3
:10DCE00050E0C82FFA01082E02C0EE0FFF1F0A9461
:10DCF000E2F72E173F0739F08F5FC83091F789E0C0
:10DD00008093CC108CC08093CC102091A20C3091C9
:10DD1000A30C2115310519F040E050E008C0209116
:10DD2000B00C3091B10C4091B20C5091B30C2093D7
:10DD3000C4103093C5104093C6105093C7104601CD
:10DD40005701860E971EA11CB11C8092D210909292
:10DD5000D310A092D410B092D510E0919D0CF09108
:10DD60009E0CF093D810E093D710B0E00E94C0DD75
:10DD7000860E971EA81EB91E8092D9109092DA10B6
:10DD8000A092DB10B092DC1085E0EE0FFF1F8A95A9
:10DD9000E1F7E150FE4FEF2FFF27E6958E0E9F1E15
:10DDA000A11CB11C8092CD109092CE10A092CF10E9
:10DDB000B092D01020919F0C3091A00C211531050C
:10DDC00021F0A90160E070E008C04091AC0C5091D6
:10DDD000AD0C6091AE0C7091AF0CD701C6018819E3
:10DDE0009909AA09BB09840F951FA61FB71F04C074
:10DDF000B695A79597958795CA95D2F78093C81041
:10DE00009093C910A093CA10B093CB10853F2FE018
:10DE10009207A105B10528F48CE08093D61010E09C
:10DE20001AC0853F9F4FA105B10510F480E111C0D4
:10DE30008091B80C9091B90CA091BA0CB091BB0C28
:10DE40008093D9109093DA10A093DB10B093DC107C
:10DE500080E28093D610812FDF91CF911F91FF90A8
:10DE6000EF90DF90CF90BF90AF909F908F900895EC
:10DE7000682F81E894E10C94AB39CF92DF92EF9256
:10DE8000FF921F93CF93DF931092190F80914C0F45
:10DE9000882321F089E49FE00E9454931092BE10E1
:10DEA0001092BB1085E38093BA100E94A551EB013C
:10DEB000A89561E08091BA100E9431A98AEB90E1A7
:10DEC0000E94B5942398229A219A209A289A85E054
:10DED0008093BC1082E58CBD1DBC1AE08FEF0E94C0
:10DEE000BA941150D9F720E030E0A90160E08AEB44
:10DEF00090E10E94BF94182F8093BD10813049F0AB
:10DF00000E94A5516C1B7D0B613D774060F381E061
:10DF100054C02AEA31E040E050E068E08AEB90E14A
:10DF20000E94BF9482FF03C01093BE100EC014E085
:10DF30000E94CD998093BD101150D1F78A3A11F00B
:10DF400082E03BC082E08093BE108091BE108230A0
:10DF500021F0C12CD12C760105C0C12CD12CE12C93
:10DF600080E4F82E20E030E0A90167E38AEB90E13D
:10DF70000E94BF94A701960169E28AEB90E10E949A
:10DF8000BF948093BD10882349F00E94A5516C1B5B
:10DF90007D0B613D774030F38AE00FC08091BE1069
:10DFA000823011F520E030E0A9016AE38AEB90E1CC
:10DFB0000E94BF94882351F088E08093BB108AEBC5
:10DFC00090E10E94B594EBE9FBE119C00E94CD9964
:10DFD000807C803C19F483E08093BE100E94CD9930
:10DFE0000E94CD990E94CD998AEB90E10E94B59450
:10DFF0001092BC1081E0E1DD811131C015C0849127
:10E00000EF012196882321F00E9488C5FE01F7CFF9
:10E01000EDE8FBE18491EF012196882309F456C0D5
:10E020000E9488C5FE01F6CF80E0C7DD811117C0D0
:10E03000E6E8FBE18491EF012196882321F00E941C
:10E0400088C5FE01F7CFE2E7FBE18491EF0121965D
:10E05000882309F43BC00E9488C5FE01F6CF6FEB10
:10E0600070E189E49FE00E940193811116C0E6E807
:10E07000FBE18491EF012196882321F00E9488C55D
:10E08000FE01F7CFE1E6FBE18491EF0121968823C1
:10E09000E9F00E9488C5FE01F7CF81E08093190F57
:10E0A000EBE9FBE18491EF012196882321F00E94A6
:10E0B00088C5FE01F7CFE5E5FBE18491EF012196EC
:10E0C000882321F00E9488C5FE01F7CF8BE1E9E4A7
:10E0D000FFE0A8E6BFE001900D928A95E1F78091FC
:10E0E000470F9091480F9093670F8093660FDF91D1
:10E0F000CF911F91FF90EF90DF90CF900895809186
:10E100002613823041F480E49BE190938B0C809342
:10E110008A0C0E945E8B0E94A55160932A13709313
:10E120002B1380932C1390932D138091190F882318
:10E1300019F081E08093180F81E0809326130895F1
:10E14000CF93DF931092180F83E080932613809172
:10E1500073138823B1F0E8E3FBE18491EF01882396
:10E1600041F0082E000C990B83DE2196FE0184916C
:10E17000F6CF8DE090E07CDE8AE090E0DF91CF91F9
:10E1800077CEECE3FBE18491EF01882391F3082E35
:10E19000000C990B6DDE2196FE018491F6CF8F92D3
:10E1A0009F92AF92BF92CF92DF92EF92FF920F9326
:10E1B0001F93CF93DF9300D01F92CDB7DEB7FC0142
:10E1C0008381813079F5818181FF2CC08189928999
:10E1D000A389B489892B8A2B8B2B09F448C07F0132
:10E1E00040E050E0BA01CF010E946A928823D1F04A
:10E1F000F70185889688A788B08CC18CD28C82E084
:10E2000090E0A0E0B0E0F60180839183A283B38325
:10E210009E012F5F3F4FB501A401C6010E9412B9B4
:10E22000811102C080E03CC000E010E09801B5011F
:10E23000A401C6010E9481B88823A1F389809A8035
:10E24000AB80BC80F6018789803141F4F8EF8F16EE
:10E25000FFEF9F06A104B10460F4DACF88EF8816BF
:10E260008FEF9806A8068FE0B80618F4D1CF81E0AA
:10E2700017C0F701158A168A178A108E118A128A1A
:10E28000138A148A818180688183C7010E9460BAE1
:10E29000882341F240E050E0BA01C7010E946A922F
:10E2A0000F900F900F900F90DF91CF911F910F91D2
:10E2B000FF90EF90DF90CF90BF90AF909F908F90A6
:10E2C000089510921B0F1092180F8091E41088236C
:10E2D00021F081EE90E10C94549308952F923F9297
:10E2E0004F925F926F927F928F929F92AF92BF9266
:10E2F000CF92DF92EF92FF920F931F93CF93DF9312
:10E30000CDB7DEB7C257D1090FB6F894DEBF0FBE46
:10E31000CDBF8C013B014A014DB75EB7E1965FAFBF
:10E320004EAFE197AD961FAEAD971B0154E0250EA1
:10E33000311C7E018FE5E80EF11C9DEE492E92E026
:10E34000592EE0E4F0E0EC0FFD1F3496E396FFAFAA
:10E35000EEAFE397F3018781823008F462C18485D0
:10E360009585A685B7858F719927AA27BB27892B05
:10E370008A2B8B2B09F055C11092290F49E25FE0DF
:10E38000BE016F5F7F4FC1010E94F8B918160CF0F3
:10E3900048C18C85982F9871903129F4209196115D
:10E3A0002150223078F42981222309F43AC1253EF4
:10E3B00089F22E3279F22091290F2E3259F28A7089
:10E3C00049F6B8C04DB75EB7AF965FAF4EAFAF97E7
:10E3D000BE016F5F7F4FC7010E94F3B701151105A2
:10E3E00021F0F801808181119BC021E081E090E063
:10E3F000F70101900020E9F73197EE19FF098E0F20
:10E400009F1F02964DB75EB7481B590B0FB6F89485
:10E410005EBF0FBE4DBF8DB79EB701965C01211147
:10E4200002C0B80102C062E273E0C5010E9444E18B
:10E43000B701C5010E9425E162E273E0C5010E94B7
:10E4400025E125961FAE259728961FAE289724967E
:10E450001FAE1EAE249722965FAE4EAE229721E0ED
:10E46000A701B101E3968EAD9FADE3970E94E098BE
:10E4700081112AC080919611811126C0EBE9FBE140
:10E4800084916F019FEFC91AD90A882321F00E9455
:10E4900088C5F601F5CFE4E2FBE184916F012FEF2F
:10E4A000C21AD20A882321F00E9488C5F601F5CF4E
:10E4B0006701F60181916F01882319F00E9488C5D8
:10E4C000F8CF8AE00E9488C58BE1FE01EC5BFF4F2C
:10E4D000DE01959601900D928A95E1F724968EAD16
:10E4E0009FAD24979CA38BA35AA249A240E050E081
:10E4F000BE016F5D7F4FC501F1DECE0181960E94A6
:10E500009F9BCE01805C9F4F0E949F9BAF964EAD1C
:10E510005FADAF970FB6F8945EBF0FBE4DBF1ACF79
:10E52000F80101900020E9F73197CF01801B910B92
:10E5300020E05ECF81E0903109F080E080931A0FF7
:10E54000903141F08985873409F004CF8A858E3770
:10E5500009F400CF80919611813029F08230D9F1F1
:10E560008111F8CE0AC0809197119091981101966F
:10E570009093981180939711EDCEBE016F5F7F4FFE
:10E580008CE19FE00E94F3B70115110529F48CE19D
:10E59000C82E8FE0D82E09C06801F60181916F0165
:10E5A0008823A9F30E9488C5F8CFF60181916F01F5
:10E5B000882319F00E9488C5F8CF80E20E9488C5A0
:10E5C0006D8D7E8D8F8D98A14AE00E948FC58AE067
:10E5D0000E9488C5BFCEBE016F5F7F4F8CE19FE078
:10E5E0000E94F3B78114910441F06CE17FE0C40113
:10E5F0000E9412E1892B69F414C0AD96FFADAD976E
:10E600008F2F90E02091A3143091A41482179307C8
:10E6100041F0AD962FADAD972F5FAD962FAFAD9773
:10E6200099CEE1968EAD9FADE1970FB6F8949EBF5F
:10E630000FBE8DBFCE58DF4F0FB6F894DEBF0FBEB2
:10E64000CDBFDF91CF911F910F91FF90EF90DF90A1
:10E65000CF90BF90AF909F908F907F906F905F9082
:10E660004F903F902F9008950F931F93CF93DF9378
:10E67000CDB7DEB76F970FB6F894DEBF0FBECDBF34
:10E680008B0122E0209396119093A4148093A314FD
:10E6900088E69FE00E94B1948BE1E8E6FFE0DE01AE
:10E6A000159601900D928A95E1F78091660F9091F1
:10E6B000670F9C838B838DEE92E09A838983A801F8
:10E6C000BE016F5F7F4F80E090E008DECE010196D3
:10E6D0000E949F9B6F960FB6F894DEBF0FBECDBF12
:10E6E000DF91CF911F910F9108952F923F924F92FA
:10E6F0005F926F927F928F929F92AF92BF92CF92D2
:10E70000DF92EF92FF920F931F93CF93DF93CDB7DA
:10E71000DEB76F970FB6F894DEBF0FBECDBF6C01AA
:10E720002DB63EB61D8218861C821B828DEE92E0AD
:10E730009A838983FB0180819E012F5F3F4F3901BE
:10E740008F3241F084E69FE0F60191838083F62EBC
:10E75000172F64C085E49FE0F601918380838B01CD
:10E760000F5F1F4F0115110509F456C04DB65EB677
:10E770006FE270E0C8010E9430E14C0108171907F0
:10E7800008F048C07C01E01AF10AFF24C701019695
:10E790002DB73EB7281B390B0FB6F8943EBF0FBEFE
:10E7A0002DBF8DB79EB701965C01A701B8010E94ED
:10E7B00059E1F501EE0DFF1D1082F60160817181B6
:10E7C0006115710511F06C5F7F4F21E0A501CE014D
:10E7D00005960E94E098811111C0B50180E19BE18E
:10E7E0000E94D9508EE20E9488C58AE00E9488C5A6
:10E7F0000FB6F8945EBE0FBE4DBE0EC0F60171821C
:10E80000608284010F5F1F4F0FB6F8945EBE0FBE8B
:10E810004DBEA8CFF02E02C0F12C10E0C3010E9423
:10E820009F9B8F2D912F0FB6F8943EBE0FBE2DBE2D
:10E830006F960FB6F894DEBF0FBECDBFDF91CF91BC
:10E840001F910F91FF90EF90DF90CF90BF90AF900E
:10E850009F908F907F906F905F904F903F902F9000
:10E860000895FF920F931F93CF93DF938C01EB01D9
:10E87000F42E80E20E9488C58FEFF81611F084E52F
:10E8800001C082E40E9488C58AE30E9488C5F8011D
:10E89000608171818281938142E00E9414C6488127
:10E8A00059816A817B818CE39EE10E94A35062E0E2
:10E8B00070E080E090E0DF91CF911F910F91FF9089
:10E8C0000C9434AA8F929F92AF92BF92CF92DF9214
:10E8D000EF92FF920F931F93CF93DF93F0E2FF2EFF
:10E8E000E12CAE2DB0E0BD016F0D711D75956795E2
:10E8F0006E1511F0F6120BC0EFE1FCE16591749119
:10E90000072E000C880B990B0E949AD962C09B01BC
:10E9100021503109220F331F220F331FF901EF5508
:10E92000F44E05911491AB01440F551F440F551F30
:10E93000FA01EF55F44EC591D4918017910714F464
:10E94000F62ED1CFC817D90714F4E62ECACFF90195
:10E95000ED55F44EE590F490FA01ED55F44EC59066
:10E96000D490BC01601B710B072E000C880B990B17
:10E970000E949AD94B015C01B6016E197F09072EDE
:10E98000000C880B990B0E949AD99B01AC01C50120
:10E99000B4010E94F9D94B015C01C01BD10BBE012F
:10E9A000DD0F880B990B0E949AD99B01AC01C50120
:10E9B000B4010E94BCDE4B015C01B701FF0C880B67
:10E9C000990B0E949AD99B01AC01C501B4010E9428
:10E9D000E0DDDF91CF911F910F91FF90EF90DF90DD
:10E9E000CF90BF90AF909F908F9008950F931F93FB
:10E9F000CF93DF93CDB7DEB728970FB6F894DEBF7D
:10EA00000FBECDBF60914A0470914B04072E000CDD
:10EA1000880B990B0E949AD96D837E838F83988788
:10EA200080914C0490914D04A0914E04B0914F04FC
:10EA300089839A83AB83BC834DEFBE016B5F7F4FAD
:10EA4000CE0101960EDF6091440470914504072EBB
:10EA5000000C880B990B0E949AD96D837E838F835B
:10EA600098878091460490914704A0914804B09102
:10EA7000490489839A83AB83BC834FEFBE016B5FEC
:10EA80007F4FCE010196EDDEE4E4FEE184918F013B
:10EA90000F5F1F4F882321F00E9488C5F801F6CF31
:10EAA000E091DB14F0E0E752FB4E608170E080E023
:10EAB00090E00E94FAC5EFE3FEE184918F010F5FC1
:10EAC0001F4F882321F00E9488C5F801F6CF60917E
:10EAD000DA1470E080E090E00E94FAC528960FB644
:10EAE000F894DEBF0FBECDBFDF91CF911F910F9184
:10EAF00008950F930FB70F9300916E000B7F009353
:10EB00006E0078940F930BB70F930CB70F921F9270
:10EB10002F933F934F935F936F937F938F939F9325
:10EB2000AF93BF93EF93FF931124DAD2FF91EF914C
:10EB3000BF91AF919F918F917F916F915F914F9115
:10EB40003F912F911F900F900CBF0F910BBF0F9112
:10EB50000460F89400936E000F910FBF0F91189509
:10EB6000CF92DF92EF92FF92C0904604D09047047C
:10EB7000E0904804F0904904609144047091450489
:10EB800066507109072E000C880B990B0E949AD9C8
:10EB90009B01AC01C701B6010E9494D987FF1FC039
:10EBA00020E030E040E050E4C701B6010E94E0DD23
:10EBB0000E9429DF70931315609312150E94A551CE
:10EBC000DC01CB01805A9541AF4FBF4F80930E15AA
:10EBD00090930F15A0931015B093111508C01092C3
:10EBE0000E1510920F151092101510921115FF901E
:10EBF000EF90DF90CF900895CF92DF92EF92FF9247
:10EC0000C0904C04D0904D04E0904E04F0904F041E
:10EC100060914A0470914B0469507109072E000CF1
:10EC2000880B990B0E949AD99B01AC01C701B601D0
:10EC30000E9494D987FF1FC020E030E040EA50E4F2
:10EC4000C701B6010E94E0DD0E9429DF70930D1517
:10EC500060930C150E94A551DC01CB0188549747A5
:10EC6000AF4FBF4F8093081590930915A0930A15D5
:10EC7000B0930B1508C01092081510920915109248
:10EC80000A1510920B15FF90EF90DF90CF9008952A
:10EC90008F929F92AF92BF92CF92DF92EF92FF92AC
:10ECA0000F931F93CF93DF93F0E4FF2EE12CAE2D53
:10ECB000B0E0BD016F0D711D759567956E1511F072
:10ECC000F6120BC0E1E9FDE165917491072E000C8D
:10ECD000880B990B0E949AD962C09B01215031097F
:10ECE000220F331F220F331FF901ED56F34E05910A
:10ECF0001491AB01440F551F440F551FFA01ED56F7
:10ED0000F34EC591D4918017910714F4F62ED1CF0C
:10ED1000C817D90714F4E62ECACFF901EB56F34E03
:10ED2000E590F490FA01EB56F34EC590D490BC01F7
:10ED3000601B710B072E000C880B990B0E949AD94F
:10ED40004B015C01B6016E197F09072E000C880B80
:10ED5000990B0E949AD99B01AC01C501B4010E9494
:10ED6000F9D94B015C01C01BD10BBE01DD0F880B33
:10ED7000990B0E949AD99B01AC01C501B4010E9474
:10ED8000BCDE4B015C01B701FF0C880B990B0E94A4
:10ED90009AD99B01AC01C501B4010E94E0DDDF916D
:10EDA000CF911F910F91FF90EF90DF90CF90BF9088
:10EDB000AF909F908F90089560E080911E15909184
:10EDC0001F1580DD60934C0470934D0480934E04B6
:10EDD00090934F0480911C1590911D1559DF6093FD
:10EDE0004604709347048093480490934904A8957F
:10EDF0001092D61408957F928F929F92AF92BF92F5
:10EE0000CF92DF92EF92FF920F931F93CF93DF93F6
:10EE100020E030E048E452E460914C0470914D04ED
:10EE200080914E0490914F040E9406E018164CF415
:10EE3000E7E2FCE1E491C1E001C0CC0FEA95EAF71A
:10EE400001C0C0E081E2E82E8CE1F82E07E21CE16F
:10EE500096E0A92E912CD0E0CC24C394D12CF701BC
:10EE60007490F801849077FC23C0892D90E0082CE1
:10EE700002C0959587950A94E2F780FD19C0BE01FE
:10EE8000082C02C0759567950A94E2F76170B62E5A
:10EE9000B1946B2D872D0E9403A96B2D70E0872DF7
:10EEA0000E946DA9C60101C0880F8A94EAF7982ACA
:10EEB000AA94FFEFEF1AFF0A0F5F1F4FA110CFCFE9
:10EEC000DF91CF911F910F91FF90EF90DF90CF9046
:10EED000BF90AF909F908F907F9008950F931F9356
:10EEE0008091B814813019F40E94A55108C0609136
:10EEF000B4147091B5148091B6149091B714009128
:10EF0000E0141091E1142091E2143091E314601B9D
:10EF1000710B820B930B28EE33E040E050E00E942F
:10EF200082DD8091DC149091DD14A091DE14B0910B
:10EF3000DF14BC01CD01620F731F841F951F1F9149
:10EF40000F9108951092B8141092E0141092E114E9
:10EF50001092E2141092E3141092B4141092B514AB
:10EF60001092B6141092B7141092DC141092DD14A3
:10EF70001092DE141092DF1408958091B81481303D
:10EF8000E1F0823051F4AADF6093DC147093DD1459
:10EF90008093DE149093DF1401C0D4DF81E080936E
:10EFA000B8140E94A5516093E0147093E11480930B
:10EFB000E2149093E31481E0089580E00895809135
:10EFC000B8148150823010F080E008951092B81487
:10EFD0000E94A5516093B4147093B5148093B61435
:10EFE0009093B71481E008951092D51480E090E0DA
:10EFF0000E949A521092450410924404B1DDDFDF62
:10F0000080E090E00E949A521092D9142C981092AD
:10F010004504109244041092DA1480910201807227
:10F02000809300010895DF92EF92FF920F931F9358
:10F03000CF93DF93F82ED62EE72E8A0180913302EC
:10F04000882309F439C0E6E8FBE18491EF012196B9
:10F05000882321F00E9488C5FE01F7CFED2DFE2DFB
:10F060008491EF012196882321F00E9488C5FE013A
:10F07000F7CFE2E3FCE18491EF012196882321F0B0
:10F080000E9488C5FE01F7CFF7FC0BC06F2DFF0C67
:10F09000770B880B990B0E94FAC58AE00E9488C5FD
:10F0A0000BC0EDE2FCE18491EF012196882321F071
:10F0B0000E9488C5FE01F7CF8091E414811108C039
:10F0C0001092330281E08093E414C8010E94C29B35
:10F0D000DF91CF911F910F91FF90EF90DF9084CF40
:10F0E000EF92FF920F931F93CF93DF93809136029D
:10F0F0008F37A0F08F579091D91490932F159923A3
:10F1000011F02C9A01C02C982091DA1420932E151E
:10F1100090910201222369F090950BC090912F15D8
:10F12000891708F02C9890912E15891728F0909146
:10F1300002019072909300018F5F8093360290914C
:10F140002D1581E0892780932D158091350285301A
:10F150001CF4C1E0C80F01C0C0E0823009F4B4C0A3
:10F1600054F4882301F1813009F0E3C088E08093F2
:10F170007B0085E4C0C0843009F4C5C00CF4B7C07E
:10F18000853009F0D6C090912C15911102C0809362
:10F190002C1580912C15815080932C15882309F40F
:10F1A000C8C0C5E0C6C0809134028F5F80311CF4B6
:10F1B00080933402BEC0109234028091D614811123
:10F1C00013C0809122159091231590931F15809361
:10F1D0001E15809120159091211590931D158093F7
:10F1E0001C1581E08093D6148AE0E2E2F5E1DF01AC
:10F1F0001D928A95E9F71092211510922015009121
:10F200001E1510911F1511950195110980914A0441
:10F2100090914B04D1E0181619062CF08091D91466
:10F22000811101C0D0E08091A40A9091A50A919526
:10F23000819591098017910734F44AEC5DE16BEEFA
:10F240007DE180E0F0DE8091280290912902919585
:10F25000819591090817190744F4DD2331F04DEF2A
:10F260005DE16EE17EE180E0DEDE8091440490911C
:10F27000450411E0181619062CF08091DA1481115A
:10F2800001C010E0E0901C15F0901D158091A20ABD
:10F290009091A30A8E159F0534F04AED5DE16BEE67
:10F2A0007DE18FEFC0DE8091260290912702E81663
:10F2B000F9060CF43EC01123E1F14DE05EE16EE190
:10F2C0007EE18FEFB0DE35C080917A0086FD2EC0E2
:10F2D000809178009091790020912215309123152A
:10F2E000820F931F909323158093221522C088E0EC
:10F2F00080937B0086E480937C0080917A00806418
:10F3000080937A0016C080917A0086FD11C08091AA
:10F310007800909179002091201530912115820F6D
:10F32000931F909321158093201503C0C2E001C064
:10F33000C4E0C09335028091A90A81110E94E3B50F
:10F340008091D7149091D8140097A9F001979093C9
:10F35000D8148093D714892B71F480E39EE19093A5
:10F360008B0C80938A0CDF91CF911F910F91FF90AE
:10F37000EF900C945E8BDF91CF911F910F91FF90D6
:10F38000EF9008952F923F924F925F926F927F92EB
:10F390008F929F92AF92BF92CF92DF92EF92FF92A5
:10F3A0000F931F93CF93DF9300D01F92CDB7DEB79B
:10F3B0005C017A8369834A01170107FD07C0802F2A
:10F3C000002E000C990B9C838B8304C0E1E0F0E0DD
:10F3D000FC83EB83F90140805180628073808B81D4
:10F3E0009C81880F991F880F991F9C838B838C5E4B
:10F3F0009A4E7C01A3019201FC016081718182819E
:10F4000093810E9494D9882391F0F7014082518220
:10F410006282738211E020E030E0A901C301B201F1
:10F420000E9406E018160CF010E0F5011083F501BB
:10F4300080818230D1F0833009F45EC0813009F0E0
:10F440007CC0EB81FC81EC5EFA4E208131814281EF
:10F450005381F40160817181828193810E9494D9EA
:10F4600087FD6BC082E0F50180838B819C818C5E7F
:10F470009A4E9C838B83B60180E090E00E9498D9DD
:10F480009B01AC01EB81FC81608171818281938160
:10F490000E94DFDD9B01AC01F401608171818281FA
:10F4A00093810E9406E087FD14C00E94A5516B0164
:10F4B0007C019101A8EEB3E00E94D0DDC60ED71EFC
:10F4C000E81EF91EE981FA81C082D182E282F382CC
:10F4D00034C00E94A551E981FA81C080D180E280C8
:10F4E000F380DC01CB018C199D09AE09BF09B7FD82
:10F4F00024C083E0F50180830F3F19F043E95DE10B
:10F5000002C046EA5DE16AEB7DE1802F0F900F902B
:10F510000F900F90DF91CF911F910F91FF90EF907F
:10F52000DF90CF90BF90AF909F908F907F906F9023
:10F530005F904F903F902F9076CD0F900F900F904F
:10F540000F90DF91CF911F910F91FF90EF90DF907F
:10F55000CF90BF90AF909F908F907F906F905F9073
:10F560004F903F902F9008954F925F926F927F92AD
:10F570008F929F92AF92BF92CF92DF92EF92FF92C3
:10F580000F931F93CF93DF93CDB7DEB760970FB67E
:10F59000F894DEBF0FBECDBF8091D614811117C085
:10F5A00060960FB6F894DEBF0FBECDBFDF91CF914E
:10F5B0001F910F91FF90EF90DF90CF90BF90AF9091
:10F5C0009F908F907F906F905F904F900895F4DBA5
:10F5D0000E94A5514B015C0160914A0470914B045B
:10F5E000072E000C880B990B0E949AD969837A83A5
:10F5F0008B839C8344E1C42ED12C5CE3E52EF12C5B
:10F6000000E09E012F5F3F4F4CE454E064E075E161
:10F6100083E095E1B7DEC0904C04D0904D04E090BB
:10F620004E04F0904F046091A60A7091A70A072E2D
:10F63000000C880B990B0E949AD99B01AC01C70161
:10F64000B6010E9406E018160CF009C160912A026A
:10F6500070912B02072E000C880B990B0E949AD9EF
:10F660009B01AC01C701B6010E9494D987FFF7C086
:10F6700000914A0410914B04B801012E000C880B34
:10F68000990B0E949AD9A70196010E94DFDD2B01F8
:10F690003C0120ED3CEC4CE45DE36091CD147091B5
:10F6A000CE148091CF149091D0140E94F9D96D831B
:10F6B0007E838F8398872091FA143091FB144091B8
:10F6C000FC145091FD14C701B6010E94DFDD9B01BF
:10F6D000AC016D817E818F8198850E94F9D96D83FF
:10F6E0007E838F83988723E333E343E75FE360916F
:10F6F000F6147091F7148091F8149091F9140E9407
:10F70000F9D99B01AC016D817E818F8198850E9422
:10F71000E0DD6D837E838F8398876093F61470930A
:10F72000F7148093F8149093F914C092FA14D092BD
:10F73000FB14E092FC14F092FD1420E030E040E273
:10F7400051E4C301B2010E9406E018160CF431C264
:10F7500020E030E040E251ECC301B2010E9494D9B4
:10F7600087FD2FC2012B09F42CC28091F514811161
:10F770002CC22091F1143091F2144091F314509165
:10F78000F41429873A874B875C872091C9143091FC
:10F79000CA144091CB145091CC14C301B2010E9401
:10F7A000F9D96B017C01A301920169857A858B856A
:10F7B0009C850E94E0DD69877A878B879C876093B0
:10F7C000F1147093F2148093F3149093F414209135
:10F7D000C5143091C6144091C7145091C8140E94AA
:10F7E000F9D9A70196010E94E0DD2D813E814F816C
:10F7F00058850E94DFDD6B017C0120E030E04FE79F
:10F8000053E40E9406E020E030E0A90118160CF451
:10F81000E3C1C701B6010E9494D987FD07C0C701A3
:10F82000B6010E9424DF759567951AC020E030E08C
:10F83000A901C301B2010E9494D987FF10C0A3019E
:10F84000920169857A858B859C850E94DFDD6093B6
:10F85000F1147093F2148093F3149093F41460E015
:10F860006093D9148091081590910915A0910A15FB
:10F87000B0910B150097A105B10521F1A5019401E7
:10F88000281B390B4A0B5B0B57FD1CC060910C15F4
:10F8900070910D1580E090E00E9498D99B01AC0119
:10F8A00060914C0470914D0480914E0490914F04EE
:10F8B0000E9494D987FF82C142E75CE164E87CE161
:10F8C00080E0B1DB8091D1149091D214A091D31437
:10F8D000B091D414A5019401281B390B4A0B5B0B82
:10F8E00057FD0FC088DAD501C4018C53964FAF4F36
:10F8F000BF4F8093D1149093D214A093D314B0939C
:10F90000D41480910E1590910F15A0911015B091FF
:10F9100011150097A105B10511F1881A990AAA0AD3
:10F92000BB0AB7FC1CC0609112157091131580E0E2
:10F9300090E00E9498D99B01AC01609146047091BF
:10F94000470480914804909149040E9494D987FF0C
:10F9500020C140E55CE163E67CE18FEF64DB609110
:10F96000440470914504072E000C880B990B0E94EB
:10F970009AD969837A838B839C8395E0C92ED12C95
:10F9800024E1E22EF12C0FEF9E012F5F3F4F46E462
:10F9900054E06EEF74E182E095E1F4DCC09046043F
:10F9A000D0904704E0904804F090490420E030E013
:10F9B00040EA50E4C701B6010E9406E087FDE5C0B9
:10F9C00020E030E04CED52E4C701B6010E9494D92A
:10F9D00018160CF4DAC06091440470914504072EA7
:10F9E000000C880B990B0E949AD9A70196010E94DE
:10F9F000DFDD4B015C012091C1143091C2144091B4
:10FA0000C3145091C4140E94F9D969877A878B87EF
:10FA10009C872091ED143091EE144091EF14509199
:10FA2000F014C501B4010E94E0DD6D837E838F83F5
:10FA300098876093ED147093EE148093EF14909375
:10FA4000F0142091BD143091BE144091BF14509118
:10FA5000C0140E94F9D96D877E878F87988B20ED1F
:10FA60003CEC4CE45DE36091B9147091BA14809160
:10FA7000BB149091BC140E94F9D92B013C01209138
:10FA8000E9143091EA144091EB145091EC14C70141
:10FA9000B6010E94DFDD9B01AC01C301B2010E94EF
:10FAA000F9D92B013C0123E333E343E75FE36091A2
:10FAB000E5147091E6148091E7149091E8140E9487
:10FAC000F9D99B01AC01C301B2010E94E0DD2B0119
:10FAD0003C016093E5147093E6148093E7149093CF
:10FAE000E814C092E914D092EA14E092EB14F09278
:10FAF000EC142D853E854F85588969857A858B85DF
:10FB00009C850E94E0DDA30192010E94DFDD6B0174
:10FB10007C0120E030E04FE753E40E9406E020E063
:10FB200030E0A9011816C4F5C501B4010E9406E031
:10FB3000181684F4A50194016D817E818F819885CA
:10FB40000E94DFDD6093ED147093EE148093EF1448
:10FB50009093F0146FE71AC020E030E0A901C501CE
:10FB6000B4010E9494D987FF10C0A50194016D8152
:10FB70007E818F8198850E94DFDD6093ED14709304
:10FB8000EE148093EF149093F01460E06093DA1415
:10FB900007CD0E94B075E3CEC701B6010E9494D98B
:10FBA00087FDDACFC701B6010E9424DF75956795FE
:10FBB000EDCF81E08093F5146FE752CE80E01CD842
:10FBC00081CE81E08093F5144ACE1092F514198607
:10FBD0001A861B861C86D9CDC301B2010E9406E09D
:10FBE000181654F7A301920169857A858B859C8547
:10FBF0000E94DFDD6093F1147093F2148093F3148C
:10FC00009093F4146FE72CCE90916F00292F2270FF
:10FC100091FF05C090916F009D7F90936F0034E03D
:10FC2000839FC0011124FC01E951FA4E40815181AA
:10FC300062817381FC01E855FB4E408351836283EE
:10FC4000738381E08093A714222329F080916F00B1
:10FC5000826080936F000895BC012091A5143091BB
:10FC6000A6144091A5145091A6142417350711F03D
:10FC70009A01F7CF81E02617370709F080E0089551
:10FC8000CF92DF92EF92FF920F931F93CF93DF9368
:10FC900088E50E94DB3AD82E89E40E94DB3AC82E20
:10FCA000882319F00E94743A1CC0DD20C1F00E9424
:10FCB000A43A20E030E040E251E40E94DFDD20E0A1
:10FCC00030E04CEB51E40E94E0DD21E43CE44EEAFC
:10FCD0005CE30E94F9D90E9424DF653010F01FEF29
:10FCE00001C0162F89E50E94DB3A082F8AE40E94A2
:10FCF000DB3AC82F882319F00E94743A1CC00023F5
:10FD0000C1F00E94A43A20E030E040E251E40E94B9
:10FD1000DFDD20E030E04CEB51E40E94E0DD21E447
:10FD20003CE44EEA5CE30E94F9D90E9424DF65308E
:10FD300010F0DFEF01C0D62F8AE50E94DB3AE82EF3
:10FD4000811105C081E50E94DB3AF82E01C0F12C3B
:10FD5000C11001C0C0E02C2F30E0D11001C000E084
:10FD6000200F311D2130310521F4E1101AC0F110AE
:10FD700018C0E6E8FBE18491EF012196811103C0F0
:10FD8000E7ECF0E204C00E9488C5FE01F4CF849144
:10FD9000EF012196882309F455C00E9488C5FE0111
:10FDA000F6CF17FD02C0D7FF17C0E6E8FBE184914C
:10FDB000EF012196811103C0E8EAF0E204C00E943D
:10FDC00088C5FE01F4CF8491EF0121968823D1F1FB
:10FDD0000E9488C5FE01F7CF0E94A43A9B01AC01A6
:10FDE000012F110F110BAD2FDD0FBB0BFF2099F071
:10FDF00085E0809FF001819FF00D1124EA0FFB1F29
:10FE0000EE0FFF1FEE0FFF1FED5CF94E6081718159
:10FE10008281938103C060E070E0CB01E5E0E09F68
:10FE2000E001E19FD00D1124CA0FDB1FCC0FDD1FB5
:10FE3000CC0FDD1FCD5CD94E0E94E0DD6883798355
:10FE40008A839B83DF91CF911F910F91FF90EF9059
:10FE5000DF90CF90089580916F00982F927081FF6E
:10FE600005C080916F008D7F80936F0080919B0E05
:10FE700080939A0E8093990E8093980E84E68093D7
:10FE8000970E28EE33E03093D8142093D71499239B
:10FE900029F080916F00826080936F0081E08093F1
:10FEA000A7140E94C4620E94FABF8091E1158823C2
:10FEB00021F085E497E10E94F4508CE0E5E4F7E15D
:10FEC000A2E3B4E001900D928A95E1F70C94518E73
:10FED0002F923F924F925F926F927F928F929F925A
:10FEE000AF92BF92CF92DF92EF92FF920F931F9348
:10FEF000CF93DF93CDB7DEB7CD54D1090FB6F894C9
:10FF0000DEBF0FBECDBF85E40E94243B882321F0D5
:10FF10000E94743A7B0102C0E12CF12C83E40E9420
:10FF2000243B882321F00E94743A6AA302C005E0B2
:10FF30000AA385E50E94243B882319F00E94953A84
:10FF400003C085E50E94DB3A8CA7F7FC07C0812C33
:10FF5000912C16E1A12E13E4B12E06C0812C912C18
:10FF6000BCE8AB2EB2E4BB2E83E50E94243B882381
:10FF700021F00E94A43A4B015C01E114F10411F458
:10FF80001092DB1410929E15ED820E94A5512B0158
:10FF90003C011D8117FF05C00CE310E022E029831E
:10FFA00004C003E210E035E03983D301C2018C5371
:10FFB000964FAF4FBF4F8093D1149093D214A0931C
:10FFC000D314B093D41461E06E0D623080F0E5E19B
:10FFD000F0E284918F010F5F1F4F1A8309838823FA
:10FFE00009F45FC30E9488C5E981FA81F2CFEFE38B
:10FFF000F0E284917F012FEFE21AF20A882321F0C8
:020000021000EC
:100000000E9488C5F701F5CF0E94F4773D8137FF44
:1000100004C08FE78093DA1408C04D81E42F440FA9
:10002000FF0BE752FB4E8FE78083C501B4010E94AE
:1000300024DF072E000C880B990B0E949AD96A873F
:100040007B878C879D878981482F50E09801A8EE97
:10005000B3E00E94D0DD6DA77EA78FA798AB8B0180
:100060009C01040D151D261D371D0AAF1BAF2CAFBB
:100070003DAF81E080932C021D811F3F39F40FE7D3
:100080001FE11FAF0EAF09E41FE106C00DE61FE13F
:100090001FAF0EAF06E31FE122961FAF0EAF2297F0
:1000A0004CA25DA26EA27FA249AA5AAA6BAA7CAA00
:1000B0001DAA1EAA1FAA18AE19AE188E10E4198F19
:1000C0000CE10A8F16E41B8F1C8E1D8E1E8E1F8E58
:1000D0001C8A1D8A1E8A1F8A188A198A1A8A1B8AF4
:1000E00019821A821B821C828FE790E0A0E0B0E0A8
:1000F0008E839F83A887B987FFE7CF2ED12CE12C71
:10010000F12C18A619A61AA61BA611E01F861E869A
:100110002D961FAE2D97212C312C2E961FAE2E978B
:100120000D81802F000F990B9C0127523B4E249686
:100130003FAF2EAF2497880F991F880F991FDC01BE
:10014000A45BBB4FB9A3A8A3CA01052E000CAA0B40
:10015000BB0B28968CAF9DAFAEAFBFAF28974C5F5F
:100160005F4FCA01550FAA0BBB0B2C968CAF9DAFEE
:10017000AEAFBFAF2C97AAA10A2E000CBB0BBBA33E
:10018000AAA380912C02882309F489C20E94A55158
:100190004B015C018091D614882309F4D4C00E94DD
:1001A000DC760D8107FD0CC0A8A1B9A1BC912D96EC
:1001B000BFAF2D97E8A1F9A12180328003810BC048
:1001C000009146042D960FAF2D9720904704309054
:1001D0004804009149042E960FAF2E972D962FAD0F
:1001E0002D97322D432D2E965FAD2E976C8D7D8DE4
:1001F0008E8D9F8D0E9494D987FF0AC02D960FADDA
:100200002D970C8F2D8E3E8E2E960FAD2E970F8F25
:10021000288D398D4A8D5B8D2D966FAD2D97722D62
:10022000832D2E969FAD2E970E9494D987FF0AC0EA
:100230002D960FAD2D97088F298E3A8E2E960FADE5
:100240002E970B8F8091D1149091D214A091D3143A
:10025000B091D414A5019401281B390B4A0B5B0BF8
:1002600057FD10C00E94FB76D501C4018C53964FF8
:10027000AF4FBF4F8093D1149093D214A093D31457
:10028000B093D4142D962FAD2D97322D432D2E964D
:100290005FAD2E976A857B858C859D851123E9F15D
:1002A0000E9494D987FF4FC0B501A4014419550994
:1002B00066097709DB01CA0188589341A109B10990
:1002C000B7FD41C0D701C6010E811F812885398540
:1002D000801B910BA20BB30B1D81B595A79597952C
:1002E000879517FF03C08093DA1405C02496EEADFE
:1002F000FFAD2497808348A759A76AA77BA70A85E3
:100300000C8F1B851D8F0C850E8F1D851F8F8CA25A
:100310009DA2AEA2BFA210E016C00E9406E0181671
:1003200094F4D501C4012CA13DA14EA15FA1821B73
:10033000930BA40BB50BAC01BD01485853416109A7
:10034000710977FFCBC120E030E040EA51E46A85D3
:100350007B858C859D850E94E0DD2D962FAD2D97A8
:10036000322D432D2E965FAD2E970E9494D987FF94
:1003700010C0E1EAFFE184918F010F5F1F4F1A83E4
:100380000983882309F48BC10E9488C5E981FA8119
:10039000F2CFD501C40129A93AA94BA95CA9821BB6
:1003A000930BA40BB50BB7FD96C00E94F6748AE0C0
:1003B0000E9488C5D501C4018053984FAF4FBF4FED
:1003C00089AB9AABABABBCAB0DA9011163C02EA935
:1003D0003FA948AD59AD2D966FAD2D97722D832D48
:1003E0002E969FAD2E970E9406E018160CF041C085
:1003F00028966CAD7DAD8EAD9FAD28970E949AD9A1
:100400002D962FAD2D97322D432D2E965FAD2E9725
:100410000E94E0DD6EAB7FAB88AF99AF2DA53EA506
:100420004FA558A9280D391D4A1D5B1D2AAF3BAFAA
:100430004CAF5DAF2C966CAD7DAD8EAD9FAD2C9766
:100440000E949AD99B01AC016A857B858C859D852C
:100450000E94DFDD2D962FAD2D97322D432D2E9648
:100460005FAD2E970E9494D9881F8827881F8DAB77
:1004700032C0D501C4012AAD3BAD4CAD5DAD821B90
:10048000930BA40BB50BB7FD26C04EAD5FAD62E973
:100490007FE11EC020E030E040EA51E46A857B85C0
:1004A0008C859D850E94DFDD9B01AC012D966FAD93
:1004B0002D97722D832D2E969FAD2E970E9494D945
:1004C00087FF09C022964EAD5FAD22976DE57FE1B3
:1004D0008D810E941378D501C401880F991FAA1F2E
:1004E000BB1F2CA13DA14EA15FA1821B930BA40BAE
:1004F000B50B84199509A609B70981389F44A24113
:10050000B10580F0E8E1FFE184918F010F5F1F4F9B
:100510001A830983882309F4C2C00E9488C5E9812F
:10052000FA81F2CF2AA13BA14E855F8524173507BA
:100530000CF027CEEBEBFEE184918F010F5F1F4F94
:100540001F830E83882329F00E9488C5EE81FF81D6
:10055000F3CF1D8117FD03C006E113E002C000EFD9
:1005600013E01F830E836E817F818AEA9EE10E94E1
:10057000D95049815A816B817C8186EA9EE10E9433
:10058000A3508AE00E9488C56E817F8185E99EE143
:100590000E94D950488959896A897B8981E99EE1FD
:1005A0000E94A3508AE00E9488C56E817F8180E806
:1005B0009EE10E94D9504C895D896E897F898CE7C4
:1005C0009EE10E94A3508AE00E9488C51CA51123C9
:1005D00009F467C00D8107FF31C029813A814B8141
:1005E0005C812093C1143093C2144093C314509380
:1005F000C4142CEA35EC47E25EE3688979898A897C
:100600009B890E94F9D96093BD147093BE148093A6
:10061000BF149093C0142CEA35EC47E25EE36C897A
:100620007D898E899F890E94BCDE6093B914709386
:10063000BA148093BB149093BC1433C089819A81FF
:10064000AB81BC818093C9149093CA14A093CB143E
:10065000B093CC142CEA35EC47E25EE368897989E3
:100660008A899B890E94F9D96093C5147093C61436
:100670008093C7149093C8142CEA35EC47E25EE3EC
:100680006C897D898E899F890E94BCDE6093CD1420
:100690007093CE148093CF149093D01402C00E9414
:1006A000F47781E080939E15C35BDF4F0FB6F8941B
:1006B000DEBF0FBECDBFDF91CF911F910F91FF9095
:1006C000EF90DF90CF90BF90AF909F908F907F90F2
:1006D0006F905F904F903F902F9008950E851F85EB
:1006E000012B09F42DC148A459A46AA47BA4480E87
:1006F000591E6A1E7B1E28A539A54AA55BA5281B85
:10070000390B4A0B5B0B6E817F81888599850E942E
:1007100073DDA30192010E94A4DDDA01C9018C0DF1
:100720009D1DAE1DBF1D84319105A105B105FCF0D5
:100730006C017D018C3E9105A105B1052CF05BEEAD
:10074000C52ED12CE12CF12C20E8C216D104E104F5
:10075000F104DCF08EEF90E0A0E0B0E08C199D0990
:10076000AE09BF098E839F83A887B98712C044E171
:10077000C42ED12CE12CF12C04E110E020E030E07B
:100780000E831F832887398704C0CE82DF82E886E4
:10079000F986EDE0F0E284918F010F5F1F4F88230F
:1007A00021F00E9488C5F801F6CFC701B6010E946A
:1007B000FAC5E8E0F0E284918F010F5F1F4F8823B4
:1007C00021F00E9488C5F801F6CF6E817F8188856F
:1007D00099850E94FAC5488D598D6A8D7B8D81E07F
:1007E00090E20E94A3504C8D5D8D6E8D7F8D8AEFBF
:1007F0009FE10E94A3500E851F85033011050CF464
:100800009FC06E817F81888599850E949AD920E05A
:1008100030E040E850E40E94F9D969837A838B8301
:100820009C83288D398D4A8D5B8D6C8D7D8D8E8D51
:100830009F8D0E94DFDD2BED3FE049E450E40E94F4
:10084000F9D920E030E040E05FE30E94F9D99B0154
:10085000AC0169817A818B819C810E94BCDE6983B5
:100860007A838B839C83C301B2010E949AD92FE6BD
:1008700032E143E85AE30E94F9D92B013C01498156
:100880005A816B817C8184EF9FE10E94A350B30168
:10089000A2018EEE9FE10E94A3502AE939E949E1C5
:1008A0005FE369817A818B819C810E94F9D9698398
:1008B0007A838B839C839B01AC010E94E0DDA301C2
:1008C00092010E94BCDE688B798B8A8B9B8B29817D
:1008D0003A814B815C81C301B2010E94F9D920E0C9
:1008E00030E040E05EE30E94F9D96C8B7D8B8E8B0B
:1008F0009F8BEEEDFFE184918F010F5F1F4F8823E7
:1009000021F00E9488C5F801F6CF49815A816B8198
:100910007C8188ED9FE10E94A350488959896A89AA
:100920007B8982ED9FE10E94A3504C895D896E898D
:100930007F898CEC9FE10E94A3508AE00E9488C5C9
:100940008E819F81A885B9858C0D9D1DAE1DBF1D13
:100950001D81B595A7959795879517FF03C080933F
:10096000DA1405C02496EEADFFAD249780830E8582
:100970001F850F5F1F4F1F870E871A85188F0B85E6
:10098000098F1C851A8F0D850B8F2401350111E00D
:10099000DACCFF920F931F93CF93DF93F82E092F9A
:1009A000162FE7E7FEE18491EF012196882321F0DD
:1009B0000E9488C5FE01F7CFEF2DF02F8491EF0143
:1009C0002196882321F00E9488C5FE01F7CFE5E734
:1009D000FEE18491EF012196882321F00E9488C5D1
:1009E000FE01F7CF612F70E080E090E00E94FAC531
:1009F0008AE0DF91CF911F910F91FF900C9488C5F1
:100A00004F925F926F927F928F929F92AF92BF921E
:100A1000CF92DF92EF92FF92CF93DF932091170452
:100A2000309118044091190450911A0460913204D5
:100A30007091330480913404909135040E94E0DD7C
:100A4000AB01BC0182E79EE10E94A35020911B04F0
:100A500030911C0440911D0450911E046091360495
:100A60007091370480913804909139040E94E0DD40
:100A7000AB01BC018EE69EE10E94A35020911F04B1
:100A800030912004409121045091220460913A0455
:100A900070913B0480913C0490913D040E94E0DD04
:100AA000AB01BC018AE69EE10E94A35040913E0446
:100AB00050913F04609140047091410486E69EE1AC
:100AC0000E94A35080916F00982F927081FF05C003
:100AD00080916F008D7F80936F004090E71550905C
:100AE000E8156090E9157090EA158090EB159090EC
:100AF000EC15A090ED15B090EE15C090EF15D090CC
:100B0000F015E090F115F090F215992329F08091FD
:100B10006F00826080936F00ECE5FEE18491EF014D
:100B20002196882321F00E9488C5FE01F7CFC301DA
:100B3000B2010E94FAC5E8E5FEE18491EF01219639
:100B4000882321F00E9488C5FE01F7CFC501B401BA
:100B50000E94FAC5E4E5FEE18491EF012196882325
:100B600021F00E9488C5FE01F7CFC701B6010E949F
:100B7000FAC58AE0DF91CF91FF90EF90DF90CF90A0
:100B8000BF90AF909F908F907F906F905F904F90AD
:100B90000C9488C52F923F924F925F926F927F92F2
:100BA0008F929F92AF92BF92CF92DF92EF92FF927D
:100BB0000F931F93CF93DF93CDB7DEB761970FB637
:100BC000F894DEBF0FBECDBF83E50E94DB3A8823D9
:100BD00041F00E94953A182F811105C080E04DD454
:100BE00002C01091E1158091320490913304A091DC
:100BF0003404B091350489839A83AB83BC8380919C
:100C0000360490913704A0913804B09139048D8353
:100C10009E83AF83B88780913A0490913B04A09162
:100C20003C04B0913D0489879A87AB87BC87F8D391
:100C3000882309F499C083E40E94DB3A882309F4ED
:100C400093C00E94A43A1B012C0105E0612C712C79
:100C500038EC388B82EC898BA12CB12C98EC9E87D8
:100C6000E2E4EF87015080F125E02D87209F4001CD
:100C700011243D8531503D873F3FA1F3F401E30F3F
:100C8000F11DEE0FFF1FEE0FFF1FED5CF94EC08050
:100C9000D180E280F3809601A701B5018E859F8502
:100CA0000E9406E018161CF45601EE86FF86960197
:100CB000A701B301888999890E9494D987FFD9CF68
:100CC0003601E88AF98AD5CF930148895989B50157
:100CD0008E859F850E94E0DD20E030E040E05FE30C
:100CE0000E94F9D9A20191010E94E0DD2B013C0193
:100CF0002DEB37E346E855EB0E9406E087FD0AC07E
:100D00002DEB37E346E855E3C301B2010E9494D9C5
:100D1000181654F580E0B1D335E0D32E45E0C42E4B
:100D2000DA949FEFD91601F105E0CD9C5001112412
:100D30000150B0F37501E00EF11CC701880F991F37
:100D4000880F991FFC01ED5CF94E7F01A301920110
:100D500060817181828193810E94DFDDF701608370
:100D6000718382839383E4CF86E50E94DB3A8823F4
:100D700091F056D3882379F0E2E9F0E284917F0183
:100D80002FEFE21AF20A882321F00E9488C5F701AA
:100D9000F5CF0E9420B58AE50E94DB3A882321F036
:100DA0000E94A43A0E94F5A7812F67D3111103C0B6
:100DB000EBE9FBE11CC08091E1158111F9CFE6E878
:100DC000FBE184918F010F5F1F4F882321F00E9468
:100DD00088C5F801F6CFE3E7F0E284918F010F5F59
:100DE0001F4F882329F30E9488C5F801F6CF84910C
:100DF0008F010F5F1F4F882321F00E9488C5F801E3
:100E0000F6CF8091E115811103C067E173E002C064
:100E100063E173E085E690E20E94D9508AE00E9487
:100E200088C5EBE9FBE184918F010F5F1F4F882399
:100E300021F00E9488C5F801F6CFE8E5F0E2849140
:100E40008F010F5F1F4F882321F00E9488C5F80192
:100E5000F6CFC090E215D090E315E090E415F09045
:100E6000E51520E030E0A901C701B6010E9406E0C7
:100E700018164CF442E0C701B6010E9414C68AE07D
:100E80000E9488C50CC0E3E5F0E284918F010F5FFA
:100E90001F4F882321F00E9488C5F801F6CF4CE04F
:100EA00050E062E374E0CE0101960E94FCE0892BE1
:100EB000C9F061960FB6F894DEBF0FBECDBFDF91CB
:100EC000CF911F910F91FF90EF90DF90CF90BF9047
:100ED000AF909F908F907F906F905F904F903F90DA
:100EE0002F908ECD61960FB6F894DEBF0FBECDBFAA
:100EF000DF91CF911F910F91FF90EF90DF90CF90F6
:100F0000BF90AF909F908F907F906F905F904F9029
:100F10003F902F9008952F923F924F925F926F9241
:100F20007F928F929F92AF92BF92CF92DF92EF9279
:100F3000FF920F931F93CF93DF93CDB7DEB76297E6
:100F40000FB6F894DEBF0FBECDBF8091820C83FD3B
:100F500099C183E50E94243B8C87811106C082E5FC
:100F60000E94243B882309F48DC10E94A43A0E9468
:100F700024DFCB010E94B33C0E94A43A20E030E081
:100F800040EA50E40E9406E0181614F40E94BD776F
:100F9000E8E4FEE18491FB83EA83882371F0082E64
:100FA000000C990B0E94386F4A815B814F5F5F4F45
:100FB0005B834A83FA018491F0CF8DE090E00E9438
:100FC000386F8AE090E00E94386F81E080932C02B5
:100FD00010929E1580919D158093DB141A821B82BE
:100FE0001C821D82188619861A861B8619821D8608
:100FF000FCE3FE872CE12F8736E4388B312C212C43
:1010000040E8498B5FEB5A8B812C912C5401609105
:10101000440470914504072E000C880B990B0E9424
:101020009AD97B018C019B01AC01632D722D8989BA
:101030009A890E9494D9882341F1209146043091E5
:10104000470440914804509149048C85B7018111AF
:101050000CC0C8010E9494D9881F8827881F8983E3
:101060003E2C2F2C098B1A8B10C0C8010E9494D9DA
:1010700087FF06C0ECE4FEE18491FB83EA83E7C0CE
:101080003E2C2F2C098B1A8B19820E94A5516B01C3
:101090007C01DC01CB01288539854A855B85821B73
:1010A000930BA40BB50BB7FD3BC0D701C60188510C
:1010B0009C4FAF4FBF4F88879987AA87BB870E94F5
:1010C000F674E0E5FEE184913F019FEF691A790A29
:1010D000882321F00E9488C5F301F5CF8114910483
:1010E000A104B104B9F0D501C401805F984DAF4FA0
:1010F000BF4FBC01CD016C197D098E099F0928EEF7
:1011000033E040E050E00E9482DDCA01B9010E9454
:10111000FAC503C08FE30E9488C58AE00E9488C593
:101120000E94099C0E94A55160939F157093A01581
:101130008093A1159093A215A0914604AE83B0911F
:101140004704BF8300914804109149040E94122A69
:101150002E813F81A801632D722D89899A890E9471
:10116000DFDD2B013C0120E030E0A9010E9406E018
:1011700087FF04C077FA709477F870948114910413
:10118000A104B10459F420E030E040E85FE3C3017A
:10119000B2010E9494D987FF0DC00AC020E030E060
:1011A00040E450E4C301B2010E9406E0181614F4B2
:1011B00046015701E981EE2391F12A813B814C815F
:1011C0005D81211531054105510541F0D701C60169
:1011D000821B930BA40BB50BB7FD21C02E813F8161
:1011E000A8016D857E858F8598890E94DFDD20E0CE
:1011F00030E040EC5FE30E9494D987FD3BCFD701FC
:10120000C601805A9541AF4FBF4F8A839B83AC8301
:10121000BD839E819D87AF81AE870F87188B80919C
:101220002C02882309F426CF81149104A104B1046F
:1012300009F4EDCEB0E1CB1AB7E2DB0AE108F10820
:10124000C818D908EA08FB08F7FE14CFE0CE8823B7
:1012500061F0082E000C990B0E94386FEA81FB8127
:101260003196FB83EA838491F2CF8DE090E00E9477
:10127000386F8AE090E00E94386F80912C0281E004
:1012800080939E1562960FB6F894DEBF0FBECDBF59
:10129000DF91CF911F910F91FF90EF90DF90CF9052
:1012A000BF90AF909F908F907F906F905F904F9086
:1012B0003F902F90089590912416E92FF0E0EA5482
:1012C000F54F80839F5F943018F49093241602C0EA
:1012D00010922416809125168F5F8093251608950D
:1012E000CF93FC0120812B33A1F0209125162430CF
:1012F00080F4C62FBC0180912416F0E68F9FC001B8
:1013000011248554954F0E9444E18C2FD4DF81E055
:1013100001C080E0CF9108959F92AF92BF92CF928B
:10132000DF92EF92FF920F931F93CF93DF9387E5A6
:10133000A82E82E0B82E03E116E1C2E3D4E097E1E3
:10134000C92E94E0D92E23E2E22E24E0F22E912C35
:10135000F50181915F010E94DB3A882309F10E9427
:10136000A43AF7012081211104C0209127042223EF
:1013700039F0288139814A815B810E94E0DD0AC011
:10138000F3E09F1639F0F6012081318142815381CB
:101390000E94DFDDF801608371838283938309C03B
:1013A00088819981AA81BB81F80180839183A2837E
:1013B000B38393940C5F1F4F2496F4E0CF0ED11C9F
:1013C0002FEFE21AF20A84E09812C2CF86E40E945C
:1013D000243B8823C9F00E94A43A20E030E0A90110
:1013E0000E9406E0181684F40E94A43A20E030E03F
:1013F00040E752E40E94BCDE6093490270934A02C7
:1014000080934B0290934C02DF91CF911F910F91EB
:10141000FF90EF90DF90CF90BF90AF909F90089596
:10142000EF92FF921F93CF93DF9383E3E82E86E141
:10143000F82E15E0C0E0D0E020E030E0A901F7018F
:10144000EC0FFD1F60817181828193810E9494D98C
:1014500081110CC02496C431D10571F7115084E17B
:10146000E80EF11C1111E6CF80E001C081E0DF91B0
:10147000CF911F91FF90EF900895CF939091E11538
:101480009817C9F0C82F0E94C462C11112C04AE364
:1014900054E066E374E082E394E00E94E6B480E006
:1014A0008093E115882339F082E394E0CF910C9486
:1014B000F450B6DFF5CFCF910895CF92DF92EF923F
:1014C0000F931F93CF93DF93CDB7DEB760970FB61F
:1014D000F894DEBF0FBECDBFE0909D15E2E3F4E0CF
:1014E00080859185A285B385448155816681778108
:1014F000008111812281338109831A832B833C83EC
:101500004D835E836F83788789879A87AB87BC8793
:101510001D861E861F86188AAE01475F5F4FBE017B
:101520006B5F7F4FCE0101960E94E6B4CE010D960F
:101530006C0109E412E02EE334E0AE01475F5F4F37
:10154000BE016B5F7F4F0C970E94A15260960FB651
:10155000F894DEBF0FBECDBFDF91CF911F910F91E9
:10156000EF90DF90CF9008950F931F93CF93DF9369
:1015700094E0899FE00111248E01095E1B4FFE015A
:10158000E655F54FDE01A455BA4E2D913D914D9192
:101590005C9160817181828193810E94E0DDF8011C
:1015A0006083718382839383FE01E75AFD4D8591A9
:1015B0009591A591B491FE01E854FA4E80839183F0
:1015C000A283B383FE01EB59FD4D85919591A591C1
:1015D000B491C35CDD4F88839983AA83BB83DF9179
:1015E000CF911F910F910895EF92FF920F931F9348
:1015F000CF93DF937C0184E50E94243BD82F88237E
:1016000049F10E94843AC82F181604F5EBE9FBE172
:1016100084918F010F5F1F4F882321F00E9488C59E
:10162000F801F6CF8DE40E9488C5B70180E090E014
:101630004AE00E948FC56C2FCC0F770B86E492E2B4
:101640000E94C0508AE00E9488C508C08093DB14C5
:10165000D0E004C080919D158093DB148D2FDF9125
:10166000CF911F910F91FF90EF900895EF92FF920D
:101670001F93CF93DF937C0160E032DE182F882325
:10168000B1F0EBE9FBE18491EF012196882321F091
:101690000E9488C5FE01F7CFB70187EE90E20E9455
:1016A000D95082E20E9488C58AE00E9488C5812FB5
:1016B000DF91CF911F91FF90EF900895DF92EF920D
:1016C000FF920F931F93CF93DF93CDB7DEB76E9743
:1016D0000FB6F894DEBF0FBECDBF60918A0C70913B
:1016E0008B0C6115710541F14DE150E0CE01019681
:1016F0007C010E943DD91E8EF7018F010E191F0932
:10170000D190DD2019F09AE0D912F7CFF701E00F60
:10171000F11F1082C701AADF882371F0DD20A9F034
:101720000F5F1F4F80918A0C90918B0C080F191F2F
:1017300010938B0C00938A0C81E020918A0C3091DD
:101740008B0C232B29F480E003C000E010E0F0CFE5
:101750006E960FB6F894DEBF0FBECDBFDF91CF916E
:101760001F910F91FF90EF90DF9008953F924F925D
:101770005F926F927F928F929F92AF92BF92CF9221
:10178000DF92EF92FF920F931F93CF93DF931F92FD
:10179000CDB7DEB793DF811171C2809125168430F9
:1017A00008F048C00E9485C6AC0197FF7DC142C0C9
:1017B0008E3409F0DAC10115110509F4D6C16AE1C8
:1017C00072E2C8010E944CD97C01892B09F48FC1B7
:1017D0006EE470E0C80104960E9430E1009709F4BD
:1017E00086C14AE050E060E070E001960E94E8D6D1
:1017F00060933015709331158093321590933315A3
:101800008090781790907917A0907A17B0907B17F6
:101810002FEF821A920AA20AB20A681579058A0580
:101820009B0509F466C1EF2809F063C187EE91E2D8
:101830000E94A4C88091180F882309F41FC28091C8
:101840002516811102C010929615EE24E394409162
:101850009211509193116091941170919511809112
:101860008E1190918F11A0919011B0919111481704
:1018700059076A077B0708F4E12C00E010E099247F
:10188000939480E6882E9FE1A92E92E2B92E2DE84E
:10189000322E80912516843008F0F0C1E110EEC19F
:1018A000809196158111EAC18091E9109091EA101A
:1018B000A091EB10B091EC10809392119093931142
:1018C000A0939411B093951141E050E0BE016F5F79
:1018D0007F4F81EE90E10E94D495019719F48981A0
:1018E00090E002C08FEF9FEFF82E40909211509041
:1018F0009311609094117090951140918E115091B8
:101900008F116091901170919111EE24E39444161F
:1019100055066606770608F4E12C44165506660659
:101920007706B0F4019609F469C08AE0F81609F464
:101930008AC09DE0F91609F486C023E2F21619F078
:101940008AE3F81297C080919515811193C070C0F9
:101950000E94C46281EE90E1A7D68091FC1088239A
:1019600051F181508093FC10389EC001112441E058
:1019700061E08F5F9E4E0E9412C7E091FC1094E0E0
:10198000E99FF0011124E350FF4E408151816281B3
:1019900073814093921150939311609394117093BB
:1019A000951181EE90E196D58091190F8823A9F0C9
:1019B0009092180F12C01092180F0E9491B00E94BE
:1019C000DF770E946E776D3371058105910528F0F0
:1019D000B0928B0CA0928A0C71DE8091180F81114D
:1019E0002BC0E2E3F2E284916F012FEFC21AD20A18
:1019F0008823F1F00E9488C5F601F5CFE6E8FBE107
:101A000084916F019FEFC91AD90A882321F00E949F
:101A100088C5F601F5CFE3E2F2E284916F012FEF82
:101A2000C21AD20A882321F00E9488C5F601F5CF98
:101A300083E2F81208C005C023E2F2121CC100E0E4
:101A400010E090929615109295150115110519F454
:101A50000E94B47A0CC080912416889E000D111D3E
:101A60001124F801E554F54F108280E024DC00E0F9
:101A700010E00FCF0F35110508F00BCF9BE3F912E3
:101A800002C09092951580919515811102CF809199
:101A90002416F801889EE00DF11D1124E554F54F40
:101AA000F0820F5F1F4FF5CE982F2091761730915F
:101AB00077178A3019F09D3009F0ABC01092941559
:101AC0002115310519F40E94B47A67CEF901EC5C56
:101AD000FA4E1082109277171092761704E315E1F0
:101AE000F8018191803209F063CE8F01F9CFC801EE
:101AF00078CE6AE270E0C8010E9468E19C0100971C
:101B000001F1982F901BF12C992339F09150F80195
:101B1000E90FF11D8081F826F7CF4AE050E060E040
:101B200070E0C90101960E94E8D6CF2CD12CE12C9F
:101B3000F12C6C157D058E059F0531F088EC91E246
:101B400077CE8EE991E274CE809130159091311567
:101B5000A0913215B091331580937817909379172F
:101B6000A0937A17B0937B170EC08091160F88232D
:101B700051F064EF73E0C8010E943BE1892B19F03A
:101B800084E791E255CE80913302811120C067E451
:101B900070E0C8010E9430E10097C9F04AE050E0CF
:101BA00060E070E001960E94E8D66430710581051E
:101BB000910568F4EDEFF0E284917F019FEFE91A5F
:101BC000F90A882321F00E9488C5F701F5CF68EF54
:101BD00073E0C8010E943BE1892B11F410922C02A2
:101BE0006DEF73E0C8010E943BE1892B21F484EF83
:101BF00090E20E94C29B62E074E0C8010E943BE157
:101C0000892B11F40E942B7F61E084E395E168DB6E
